:100000000C94551B0C94861B0C94861B0C94861B1D
:100010000C94861B0C94861B0C94861B0C94861BDC
:100020000C94861B0C94861B0C94861B0C94861BCC
:100030000C94861B0C94861B0C94861B0C94861BBC
:100040000C94861B0C94979C0C94861B0C94861B1A
:100050000C94861B0C94861B0C9435890C94D574D7
:100060000C94861B0D947F1F0D94751F0C94861B9A
:100070000C94861B0C94861B0C94861B0C94861B7C
:100080000C94ECF50C94861B0C94861B0C94861B2C
:100090000C94861B0C94861B0C94861B0C94861B5C
:1000A0000C94861B0C94861B0C94BEF50C94861B3A
:1000B0000C94861B0C94861B0C94861B0C94861B3C
:1000C0000C94861B0C94861B0C94861B0C94A1F636
:1000D0000C946BF60C94861B0C94861B0C94861B5C
:1000E0000C94861B084AD73B3BCE016E84BCBFFDF7
:1000F000C12F3D6C74319ABD56833DDA3D00C77FF8
:1001000011BED9E4BB4C3E916BAAAABE0000008090
:100110003F05A84CCDB2D44EB93836A9020C50B91F
:10012000918688083CA6AAAA2ABE000000803F004B
:100130000C942B730C9437F70C944CC70C9453C845
:100140000C94DAC70D9425200C9421C80D94192025
:100150000C94DFDB0C9432D60C9441430D941120A7
:100160000C94AB720C9436D70C9445430C94B24566
:100170000C94ABDA0C94C86F0C943FF70C94F0DB42
:100180000C9408C80D941D200C9435C80C9416725C
:100190000C940EF70C94456F0C94C4DA0C9469D748
:1001A0000D94EC1F0C9452F70C94CC720C94ABD7BA
:1001B0000C94A2D50C9413D70C9441C70D94BD1F79
:1001C0000C9454CE0C9425CF0C947A450C94337235
:1001D0000C942CF70C945CC70C94B3DC0C9456C7AD
:1001E0000C9478C70C9410730C94E4C70D941520EC
:1001F0000C94BED70C94ECC70C947CC70C9449C8E3
:100200000C9445C70D94AC260C94C76F0C94F1DA8E
:100210000C94FEDA0C94C6C70C943FC80C9443F7B8
:100220000C94F2420C94DDDA0C943BF70C9464C706
:100230000C944AD70C94D0C70C94FFD60C94D3DA04
:100240000C945DF70C94E8730C9439450D9443209D
:100250000C9433F70C9465F70D943B200C9493DFCA
:100260000C943DD30C941DF70C9406D50C94C1C787
:100270000C944BF70C94BCCA0C942BC80D94FB1F28
:100280000C94A9730C947BDA0C94F4C70C94BB7394
:100290000C946ED80C942BC70C94D6D60C9468D6BC
:1002A0000C946AC70C94A2DA0C943DC70D942920D3
:1002B0000C9426C70C9460C70C94D2D40C940D45B2
:1002C0000C9412C80D9430200C94C2CC0C94DFF620
:1002D0000C94ECCC0C9483D40C94A3D00C94B6D492
:1002E0000D948E260D9421200C94A8DA0C946EC7E0
:1002F0000C9449C70C94B2740C94FEC70C9447F745
:100300000C9452C70C94DDCB0D940A200C9472C748
:100310000C94B9C74E414E494E495459494E46CDA9
:10032000CCCC3D0AD7233C17B7D13877CC2B3295AC
:1003300095E6241FB14F0A000020410000C842008A
:10034000401C4620BCBE4CCA1B0E5AAEC59D740054
:10035000407A10F35A00A0724E18090010A5D4E894
:100360000000E87648170000E40B54020000CA9A27
:100370003B000000E1F50500008096980000004079
:10038000420F000000A086010000001027000000BE
:1003900000E803000000006400000000000A000004
:1003A0000000000100000000002C76D888DC674FB8
:1003B0000823DFC1DFAE59E1B1B796E5E3E453C6E8
:1003C0003AE651997696E8E6C28426EB898C9B62E0
:1003D000ED407C6FFCEFBC9C9F40F2BAA56FA5F48A
:1003E00090055A2AF75C936B6CF9676DC11BFCE0B2
:1003F000E40D47FEF520E6B500D0ED902E03009405
:100400003577050080841E080000204E0A00000099
:10041000C80C333333330F986E12831141EF8D21A3
:1004200014893BE65516CFFEE6DB18D1844B381B0A
:10043000F77C1D901DA4BBE424203284725E2281CF
:1004400000C9F124ECA1E53D27434F4D4D554E49E0
:10045000434154494F4E0044525952554E00455263
:10046000524F525300494E464F004543484F004FAC
:100470004646004F4E0020204D61783A2000200073
:1004800020204D696E3A2000536F667420656E64BB
:1004900073746F70733A20003D3D4F6E506F7765F7
:1004A000724C6F7373526573756D653D3D004D32CF
:1004B000342053256C642054256C64004739322E57
:1004C00039204525730047312046256400473932DD
:1004D0002E39205A2573004731205A3020463230B9
:1004E000300047312058257320592573204633307A
:1004F0003030004D34323020532569205A257300A6
:100500004D3130362050256920532569004D323059
:10051000302044257300473238523058590047394B
:10052000322E39204530205A300A47315A2573007F
:100530004D31303920532569004D31393020532554
:1005400069004D343230205330205A300020496E3B
:1005500076616C69642065787472756465722000D8
:1005600047322F47332062616420706172616D658C
:10057000746572730A00536C6565702E2E2E005AD6
:100580002050726F62652050617374204265640A66
:10059000005A2050726F626520506173742042656A
:1005A00064004732384C30004D3131372050726F83
:1005B0006265206661696C65642E0A4732380A00FC
:1005C00070726F62655F7265776970650047323976
:1005D000205265747279696E670050726F62696E3D
:1005E00067204661696C6564004D31313720426592
:1005F00064206C6576656C696E67206661696C6500
:10060000642E0A4730205A31300A4D3330302050A2
:10061000323520533838300A4D33303020503530A1
:100620002053300A4D333030205032352053383883
:10063000300A4D333030205035302053300A4D339E
:1006400030302050323520533838300A4D33303076
:10065000205035302053300A473420533100707217
:100660006F62655F6661696C6564004D313137208A
:10067000426564206C6576656C696E6720646F6E98
:10068000652E00205A3A200020593A200042656425
:1006900020583A20004D65736820706F696E742091
:1006A0006F7574206F662072616E67650A004D3049
:1006B0002053746F70004D312053746F7000436F7E
:1006C0006E74696E756500436C69636B20746F208E
:1006D000526573756D652E2E2E004E6F204D6F7610
:1006E000652E00456E642066696C65206C697374C4
:1006F0000A00426567696E2066696C65206C6973E3
:10070000740A004E6F206D656469610A005265735A
:10071000756D696E6720534400286E6F2066696CA2
:1007200065290043757272656E742066696C653A5E
:1007300020005072696E742074696D653A20000A59
:1007400053746174733A2046696C616D656E7420F0
:10075000757365643A20002C204C6F6E6765737466
:10076000206A6F623A2000546F74616C2074696D66
:10077000653A200053746174733A20002C2046615E
:10078000696C65643A20002C2046696E697368655F
:10079000643A20005072696E74733A200053746199
:1007A00074733A2000436F6F6C696E672E2E2E00B3
:1007B00048656174696E672E2E2E00452025530012
:1007C0006F6B006F6666006A0465045E0457044937
:1007D0000444454255473A004D31313320530042DD
:1007E000656420436F6F6C696E672E2E2E00426524
:1007F000642048656174696E672E2E2E00544D3357
:100800004420453520506C7573204F46462E002FEE
:100810002F00205200416363656C65726174696FDB
:100820006E3A2050004D32303620580046523A0081
:1008300020466C6F773A20003A200020536572768C
:100840006F2000206F7574206F662072616E67657F
:100850000A00536572766F200020643A0020693ADE
:100860000020703A00496E76616C69642065787486
:1008700072756465720A0020643A0020693A0020AB
:10088000703A0064697300656E0043290A00616272
:100890006C656420286D696E2074656D702000435E
:1008A0006F6C64206578747275646573206172651D
:1008B0002000504944204175746F74756E65005076
:1008C0004944204175746F74756E65206661696C6A
:1008D00065642120426164206865617465722069E5
:1008E000640A0046696C616D656E742072756E6F86
:1008F00075742064697374616E636520286D6D2959
:100900003A200046696C616D656E742072756E6F79
:10091000757420004D34323120696E636F727265D8
:10092000637420706172616D6574657220757361A6
:1009300067650A004D65736820706F696E74206F7B
:100940007574206F662072616E67650A004F666677
:1009500073657473204170706C69656400457272D0
:100960003A20546F6F206661722100546F6F2066C9
:1009700061722066726F6D207265666572656E6366
:100980006520706F696E740A00454550524F4D20C6
:100990004F4B0A00506F7765722D6C6F7373207226
:1009A00065636F7665727920004D383400446F6E50
:1009B00065207072696E74696E672066696C650A7D
:1009C000004D3737004D3331004361703A004D45DB
:1009D00041545041434B00434F4F4C45525F5445A7
:1009E0004D5045524154555245004348414D4245B2
:1009F000525F54454D504552415455524500424175
:100A000042595354455050494E47004152435300B8
:100A10004D4F54494F4E5F4D4F4445530054484548
:100A2000524D414C5F50524F54454354494F4E0034
:100A30004C4F4E475F46494C454E414D4500415550
:100A4000544F5245504F52545F53445F5354415496
:100A500055530053445F5752495445005245504541
:100A60004154005344434152440050524F4D50545E
:100A70005F535550504F525400454D455247454ED7
:100A800043595F50415253455200434153455F4CD7
:100A9000494748545F4252494748544E45535300D2
:100AA000544F47474C455F4C494748545300534FB8
:100AB0004654574152455F504F57455200425549A1
:100AC0004C445F50455243454E54004C4556454CAE
:100AD000494E475F44415441005A5F50524F42458E
:100AE0000052554E4F5554004155544F4C455645B4
:100AF0004C005052494E545F4A4F420050524F47AB
:100B000052455353004155544F5245504F52545F34
:100B100054454D5000564F4C554D45545249430095
:100B2000454550524F4D0042494E4152595F46494A
:100B30004C455F5452414E5346455200534552492D
:100B4000414C5F584F4E5F584F4646004649524D04
:100B5000574152455F4E414D453A4D61726C696E49
:100B600020322E302E375F4457372E3320544D33EA
:100B70004420453550534D44424220284170722054
:100B8000323420323032312032303A35313A343456
:100B90002920534F555243455F434F44455F5552BB
:100BA0004C3A68747470733A2F2F67697468756271
:100BB0002E636F6D2F496E73616E69747941757420
:100BC0006F6D6174696F6E2F4D61726C696E2F74F9
:100BD0007265652F437265616C6974794477696EDB
:100BE0005F322E302050524F544F434F4C5F56458A
:100BF0005253494F4E3A312E30204D414348494ED1
:100C0000455F545950453A544D33442045352050A2
:100C10006C75732045585452554445525F434F55A7
:100C20004E543A3120555549443A63656465326102
:100C300032662D343161322D343734382D396231FA
:100C4000322D6335356336326633363766660A00D1
:100C500050726F6265204F6666736574205A00504B
:100C6000726F6265204F6666736574205A00290AA8
:100C70000020746F20003F5A206F7574206F66202B
:100C800072616E6765202800290A0020746F2000B9
:100C90003F59206F7574206F662072616E67652002
:100CA000282D00290A0020746F20003F58206F75FE
:100CB00074206F662072616E676520282D00507267
:100CC0006F6265204F666673657420580043616EDD
:100CD0006E6F74206F70656E207375626469722028
:100CE000002569730025696D2025697300256968F1
:100CF0002025696D202569730025696420256968B0
:100D00002025696D2025697300256979202569648E
:100D1000202569682025696D20256973003D3D44C3
:100D200077696E20496E697420436F6D706C6574CD
:100D3000653D3D002A2A2A4E6F7A7A6C6554656DAE
:100D4000705374617475735B325D203D003D3D48A6
:100D5000656174696E6720446F6E65204368616EDB
:100D600067652046696C616D656E743D3D002020AD
:100D7000737461727470726F677265737320003D73
:100D80003D7761697477617920353D3D003D3D7760
:100D900061697477617920343D3D003D3D7761693B
:100DA0007477617920333D3D003D3D77616974770B
:100DB000617920313D3D003D3D6F6E5072696E742A
:100DC00054696D657253746F707065643D3D003D8C
:100DD0003D6F6E466163746F727952657365743DE1
:100DE0003D00270A0A0000272027002027002D00A9
:100DF0006E6F74696669636174696F6E2000636108
:100E00006E63656C005072696E742041626F72741B
:100E10006564004469736D697373005549204162CC
:100E20006F7274656400726573756D65004D323460
:100E3000002A2A2A43506C617920546F6E652A2A51
:100E40002A003D3D6F6E5072696E7454696D657213
:100E50005061757365643D3D00486F6D696E672034
:100E60004661696C6564006F70656E005452494755
:100E70004745524544003A200066696C616D656ED5
:100E800074007A5F6D696E00795F6D617800785FDC
:100E90006D6178005265706F7274696E6720656E5F
:100EA0006473746F70207374617475730A002074B6
:100EB0006F6F206C6F6E6720657874727573696FE1
:100EC0006E2070726576656E7465640A0020636FCB
:100ED0006C6420657874727573696F6E20707265CA
:100EE00076656E7465640A00486F6D65202573250C
:100EF000732573204669727374005761726E696E50
:100F0000673A20486F6D696E672042756D702044A6
:100F1000697669736F72203C20310A000202040076
:100F200000B4430000B443000000000000B44300DC
:100F300000B4430000C8430000004100000041002D
:100F40000000400101FF000000010000000100005E
:100F50008000555555000000400033333300AAAAE5
:100F60002A004992240000002000C7711C009999B2
:100F70001900D1451700555515003BB11300244900
:100F8000120011111100000010000F0F0F00E338C4
:100F90000E0043790D00CCCC0C00C3300C00E8A24D
:100FA0000B0064210B00AAAA0A00703D0A009DD81C
:100FB0000900427B090092240900DCD308008888DC
:100FC00008001042080000000800F0C107008787F1
:100FD000070075500700711C07003EEB0600A1BC1E
:100FE00006006990060066660600703E06006118FD
:100FF000060017F4050074D105005BB00500B2903F
:101000000500627205005555050078390500B81EC7
:101010000500050505004EEC040087D40400A1BDC1
:10102000040090A7040049920400C17D0400EE6909
:101030000400C7560400444404005C320400082144
:10104000040041100400000004003FF00300F8E039
:10105000030026D20300C3C30300CCB503003AA8A3
:1010600003000A9B0300388E0300C08103009F75B4
:101070000300D0690300505E03001D530300344891
:101080000300913D03003333030016290300381F8A
:10109000030097150300300C0300030303000BFA51
:1010A000020049F10200BAE802005CE002002DD81B
:1010B00002002DD0020059C80200B0C0020031B9B0
:1010C0000200DAB10200AAAA0200A0A30200BC9C9E
:1010D0000200FA9502005C8F0200DF880200828223
:1010E0000200457C02002776020027700200436A56
:1010F00002007C640200D05E02003F590200C85327
:101100000200FFFDFCFAF8F6F4F2F0EEECEAE9E793
:10111000E5E3E1E0DEDCDAD9D7D5D4D2D0CFCDCB50
:10112000CAC8C7C5C3C2C0BFBDBCBAB9B7B6B4B3DD
:10113000B2B0AFADACAAA9A8A6A5A4A2A1A09E9D3D
:101140009C9A99989795949392908F8E8D8B8A897B
:1011500088878684838281807F7E7D7B7A79787799
:10116000767574737271706F6E6D6C6B6A69686797
:10117000666564636261605F5E5D5C5B5A59585886
:101180005756555453525150504F4E4D4C4B4A4A5E
:101190004948474646454443424241403F3E3E3D22
:1011A0003C3B3B3A393838373635353433323231D7
:1011B00030302F2E2E2D2C2B2B2A2929282727267D
:1011C000252524232322212120201F1E1E1D1C1C17
:1011D0001B1B1A19191818171616151514131312A4
:1011E000121111100F0F0E0E0D0D0C0C0B0A0A0927
:1011F000090808070706060505040403030202019F
:1012000000003D3D6F6E5072696E7454696D657279
:10121000537461727465643D3D000000B443000086
:10122000B4430000C84300000000000000000000BC
:1012300000003D3D6F6E53746F7265536574746941
:101240006E67733D3D003D3D6F6E436F6E6669672F
:1012500075726174696F6E53746F726557726974D9
:1012600074656E3D3D0053657474696E67732053F9
:10127000746F726564000A20696E6974207A7072F6
:101280006F62655F7A6F6666736574203D20003D0E
:101290003D6F6E436F6E66696775726174696F6EDC
:1012A00053746F7265526561643D3D00454550520F
:1012B0004F4D20496E697469616C697A65640A00F2
:1012C0003B20003A0A0020204D36303320002044D5
:1012D0000020204D34313220530046696C616D6529
:1012E0006E742072756E6F75742073656E736F7295
:1012F0003A002055004C0046696C616D656E7420A3
:101300006C6F61642F756E6C6F6164206C656E67C5
:101310007468733A0020204D3835312058005A2D1A
:1013200050726F6265204F66667365740020204DB1
:10133000343133205300506F7765722D4C6F7373C7
:10134000205265636F766572793A00204400204927
:101350000020204D3330342050002044002049002C
:1013600020204D33303120500050494420736574A3
:1013700074696E67733A00204A0020204732392092
:101380005720490020204D343230205300417574DD
:101390006F20426564204C6576656C696E673A0023
:1013A00020204D323036205800486F6D65206F6622
:1013B000667365743A0020580020530020204D3297
:1013C0003035204200416476616E6365643A2042A4
:1013D0003C6D696E5F7365676D656E745F74696D92
:1013E000655F75733E20533C6D696E5F666565642D
:1013F000726174653E20543C6D696E5F74726176F3
:10140000656C5F66656564726174653E20583C6D0D
:1014100061785F785F6A65726B3E20593C6D6178D8
:101420005F795F6A65726B3E205A3C6D61785F7AC6
:101430005F6A65726B3E20453C6D61785F655F6AEF
:1014400065726B3E0020540020520020204D323047
:1014500034205000416363656C65726174696F6E1E
:101460002028756E6974732F7332293A20503C70AE
:1014700072696E745F616363656C3E20523C726595
:1014800074726163745F616363656C3E20543C7485
:10149000726176656C5F616363656C3E0020204D10
:1014A0003230312058004D6178696D756D2041638F
:1014B00063656C65726174696F6E2028756E6974FE
:1014C000732F7332293A0020204D323033205800D8
:1014D0004D6178696D756D206665656472617465CE
:1014E000732028756E6974732F73293A00537465DD
:1014F00070732070657220756E69743A0020440024
:1015000020204D3230302053002044697361626CDA
:1015100065640A0046696C616D656E74207365745C
:1015200074696E67733A0020286D6D29002020478A
:101530003231202020203B20556E69747320696E63
:10154000206D6D003D3D6F6E4C6F6164536574742A
:10155000696E67733D3D0000803B4400803B440062
:10156000002041000096420000A0420000A042007E
:101570000048440000BE42D0070000D007000064CD
:101580000000004B00000024F4D43050C38E20C271
:10159000A24017828B7011127A910D816CD90AA822
:1015A00061E108C7586607615143061E4B5D05C1DE
:1015B00045A7041A411104093D98037139310340CC
:1015C00036DB0265339102D4305402802E1D026353
:1015D0002CEE01752AC501B028A001102781018FCA
:1015E0002564012B244B01E0223401AC211F018D25
:1015F000200D01801FFC00841EED00971DDF00B848
:101600001CD200E61BC600201BBC00641AB200B24C
:1016100019A8000A19A0006A189900D11791004072
:10162000178B00B516840031167E00B31579003A89
:10163000157300C7146F0058146A00EE1366008813
:1016400013630025135E00C7125B006C1257001570
:10165000125400C111510070114F0021114B00D6DE
:101660001049008D1047004610440002104200C08F
:101670000F4000800F3E00420F3C00060F3B00CBA6
:101680000E3800930E37005C0E3500270E3400F341
:101690000D3200C10D3100900D3000600D2E003272
:1016A0000D2D00050D2C00D90C2B00AE0C2900854A
:1016B0000C29005C0C2700350C27000E0C2600E8D6
:1016C0000B2400C40B2400A00B23007D0B23005A25
:1016D0000B2100390B2100180B2000F80A1F00D93C
:1016E0000A1E00BB0A1E009D0A1D00800A1D006321
:1016F0000A1C00470A1B002C0A1B00110A1A00F7DB
:10170000091A00DD091900C4091900AB0919009272
:101710000917007B091800630917004C09160036E9
:10172000091600200916000A091500F5081500E041
:10173000081400CC081400B8081400A40814009081
:101740000813007D0812006B0813005808120046A9
:1017500008120034081100230811001208110001BA
:10176000081100F0071000E0071000D0071000C0BB
:10177000071000B0070F00A107100091070E0083AB
:10178000070F0074070F0065070E0057070E00498A
:10179000070E003B070D002E070E0020070D00135B
:1017A000070D0006070D00F9060C00ED060D00E020
:1017B000060C00D4060C00C8060C00BC060C00B0D9
:1017C000060C00A4060B0099060C008D060B008287
:1017D000060B0077060B006C060B0061060A00572B
:1017E000060B004C060A0042060A0038060A002EC4
:1017F000060A0024060A001A060A00100609000755
:10180000060A00FD050900F4050900EB050900E2E0
:10181000050900D9050900D0050900C7050900BE62
:10182000050900B5050800AD050800A50509009CDF
:10183000050800940508008C050800840508007C54
:10184000050800740508006C050700650508005DC3
:10185000050700560508004E05070047050700402C
:1018600005080038050700310507002A0507002391
:101870000507001C050600160507000F05070008F0
:1018800005060002050700FB040600F5040700EE4C
:10189000040600E8040600E2040700DB040600D5A5
:1018A000040600CF040600C9040600C3040600BDF8
:1018B000040600B7040600B1040500AC040600A647
:1018C000040600A00405009B040600950405009092
:1018D0000406008A04050085040500800406007AD9
:1018E00004050075040500700405006B040500661E
:1018F000040500610405005C04050057040500525E
:101900000405004D04050048040500430405003E9D
:101910000404003A04050035040500300404002CDA
:1019200004050027040400230405001E0404001A13
:1019300004040016040500110404000D0404000949
:101940000405000404040000040400FC030400F87F
:10195000030400F4030400F0030400EC030400E8B3
:10196000030400E4030400E0030400DC030400D8E3
:10197000030400D4030400D0030400CC030400C813
:10198000030300C503030024F404D9201BC40C5C2A
:101990000E9804C4095F0265077101F405F900FBA4
:1019A00004B30048048700C10369005803550003CD
:1019B000034500BE023A008402310053022A002986
:1019C00002250004022000E4011C00C8011900AF38
:1019D00001170098011400840113007101100061C7
:1019E00001100051010E0043010D0036010B002BC8
:1019F000010B0020010B00150109000C0109000377
:101A0000010800FB000800F3000800EB000700E4F9
:101A1000000600DE000600D8000600D2000600CC5A
:101A2000000500C7000500C2000500BD000400B9A4
:101A3000000400B5000400B1000400AD000400A9DA
:101A4000000400A5000300A20003009F0004009B07
:101A5000000300980003009500020093000300902B
:101A60000003008D0002008B000300880002008646
:101A700000020084000300810002007F0002007D5C
:101A80000002007B0002007900020077000100766E
:101A90000002007400020072000100710002006F79
:101AA0000002006D0001006C0002006A0001006984
:101AB000000200670001006600010065000100648B
:101AC0000002006200010061000100600001005F8F
:101AD0000002005D0001005C0001005B0001005A93
:101AE0000001005900010058000100570001005694
:101AF0000001005500010054000100530000005394
:101B00000001005200010051000100500001004F8F
:101B10000001004E0000004E0001004D0001004C8D
:101B20000001004B0000004B0001004A0001004989
:101B30000001004800000048000100470001004685
:101B4000000000460001004500000045000100447F
:101B50000001004300000043000100420000004279
:101B60000001004100000041000100400001003F71
:101B70000000003F0001003E0000003E0001003D6B
:101B80000000003D0001003C0000003C0000003C63
:101B90000001003B0000003B0001003A0000003A59
:101BA0000001003900000039000100380000003851
:101BB0000000003800010037000000370001003647
:101BC000000000360000003600010035000000353E
:101BD0000000003500010034000000340000003433
:101BE0000001003300000033000000330001003228
:101BF000000000320000003200010031000000311E
:101C00000000003100010030000000300000003012
:101C10000001002F0000002F0000002F0000002F07
:101C20000001002E0000002E0000002E0001002DFB
:101C30000000002D0000002D0000002D0001002CF0
:101C40000000002C0000002C0000002C0001002BE4
:101C50000000002B0000002B0000002B0001002AD8
:101C60000000002A0000002A0000002A00010029CC
:101C700000000029000000290000002900000029C0
:101C800000010028000000280000002800000028B3
:101C900000000028000100270000002700000027A6
:101CA0000000002700000027000100260000002699
:101CB000000000260000002600000026000100258C
:101CC0000000002500000025000000250000002580
:101CD0000000002500010024000000240000002472
:101CE0000000002400000024000100230000002365
:101CF0000000002300000023000000230000002358
:101D00000000002300010022000000220000002249
:101D1000000000220000002200000022000100213B
:101D2000000000210000002100000021000000212F
:101D30000000002100000021000100200000002020
:101D40000000002000000020000000200000002013
:101D500000000020000000200001001F0000001F04
:101D60000000001F0000001F0000001F0000001FF7
:101D70000000001F0001001E0000001E0000001EE9
:101D80000000001E000000393000003325000087ED
:101D9000190000B00F0000DB080000BD0400007453
:101DA0000200003F01000020436F756E7420583A16
:101DB0000023646566696E652044454641554C5470
:101DC0005F0000626564004B6420004B6920004B9B
:101DD000702000504944204175746F74756E652001
:101DE00066696E6973686564212050757420746833
:101DF00065206C617374204B702C204B6920616EE0
:101E000064204B6420636F6E7374616E747320661C
:101E1000726F6D2062656C6F7720696E746F2043FE
:101E20006F6E66696775726174696F6E2E680A00FD
:101E3000504944204175746F74756E652066616900
:101E40006C6564212074696D656F75740A00504972
:101E500044204175746F74756E65206661696C65A8
:101E600064212054656D70657261747572652074AB
:101E70006F6F20686967680A00204B643A20002071
:101E80004B693A2000204B703A200020436C61736C
:101E900073696320504944200A00204E6F206F76FA
:101EA000657273686F6F740A002054753A200020C1
:101EB0004B753A2000206D61783A2000206D696EE4
:101EC0003A200020643A200020626961733A2000C1
:101ED000504944204175746F74756E652073746148
:101EE00072740A00504944204175746F74756E65B0
:101EF000206661696C6564212054656D706572614E
:101F00007475726520746F6F20686967680A004293
:101F1000656400453100626564002C207379737438
:101F2000656D2073746F70706564212048656174FD
:101F300065725F49443A200048656174696E6720A4
:101F40004661696C65640048656174696E67206606
:101F500061696C6564004D31313220536875746479
:101F60006F776E001000C90210012C0140012201A0
:101F700070011801B0010E01F00104015002FA00D5
:101F8000B002F0003003E600D003DC009004D20081
:101F90007005C800A006BE000008B400B009AA0081
:101FA000D00BA000600E960060118C00001582001E
:101FB00020197800C01D6E00A0226400B0275A00CE
:101FC000902C500000314600E0343C0010383200C4
:101FD000903A2800603C1E00A03D1400803E0A009C
:101FE000203F0000544845524D414C2052554E412F
:101FF00057415900546865726D616C2052756E616D
:10200000776179004572723A204D415854454D50E0
:10201000004D415854454D50207472696767657290
:102020006564004572723A204D494E54454D50004A
:102030004D494E54454D502074726967676572650D
:102040006400202F002042403A0020403A002057F0
:102050003A0020573A00496E76616C6964206578D1
:102060007472756465720A007C3C3E5E2B3D3F2FA6
:102070005B5D3B2C2A225C0043616E6E6F74206FA7
:1020800070656E2073756264697220005344204944
:102090006E6974204661696C005344206361726408
:1020A000206F6B0A006F70656E526F6F74206661EF
:1020B000696C65640A00766F6C756D652E696E6972
:1020C00074206661696C65640A004E6F2053442079
:1020D000636172640A000A4D3234004D32332025A8
:1020E00073002E0A006F70656E206661696C65640E
:1020F0002C2046696C653A200046696C6520736542
:102100006C65637465640A002053697A653A20003F
:1021100046696C65206F70656E65643A2000454EB7
:102120004420535542524F5554494E450A002220EF
:10213000706F73002220706172656E743A220053D2
:102140005542524F5554494E452043414C4C207402
:1021500061726765743A220053756263616C6C202A
:102160004F766572666C6F77004578636565646568
:1021700064206D617820535542524F5554494E4565
:102180002064657074683A002E0A0044656C6574BA
:10219000696F6E206661696C65642C2046696C65A8
:1021A0003A200046696C652064656C657465643A24
:1021B000005344207072696E74696E67206279748E
:1021C0006520004E6F74205344207072696E7469EC
:1021D0006E670A0057726974696E6720746F2066B3
:1021E000696C653A2000667265736800646F696E99
:1021F00067002066696C653A20004E6F7720002FDB
:102200006175746F25632E67002020506C616E6EBF
:10221000657242756666657242797465733A20002C
:102220002046726565204D656D6F72793A200043D6
:102230006F6D70696C65643A204170722032342091
:10224000323032310A00204C617374205570646161
:102250007465643A20323032312D30342D313820DB
:102260007C20417574686F723A2054696E794D61B3
:102270006368696E657333440A00322E302E375F0F
:102280004457372E330A004D61726C696E0020533B
:102290006F6674776172652052657365740A0020F9
:1022A0005761746368646F672052657365740A00D0
:1022B0002042726F776E206F75742052657365745B
:1022C0000A002045787465726E616C2052657365F2
:1022D000740A00506F77657255700A0073746172EA
:1022E000740A004732385859004D3130303100659A
:1022F00072726F722077726974696E6720746F20D2
:1023000066696C650A00446F6E6520736176696E5C
:10231000672066696C652E0A004D323900456E648F
:1023200073746F7073002553202563202563202567
:102330006320256300205A3A0020593A0020583A79
:1023400000656E6473746F7073206869743A20005E
:102350006001F4017001EA019001E001B001D601D1
:10236000D001CC010002C2013002B8016002AE010E
:102370009002A401D0029A0120039001700386010B
:10238000C0037C0130047201A004680120055E01D5
:10239000B005540160064A0120074001F0073601EC
:1023A000F0082C01100A2201500B1801C00C0E017C
:1023B000500E04013010FA002012F0005014E60014
:1023C000C016DC007019D200501CC800501FBE009F
:1023D0007022B400B025AA00F028A000202C96009E
:1023E000302F8C0010328200A0347800F0366E005E
:1023F000E0386400803A5A00403B5500E03B500012
:10240000F03C4600C03D3C00603E3200E03E28000B
:10241000303F1E00503F1900703F1400A03F0A00DB
:10242000C03F0000D03FF6FFE03FECFF00000A0B8A
:1024300002090C0D0E080703040100000000000053
:10244000000000000000000000000000000000008C
:102450000000000000000000121110000000000049
:10246000000000000000000000000000000000006C
:10247000000050726F62696E67204661696C656426
:1024800000205A3A200020593A2000426564205822
:102490003A20003D3D6F6E55736572436F6E6669FD
:1024A000726D52657175697265643D3D00220A0066
:1024B000556E6B6E6F776E20636F6D6D616E643AF3
:1024C0002022002042002050006F6B002045002099
:1024D0005A00205900204D393220580020453A003A
:1024E000205A3A0020593A00583A0020746F6F2061
:1024F0006C6F6E6720657874727573696F6E20708B
:10250000726576656E7465640A0020636F6C642082
:10251000657874727573696F6E2070726576656E1A
:102520007465640A0043616E6E6F7420656E746535
:1025300072207375626469723A20004D3235205002
:102540000A4D323400526573756D6500554920504F
:1025500061757365004E6F204D61746368203A00A9
:1025600050675570005067446F776E00497320467E
:10257000696C6520004973204469722000476F55DB
:102580007044697200486173204D6564696100465A
:10259000696C656E616D652053656C656374656417
:1025A000004D3130303043004D313030300046691D
:1025B0006C616D656E7420537461742030202D2021
:1025C000330046696C616D656E74205374617420CC
:1025D00030202D20320046696C616D656E74205389
:1025E0007461742030202D2031002046696C616DAB
:1025F000656E7420526573706F6E7365204E6F0048
:10260000526573756D652059657320647572696EC6
:1026100067207072696E74000A204E6F2046696CE4
:10262000616D656E7400496E76616C6964204F70EF
:1026300074696F6E004D3530300053746F726520D1
:1026400053657474696E6773004265642050494431
:102650002053746172746564004D3939390A4D3202
:10266000383050305331363000424C546F75636807
:10267000205265736574004D3530320A4D35303067
:1026800000496E697420454550524F4D00486F74A3
:10269000656E64205049442053746172746564000F
:1026A000456E676C69736820416C7265616479205E
:1026B000536574004368696E657365204E6F7420BE
:1026C000537570706F7274656400496E4C616E670B
:1026D00043686F696365000A202A2A2A7265636469
:1026E00061742E646174615B305D203D0047323857
:1026F0000A4731204631303030205A313000556E93
:10270000737570706F72746564204F7074696F6E4A
:102710002053656C65637465640047323652323508
:1027200035004D3139305335350A4732380A473391
:102730003449380A4732390A4D3430300A4D313085
:1027400034533231350A4732380A4D313039533239
:1027500031350A4D34323053310A47315831303037
:102760005931303046353030300A47315A300A4D11
:102770003530300A4D31313720536574205A204F9F
:102780006666736574004731204631303030205A18
:10279000302E30004732380A473120463130303051
:1027A000205A302E30004D353030005A204F6666AA
:1027B000736574203A202573004D353030005A205F
:1027C0004F6666736574203A202573004732380AD5
:1027D000473146313530305A302E30004732385A82
:1027E0000A473146313530305A302E30004D3834BA
:1027F00000473146313030305A302E3000473238C1
:102800000A473146313030305A302E30004D616E3B
:1028100075616C53657454656D70005A204F66661F
:10282000736574203A2025730053746F70205472BE
:10283000696767657265640053746F70204E6F003E
:1028400053746F705072696E740048616E646C6589
:1028500020446174612041646A757374203220538E
:10286000657474696E672053637265656E200048F5
:10287000616E646C652044617461205072696E748D
:1028800046696C6520332053657474696E67205304
:10289000637265656E200048616E646C65204461FA
:1028A0007461205072696E7446696C6520322053E1
:1028B000657474696E672053637265656E20004DA0
:1028C00038340048616E646C652044617461205046
:1028D00072696E7446696C6520506F73740048614C
:1028E0006E646C652044617461205072696E744638
:1028F000696C652050726500426567696E5377693F
:10290000746368003D3D20436865636B6B65793D8A
:102910003D007265636461742E61646472203D3DA4
:10292000007265636461742E646174615B305D2064
:102930003D3D0077616974776179203D3D0020203D
:102940002A2A2A2A2A2A2A5254535F48616E646C22
:1029500065446174612A2A2A2A2A2A2A2A200052D6
:102960006573656E643A200000002200250028008F
:102970002B002E0031003400020100000501080187
:102980000B0100002100240027002A002D00300048
:10299000330001010000040107010A0105050505D6
:1029A000070508080808020202020A0A08080404C7
:1029B00004040101010101010101030303030303F5
:1029C0000303040707070C0C0C0C0C0C0C0C020284
:1029D000020206060606060606060B0B0B0B0B0B81
:1029E0000B0B01021020200808102040102040800E
:1029F00002010201080402010102040810204080C3
:102A00008040201008040201800402018040201050
:102A10000804020108040201010204081020408099
:102A20000102040810204080544D334420453520D5
:102A3000506C75732052656164792E005072696E16
:102A400074696E672E2E2E005072696E742050616C
:102A500075736564006E6F74696669636174696F2C
:102A60006E20005049442054756E652046696E6999
:102A700073686564004572726F7220777269746959
:102A80006E6720746F20454550524F4D210A005308
:102A9000544F505045442E20005072696E74657238
:102AA0002073746F707065642064756520746F2086
:102AB0006572726F72732E20466978207468652083
:102AC0006572726F7220616E6420757365204D3976
:102AD000393920746F20726573746172742E2028E6
:102AE00054656D70657261747572652069732072CA
:102AF000657365742E205365742069742061667453
:102B000065722072657374617274696E67290A0058
:102B10004E6F20436865636B73756D2077697468C9
:102B2000206C696E65206E756D6265722C204C613B
:102B30007374204C696E653A20004E6F20436865BF
:102B4000636B73756D2077697468206C696E65209E
:102B50006E756D6265722C204C617374204C696EC9
:102B6000653A2000636865636B73756D206D6973EA
:102B70006D617463682C204C617374204C696E65C0
:102B80003A20004C696E65204E756D626572206951
:102B900073206E6F74204C617374204C696E6520D5
:102BA0004E756D6265722B312C204C617374204C14
:102BB000696E653A20004D313130005365726961AC
:102BC0006C20737461747573206D69736D617463C7
:102BD000680A00776169740A005344207265616471
:102BE000206572726F720A002121204B494C4C20E3
:102BF00063617573656420627920746F6F206D75F1
:102C0000636820696E6163746976652074696D65B7
:102C1000202D2063757272656E7420636F6D6D6117
:102C20006E643A2000486F74656E642049646C6578
:102C30002054696D656F757400486F74656E64200B
:102C400049646C652054696D656F75740A003D3D7B
:102C50006F6E46696C616D656E7452756E6F7574DA
:102C60003D3D007061757365004D36303000206663
:102C7000696C616D656E745F72756E6F757420003E
:102C800066696C616D656E745F72756E6F757420C8
:102C9000540046696C616D656E7452756E6F757423
:102CA0002054002A2A2A496E6974696E672063617C
:102CB0007264206973204F4B2A2A2A004D6564698B
:102CC0006120496E736572746564004D6564696165
:102CD0002052656D6F766564004D313030305300A1
:102CE000627573793A2070617573656420666F72DE
:102CF00020696E7075740A00627573793A2070618C
:102D00007573656420666F7220757365720A006260
:102D10007573793A2070726F63657373696E670AB1
:102D2000002A2A2A6B696C6C2A2A2A00706F776540
:102D3000726F6666004B494C4C45442E2000507221
:102D4000696E7465722068616C7465642E206B69AD
:102D50006C6C28292063616C6C6564210A005354F3
:102D60004F505045442E20005072696E7465722099
:102D700073746F707065642064756520746F20656E
:102D800072726F72732E20466978207468652065B0
:102D900072726F7220616E6420757365204D3939CF
:102DA0003920746F20726573746172742E202854F8
:102DB000656D7065726174757265206973207265E6
:102DC0007365742E20536574206974206166746580
:102DD000722072657374617274696E67290A006586
:102DE00063686F3A004572726F723A0042696C69AB
:102DF0006E656172204C6576656C696E67204772FE
:102E000069643A0A0021212053544F502063616CB9
:102E10006C65642062656361757365206F6620422E
:102E20004C546F756368206572726F72202D20722A
:102E30006573746172742077697468204D3939390B
:102E40000A0021212053544F502063616C6C65644B
:102E50002062656361757365206F6620424C546F14
:102E6000756368206572726F72202D2072657374AD
:102E70006172742077697468204D3939390A002FDE
:102E80002F616374696F6E3A0070726F6D70745F5A
:102E900000656E640053656E64204D3130382074D7
:102EA0006F20726573756D650A00496E7365727483
:102EB0002066696C616D656E7420616E6420736557
:102EC0006E64204D3130380A0052656865617420A7
:102ED00066696E69736865642E0052656865617421
:102EE00020446F6E6500526568656174696E672E77
:102EF0002E2E0052656865617400486561746572C4
:102F00002054696D656F75740053656E64204D3192
:102F1000303820746F2068656174206E6F7A7A6C27
:102F2000650A004E6F7A7A6C65205061726B656439
:102F300000486F74656E6420746F6F20636F6C64FB
:102F40000A007061757365640050617573650044B3
:102F5000697361626C6552756E6F7574005075723D
:102F600067654D6F726500506175736564007368C5
:102F70006F7700627574746F6E00626567696E00CA
:102F80004C6F61642046696C616D656E74004C6FB6
:102F900061642046696C616D656E74205400496EF1
:102FA000736572742066696C616D656E7420616E04
:102FB000642073656E64204D3130380A0072657389
:102FC000756D656400526573756D696E6700576154
:102FD0006974696E6720666F7220686561747570C8
:102FE0002E0A004C656176696E6720473236003FD5
:102FF00053706563696669656420582C5920636F56
:103000006F7264696E617465206F7574206F6620DD
:10301000626F756E64732E0A003F285229657065D1
:1030200061742076616C7565206E6F7420706C61C0
:10303000757369626C653B206D75737420626520E1
:103040006174206C6561737420312E0A003F285230
:10305000296570656174206D7573742062652073D5
:103060007065636966696564207768656E206E6F58
:1030700074207573696E6720616E204C43442E0A7C
:10308000003F537065636966696564206E6F7A7A84
:103090006C652074656D7065726174757265206E03
:1030A0006F7420706C61757369626C652E0A003FE5
:1030B0005370656369666965642066696C616D65F6
:1030C0006E742073697A65206E6F7420706C617500
:1030D0007369626C652E0A003F53706563696669A7
:1030E0006564207072696D65206C656E6774682018
:1030F0006E6F7420706C61757369626C652E0A0066
:103100003F5072696D65206C656E677468206D75DF
:1031100073742062652073706563696669656420F5
:103120007768656E206E6F74207573696E672061B5
:103130006E204C43442E0A003F53706563696669F4
:103140006564206E6F7A7A6C652073697A65206E8B
:103150006F7420706C61757369626C652E0A003F34
:1031600052657472616374696F6E204D756C746919
:10317000706C696572206D75737420626520737060
:10318000656369666965642E0A003F53706563690B
:10319000666965642052657472616374696F6E203C
:1031A0004D756C7469706C696572206E6F742070F7
:1031B0006C61757369626C652E0A003F53706563BC
:1031C0006966696564206C61796572206865696704
:1031D0006874206E6F7420706C61757369626C65C1
:1031E0002E0A0043292E0A003F5370656369666901
:1031F0006564206265642074656D706572617475C4
:103200007265206E6F7420706C61757369626C6595
:10321000202834302D00473236207374617274696F
:103220006E672E2E2E0A004F46460A0046616465E0
:10323000204865696768742000426564204C6576A3
:10324000656C696E6720004661696C656420746F07
:1032500020656E61626C6520426564204C65766510
:103260006C696E670A00496E76616C6964206D65F1
:1032700073682E0A0050726F62696E6720506F6922
:103280006E740025532025692F2569002E0A002F12
:103290000050726F62696E67206D65736820706F91
:1032A000696E742000202844525952554E29004717
:1032B0003239204175746F20426564204C65766513
:1032C0006C696E67003F20284C2C522C462C4229FA
:1032D000206F7574206F6620626F756E64732E0A9E
:1032E000003F2856296572626F7365206C657665AC
:1032F0006C20696D706C61757369626C6520283033
:103300002D34292E0A00426164205A2076616C75A2
:10331000650A004E6F2062696C696E656172206794
:103320007269640A00416363757261637920446560
:103330006372656173696E672100446563726561DC
:1033400073696E67204163637572616379204465B8
:103350007465637465642E0A00473238004732385A
:103360005A0041636375726163793A2000206F6689
:10337000200044696420004733342061626F727416
:1033800065642E0A0041636375726163792041634D
:10339000686965766564005461726765742061636D
:1033A0006375726163792061636869657665642E0F
:1033B0000A004469666673205A312D5A323D2573DE
:1033C000000A444946464552454E4345205A312D50
:1033D0005A323D0050726F62696E67204661696CB7
:1033E00065640050726F62696E67206661696C6522
:1033F000640A0047333420497465726174696F6EE2
:103400003A202569000A4733342049746572617493
:10341000696F6E3A20003F2841296D706C696669BA
:10342000636174696F6E206F7574206F6620626FC0
:10343000756E64732028302E352D322E30292E0AD9
:10344000003F285429617267657420616363757257
:10345000616379206F7574206F6620626F756E648A
:10346000732028302E30312D312E30292E0A003F86
:103470002849297465726174696F6E206F757420B4
:103480006F6620626F756E64732028312D3330298A
:103490002E0A003F285929206F7574206F6620621C
:1034A0006F756E64732E0A003F285829206F75745B
:1034B000206F6620626F756E64732E0A003F28537A
:1034C000292050726F62652D706F736974696F6E19
:1034D00020696E64657820696E76616C69642E0A75
:1034E000003F2853292069732072657175697265E0
:1034F000642E0A004D3432322053004465766961EF
:1035000074696F6E0025533A2025730046696E6911
:1035100073686564210A003A207A3A2000206F66B9
:103520002000476F696E6720746F3A205800435738
:103530000A00206469723A0020616E676C653A0087
:103540005374617274207261646975733A004D340A
:103550003820506F696E740025533A2025642F255A
:103560006400506F736974696F6E696E6720746868
:10357000652070726F62652E2E2E0A003F4C6567C3
:1035800073206F66206D6F76656D656E7420696D52
:10359000706C61757369626C652028302D31352936
:1035A0002E0A003F2028582C5929206F7574206F4F
:1035B0006620626F756E64732E0A0050726F6265CA
:1035C000206F7574206F6620626F756E6473003FA4
:1035D00053616D706C652073697A65206E6F74201D
:1035E000706C61757369626C652028342D353029E3
:1035F0002E0A004D3438205A2D50726F62652052C9
:1036000065706561746162696C6974792054657371
:10361000740A003F2856296572626F7365206C65D5
:1036200076656C20696D706C61757369626C65207C
:1036300028302D34292E0A005374616E646172643F
:1036400020446576696174696F6E3A20002052618A
:103650006E67653A2000204D61783A2000204D6960
:103660006E3A2000205369676D613A20004D656114
:103670006E3A20005741524E494E4721204C6F77F9
:10368000205A204A65726B206D6179206C656164F7
:1036900020746F20756E77616E746564207061753B
:1036A0007365732E0A000201700111241FBECFEF53
:1036B000D1E2DEBFCDBF00E00CBF14E0A0E0B2E07D
:1036C000EEE3FFE602E00BBF02C007900D92A032CE
:1036D000B107D9F726E1A0E2B4E001C01D92A335FD
:1036E000B207E1F71BE1C4E5DBE100E006C021978A
:1036F0000109802FFE010F94CC33C335D10780E040
:103700000807A9F70F943E210D948D370C94000003
:103710009F92AF92BF92CF92DF92EF92FF920F9360
:103720001F93CF93DF9300D01F921F92CDB7DEB7C8
:10373000E2E0F1E10027BB27462F572FA82FAA234D
:1037400041F4A52F542FB85FAA2319F4A52F5527AC
:10375000B85FA03138F45295A295452F4F70507F35
:10376000A42BBC5FA03428F4550FAA1F550FAA1F25
:10377000BE5FA03818F4550FAA1FB395550FAA1FA6
:10378000EA0FF01F449151E0AA27B85081F1C8F028
:10379000B0FF02C0440F551FB1FF04C0440F551FB6
:1037A000440F551FB2FF06C052954295142F1F704B
:1037B000407F512BB3FF1BC0A52F542F44270C94DF
:1037C000F71BB195B0FF02C055954795B1FF04C0F6
:1037D0005595479555954795B2FF05C05295407F41
:1037E0004295452B5F70B3FF02C0452F5527DD245E
:1037F000CC24BB24B2E0649FD018C108B00AB00B3F
:10380000749FC018B108B00B849FB018B109659FB0
:10381000C018B108B00B759FB018B109859FB019D9
:103820006A9FB018B1097A9FB0194D9DA12C9924B7
:103830003327992722275D9DA00C911C301F901FD4
:10384000201FAD9D900C311D901F201F4C9DA00C82
:10385000911C301F901F201F5C9D900C311D901FEC
:10386000201FAC9D300D911D201F4B9D900C311DD4
:10387000901F201F5B9D300D911D201FAB9D900D53
:10388000211D4B9F300D911D201F5B9F900D211D11
:10389000AB9F200DB1E0BB24CC24DD24639FD01866
:1038A000C108B00AB00B739FC018B108B00B839F5A
:1038B000B018B109699FC018B108B00B799FB01852
:1038C000B109899FB019629FB018B109729FB019F0
:1038D000D61AC70AB80A20F0B1E03B0F901F201F8C
:1038E0001124792F632F90E0822F0F900F900F906B
:1038F0000F900F90DF91CF911F910F91FF90EF905C
:10390000DF90CF90BF90AF909F900895AF92BF92FD
:10391000CF92DF92EF92FF920F931F93CF93DF939B
:10392000CCE5DBE00BE118E08CE6A82E8BE0B82EAE
:10393000C12CD12C7601C394699179918991999187
:103940000F940A2D288939894A895B890F946B2D38
:103950000F944835F80161937193819391938F018E
:10396000C616D706E806F90610F46B017C01AC1602
:10397000BD0611F76FEF7FEFCB01A70196010F9402
:10398000493320932B0830932C0840932D085093F3
:103990002E08DF91CF911F910F91FF90EF90DF9054
:1039A000CF90BF90AF900895CF93DF9324E0829F94
:1039B000C0011124EC01C250D84FFC01EC5CF84F5F
:1039C000885D984FDC012D913D914D915C91608116
:1039D0007181828193810F94D533688379838A833F
:1039E0009B83DF91CF9108958091A7119091A811A9
:1039F000891B877089F48091AF0C81110DC0809173
:103A0000A40B9091A50B892B39F481E09091D605F8
:103A1000911103C080E0089581E0089590E080E076
:103A20000895282F90912207833021F495FD0FC02F
:103A300094FD0FC0892F90E0B0E0A0E004C0B695DF
:103A4000A795979587952A95D2F78170089581E07B
:103A5000089580E00895CF93C82FCB010E94B1F75D
:103A600086E79EE00E94B1F787E69EE0CC2311F046
:103A70008CE69EE00E94B1F78AE0CF910C9489F722
:103A80000F931F93CF938C01C62F89EC99E00E946E
:103A9000B1F7C8010E94B1F78AE30E9489F780E379
:103AA0008C0F0E9489F78AE0CF911F910F910C949F
:103AB00089F78CE49BE00E94B1F760E08CE39BE027
:103AC0000E94401D60E087E29BE00E94401D61E093
:103AD00080E29BE00E94401D61E085E19BE00E9446
:103AE000401D61E085E09BE00E94401D60E08CEF9E
:103AF0009AE00E94401D61E082EF9AE00E94401D22
:103B000061E088EE9AE00E94401D61E081EE9AE05B
:103B10000E94401D61E089ED9AE00E94401D61E035
:103B20008BEC9AE00E94401D61E08DEB9AE00E94D0
:103B3000401D60E08EEA9AE00E94401D60E080EA4D
:103B40009AE00E94401D60E08AE89AE00E94401DD1
:103B500061E089E79AE00E94401D61E08AE69AE010
:103B60000E94401D61E083E69AE00E94401D60E0F3
:103B70008CE59AE00E94401D61E083E59AE00E9496
:103B8000401D61E08EE39AE00E94401D61E080E309
:103B90009AE00E94401D61E08DE19AE00E94401D84
:103BA00060E080E19AE00E94401D61E08BE09AE0D5
:103BB0000E94401D61E08EEF99E00E94401D60E090
:103BC0008AEE99E00E94401D60E087ED99E00E9436
:103BD000401D60E082E593E10E940E1D682F617038
:103BE0008EEC99E00C94401DCF93DF938091A71148
:103BF0009091A811891B8095877019F40F944C0F30
:103C0000F5CF8091A7118F5F8770A091A7119CE5D8
:103C1000A99FD0011124FD01EC5CF74FEF0119922F
:103C20009A95E9F798E09083A75BB74F90E1E9EAAE
:103C3000F1E101900D929A95E1F72091A7119091F1
:103C4000A811291303C094E69093A4118093A7119F
:103C5000DF91CF910C94C4F22F923F924F925F92DA
:103C60006F927F928F929F92AF92BF92CF92DF928C
:103C7000EF92FF920F931F93CF93DF93D62FC72F0F
:103C8000FC0180809180A280B380C501B40120E84E
:103C900031E541E050E00F944933C9016DE671E030
:103CA0000F94B8336B017C01C501B40120E13EE003
:103CB00040E050E00F944933CA01B90128E130E0F7
:103CC00040E050E00F944933362E272E062F172F51
:103CD0008CE3482E512C612C712CC501B401A30139
:103CE00092010F944933B62EA72ECA01B901A30140
:103CF00092010F944933CB01C114D10479F1AF92F1
:103D0000BF927F936F932F923F92FF92EF92DF9239
:103D1000CF9289E09DE09F938F93CF93DF930F9491
:103D20009C2C8DB79EB70E960FB6F8949EBF0FBE13
:103D30008DBF8D2F9C2FDF91CF911F910F91FF9001
:103D4000EF90DF90CF90BF90AF909F908F907F903B
:103D50006F905F904F903F902F900895E114F10481
:103D6000C9F0AF92BF927F936F932F923F92FF92D1
:103D7000EF9289EF9CE09F938F93CF93DF930F9403
:103D80009C2CEDB7FEB73C960FB6F894FEBF0FBE65
:103D9000EDBFCFCF012BB9F0AF92BF927F936F935E
:103DA0002F923F928DEE9CE09F938F93CF93DF9362
:103DB0000F949C2C8DB79EB70A960FB6F8949EBFB1
:103DC0000FBE8DBFB6CF892BA9F0AF92BF927F9364
:103DD0006F9385EE9CE09F938F93CF93DF930F9427
:103DE0009C2CEDB7FEB738960FB6F894FEBF0FBE09
:103DF000EDBF9FCFAF92BF9281EE9CE09F938F93D8
:103E0000CF93DF930F949C2C0F900F900F900F90F7
:103E10000F900F908ECFCF93DF9300D01F92CDB72E
:103E2000DEB784EF91E0A0E0B0E089839A83AB83B2
:103E3000BC83BE016F5F7F4F8CE30E944DF584E928
:103E40009EE00E94B1F78CB16EE87EE085FB88278A
:103E500080F90E942B1D8091030168E87EE0869521
:103E600081700E942B1D89B162E87EE083FB882768
:103E700080F90E942B1D8CB169E77EE082958170EC
:103E80000E942B1D4B9909C00E9488F50F900F903E
:103E90000F900F90DF91CF9108950E946DF50F90D4
:103EA0000F900F900F90DF91CF910895809116069B
:103EB000882319F010921606089540E070E060E043
:103EC00089E59EE00F947B0ECF93C091A704CF7736
:103ED00039F50E94E0F3882319F1809147139091FE
:103EE0004813A0914913B0914A130097A105B10559
:103EF000B9F0BC01CD016D597F4F8F4F9F4F24E624
:103F000030E040E050E00F94493360914B137091E2
:103F10004C1380914D1390914E130F944933C22F3F
:103F20008C2FCF910895CF93DF93EB010E947EEE0B
:103F3000882319F00E94CEEDEB01CE01DF91CF91E5
:103F400008954F925F926F927F928F929F92AF925D
:103F5000BF92CF92DF92EF92FF921F93CF93DF93A6
:103F600000D01F92CDB7DEB719821A821B821C8245
:103F7000CE0101964C0182EAC82E86E0D82E9AE442
:103F8000E92E92E0F92E2EEFA22E27E0B22E10E0BD
:103F900088E5810F0E947EEEF40181934F01882312
:103FA00009F4E0C00E9406EE2B013C01812F0E9423
:103FB000111D882309F4CCC0F70120813181428191
:103FC0005381C301B2010F94D533F601608371832D
:103FD000828393831F5FF4E0CF0ED11C84E0E80E50
:103FE000F11C94E0A90EB11C133091F685E40E94F7
:103FF0007EEE8C83882309F4C0C00E9406EE6B011C
:104000007C0183E00E94111D882371F020915602EB
:10401000309157024091580250915902C701B601A0
:104020000F94D5336B017C01C092AE06D092AF06DF
:10403000E092B006F092B1068091E804882359F12D
:1040400080914F1382FF27C08C81882321F18981C1
:10405000811103C08A818823F1F02DEC3CEC4CE403
:104060005DE36091490770914A0780914B079091F9
:104070004C070F94D5339B01AC01609152027091B3
:10408000530280915402909155020F9435361816C0
:1040900014F40E945DC240E050E0BA0186E40E9440
:1040A000EBEE20E030E0A9010F943536181684F4C9
:1040B0000E9406EE20E030E040E752E40F94CF3457
:1040C00060932A0270932B0280932C0290932D020E
:1040D0008091140B83FD28C08091C105882321F1B4
:1040E0002091560230915702409158025091590246
:1040F0006091AE067091AF068091B0069091B106C6
:104100000F94D4332091CE053091CF054091D00546
:104110005091D1050F94D5336093CE057093CF05A0
:104120008093D0059093D1050F900F900F900F9032
:10413000DF91CF911F91FF90EF90DF90CF90BF90D4
:10414000AF909F908F907F906F905F904F90089569
:10415000F5012081318142815381C301B2010F9465
:10416000D43333CFF70180819181A281B381F601ED
:1041700080839183A283B3832DCF80915602909147
:104180005702A0915802B09159028093AE069093C5
:10419000AF06A093B006B093B1064ECFCF9384E59F
:1041A0000E947EEEC0E08823D9F00E94DEEDC82F89
:1041B0001816B4F40F94A10B8DE40E9489F7809136
:1041C0009804909199040E9429AD6C2FCC0F770B25
:1041D0008DE495E00E9404FA8AE00E9489F7CFEF0F
:1041E0008C2FCF910895CF92DF92EF92FF920F9391
:1041F0001F93CF93DF93CDB7DEB7A0970FB6F89498
:10420000DEBF0FBECDBF0E94CE2087FDCCC085E4AF
:104210000E9430EE882309F4D5C00E9406EE6B019F
:104220007C0120E030E0A9010F94353687FF04C0FF
:10423000F7FAF094F7F8F094F7FAF094F7F8F094AE
:10424000CD8EDE8EEF8EF8A28CE0EBE8F2E0DE01A0
:10425000119601900D928A95E1F78AE50E947EEE13
:10426000882351F040E050E0BA018AE50E94EBEE6D
:1042700069877A878B879C8788E50E947EEE8823F2
:1042800051F040E050E0BA0188E50E94EBEE69830E
:104290007A838B839C8389E50E947EEE882351F08C
:1042A00040E050E0BA0189E50E94EBEE6D837E8329
:1042B0008F83988785E50E9430EE882309F489C0B2
:1042C0000E9406EE6B017C0120E030E0A901C701ED
:1042D000B6010F94353687FF04C0F7FAF094F7F86B
:1042E000F094F7FAF094F7F8F094C98EDA8EEB8E2A
:1042F000FC8E1D8A1E8A1F8A188E8CE40E9430EE66
:10430000882309F46FC00E9406EE6B017C0120E057
:1043100030E0A901C701B6010F94353687FF04C00C
:10432000F7FAF094F7F8F094C98ADA8AEB8AFC8AF3
:1043300062E070E082E40E9402EFF82E809141106A
:10434000811131C021E0AE01475E5F4FBE016F5F5A
:104350007F4FCE014D960F94FB1D882321F16F2DC9
:1043600081E00F94CD1E82E50E947EEE882309F441
:1043700042C00E9402EE40E050E060EA71E44D87E6
:104380005E876F87788B20914110222361F08C012A
:104390002F2DAE01435F5F4FBE016F5E7F4FCE0199
:1043A00045960F94B81CA0960FB6F894DEBF0FBECA
:1043B000CDBFDF91CF911F910F91FF90EF90DF90D4
:1043C000CF900895C12CD12C80E8E82E80E4F82EFF
:1043D00033CFC090E004D090E104E090E204F0908C
:1043E000E30472CFC090E404D090E504E090E604CA
:1043F000F090E7048CCF90E080E0BDCFCF92DF92C9
:10440000EF92FF920F931F93CF93DF93CDB7DEB759
:104410006C970FB6F894DEBF0FBECDBF8CE40E9440
:1044200030EE882309F4B0C00E9406EE6B017C01D7
:1044300020E030E0A9010F94353687FF04C0F7FA79
:10444000F094F7F8F094F7FAF094F7F8F094C98E36
:10445000DA8EEB8EFC8E8CE0EBE8F2E0DE0111965A
:1044600001900D928A95E1F788E50E947EEE8823FF
:10447000A1F040E050E0BA0188E50E94EBEE209107
:10448000FE073091FF0740910008509101080F94FA
:10449000D43369837A838B839C8389E50E947EEE83
:1044A0008823A1F040E050E0BA0189E50E94EBEEDC
:1044B0002091FE073091FF074091000850910108BC
:1044C0000F94D4336D837E838F8398878AE50E940F
:1044D0007EEE882351F040E050E0BA018AE50E9468
:1044E000EBEE69877A878B879C871D861E861F86E1
:1044F000188A80914110811138C020E0AE01435FDD
:104500005F4FBE016F5F7F4FCE0149960F94FB1D39
:10451000882359F18091E80481110E945DC260E016
:1045200080E00F94CD1E898D9A8DAB8DBC8DB058D7
:104530008D8B9E8BAF8BB88F198A1A8A1B8A1C8A27
:104540001D861E861F86188A80914110882369F077
:1045500010E000E020E0AE014B5E5F4FBE016F5EF9
:104560007F4FCE010D960F94B81C6C960FB6F89441
:10457000DEBF0FBECDBFDF91CF911F910F91FF9096
:10458000EF90DF90CF900895C12CD12C80E8E82ED9
:1045900080E4F82E58CF84E690E09093DF04809377
:1045A000DE0410920F0510920E050C94CFA60F9307
:1045B000AB0100910D0521E002272EE035E0BC01A2
:1045C0008EED94E00E940AF40F910895CF93DF934B
:1045D00000D01F92CDB7DEB78091C1058823C1F00E
:1045E00083E390E09C838B831A8219829E012F5F64
:1045F0003F4F40E150E062EC75E0CE0103960F942E
:104600000B0E86E492E10E94B1F78AE00E9489F7DE
:104610000F900F900F900F90DF91CF910895CF934F
:10462000DF9300D01F921F92CDB7DEB781E0809359
:10463000C10580E1E2ECF5E0DF011D928A95E9F722
:104640000E94E62286E18D8382E390E09C838B8347
:104650001A8219829E012F5F3F4F41E050E0BE0158
:104660006B5F7F4FCE0103960F940B0E0F900F9050
:104670000F900F900F90DF91CF910895CF92DF921E
:10468000EF92FF92CF93DF93EC0108960E94EEE940
:104690006B017C0120E030E0A9010F94052D20E0A2
:1046A00030E0A901882359F0CE010E94D7EF9B0189
:1046B000AC01C701B6010F946B2D9B01AC0168855D
:1046C00079858A859B850F94D433688779878A8713
:1046D0009B87DF91CF91FF90EF90DF90CF9008956F
:1046E000833B21E0920714F083EB91E090930C114F
:1046F00080930B110C9497C80F931F93CF93DF9364
:1047000000E71BE0C4E8D0E1F8012191319141912B
:1047100051918F0160E070E080E89FE30F94CF3407
:104720006993799389939993F0E1C439DF0761F72D
:104730000E949CC0DF91CF911F910F910C94861C19
:104740009091A7118091A811981306C0809132080A
:1047500090913308892B21F080E00F944C0FF0CF1B
:1047600008959091A7118091A811981308C0809185
:10477000320890913308892B11F40C94C6F380E031
:104780000F944C0FEECFCF92DF92EF92FF92CF9328
:10479000DF932091570B222329F1EC0108960E9408
:1047A000EEE96B017C0120E030E0A9010F94052DBA
:1047B00020E030E0A901882359F0CE010E94D7EF14
:1047C0009B01AC01C701B6010F946B2D9B01AC019D
:1047D000688579858A859B850F94D5336887798725
:1047E0008A879B87DF91CF91FF90EF90DF90CF90EA
:1047F0000895CF92DF92EF92FF928091270788234E
:1048000009F457C0C0902307D0902407E0902507F3
:10481000F090260720E030E0A901C701B6010F940F
:10482000052D882309F445C020E030E040E05FE337
:10483000C701B6010F946B2D9B01AC010F946B2D3A
:104840002BED3FE049E450E40F946B2D9B01AC014C
:1048500060E070E080E89FE30F94CF346B017C014F
:10486000C092580BD092590BE0925A0BF0925B0B0E
:1048700060915E0270915F02072E000C880B990B0D
:104880000F940C2D2AE037ED43E25CE30F946B2D7F
:10489000A70196010F946B2D60935A0270935B02EF
:1048A00080935C0290935D02FF90EF90DF90CF9039
:1048B0000895C12CD12C80E8E82E8FE3F82ED0CFBC
:1048C0000F931F93CF93DF9350E0FC01E40FF51F8C
:1048D0008081440F551F440F551F42545B4FEA011E
:1048E000882329F188819981AA81BB81EB01088104
:1048F00019812A813B810097A105B10569F40C5902
:104900001F4F2F4F3F4FDA010D931D932D933C9373
:1049100013978FEF808306C0081B190B2A0B3B0BE4
:1049200037FDF7CFDF91CF911F910F910895188236
:1049300019821A821B82F6CF2F923F924F925F927A
:104940006F927F928F929F92AF92BF92CF92DF929F
:10495000EF92FF920F931F93CF93DF93CDB7DEB704
:104960006C970FB6F894DEBF0FBECDBF8C015B0114
:104970005A834983FC01EA5BFF4F208131814281E8
:10498000538129873A874B875C87CA01B9010F9405
:104990000A2D6B017C01D5012D913D914D915C91CA
:1049A0000F946B2D0F94B3342B013C01E981FA81F4
:1049B0002081318142815381C701B6010F946B2D53
:1049C0000F94B3344B015C01C301B2010F9448351D
:1049D000698B7A8B8B8B9C8B683771058105910570
:1049E00040F428E730E040E050E0298B3A8B4B8BD5
:1049F0005C8BC501B4010F9448356D877E878F8726
:104A0000988B683771058105910540F448E750E0BF
:104A100060E070E04D875E876F87788BF801EE5A13
:104A2000FF4F4080518062807380C301B2010F94B8
:104A30000C2D69837A838B839C8369897A898B891E
:104A40009C890F940A2D6D8B7E8B8F8B988F20E025
:104A500030E0A90169817A818B819C810F94052DB9
:104A6000882309F4E1C1A7019601C701B6010F949B
:104A70006B2D4B015C012D893E894F89588DCA01F0
:104A8000B9010F946B2D9B01AC01C501B4010F94CA
:104A9000D4334B015C0129813A814B815C81CA018D
:104AA000B9010F94D5339B01AC01C501B4010F943A
:104AB000CF340F94B3340F9448356D837E838F8346
:104AC000988766277727CB016419750986099709A6
:104AD0000F940C2D4B015C016D857E858F85988927
:104AE0000F940A2D2B013C0120E030E0A901C50103
:104AF000B4010F94052D882309F49AC1A3019201F2
:104B0000C301B2010F946B2D698F7A8F8B8F9C8FAD
:104B1000A7019601C701B6010F946B2D9B01AC0153
:104B2000698D7A8D8B8D9C8D0F94D4336B017C01B4
:104B3000A5019401C501B4010F94D5339B01AC01CB
:104B4000C701B6010F94CF340F947735D8019596ED
:104B50008D909D90AD90BC909897750164012D81CA
:104B60003E814F815885C21AD30AE40AF50A0F9490
:104B70004835C61AD70AE80AF90AF7FE8EC02D8909
:104B80003E894F89588DCA01B9010F946B2D6B0175
:104B90007C0129813A814B815C81CA01B9010F9462
:104BA000D53369877A878B879C8720E030E0A9011D
:104BB00069817A818B819C810F94052D882309F46A
:104BC0003BC1C501B4010F940A2D29853A854B8557
:104BD0005C850F946B2DA70196010F94D4336D83E0
:104BE0007E838F839887A3019201C301B2010F9442
:104BF0006B2D9B01AC016D817E818F8198850F9417
:104C0000D5332B013C0120E030E040E850E46981DD
:104C10007A818B819C810F946B2D9B01AC01C30128
:104C2000B2010F94CF340F94B3342B013C0120E038
:104C300030E0A9010F94353618161CF0412C512C88
:104C40003201C301B2010F9448356D837E838F8397
:104C5000988786169706A806B90620F48D829E824C
:104C6000AF82B8866D817E818F8198850F940A2DE1
:104C700029853A854B855C850F946B2DA70196019C
:104C80000F94D5330F9483360F94483569877A870C
:104C90008B879C87C12CD12C760169857A858B8581
:104CA0009C8529893A894B895C89621B730B840B2B
:104CB000950B0F940A2D29813A814B815C810F94C9
:104CC000CF3420E034E244EF59E40F946B2D0F947D
:104CD00048354B015C0169857A858B859C852D85DE
:104CE0003E854F855889621B730B840B950B0F947F
:104CF0000A2D29813A814B815C810F94CF3420E0C9
:104D000034E244EF59E40F946B2D0F9448352B0196
:104D10003C013FE683169104A104B10408F090C061
:104D2000F401EE0FFF1FEE0FFF1FEA5BF04F8591BE
:104D30009591A591B4918983292E3A2EBD8B4FE68A
:104D4000441651046104710408F083C0F201EE0FAF
:104D5000FF1FEE0FFF1FEA5BF04F459155916591E4
:104D600074919A01CB014D815E816F817885D80164
:104D700099964D935D936D937C939C974C0D5D1D1F
:104D80006E1D7F1DF80145A756A767A770ABE65BB0
:104D9000FF4F49895A896B897C894083518362839B
:104DA0007383D5968D929D92AD92BC92D897F8015F
:104DB00041AE52AE63AE74AEFD964981408321820E
:104DC00032825D8953833496208331838283938337
:104DD00069857A858B859C85D1966D937D938D931E
:104DE0009C93D4973D962D853E854F855889208389
:104DF0003183428353836C960FB6F894DEBF0FBEA7
:104E0000CDBFDF91CF911F910F91FF90EF90DF9079
:104E1000CF90BF90AF909F908F907F906F905F905A
:104E20004F903F902F90089560E070E0CB0141CE0D
:104E300060E070E0CB0188CE60E070E0CB01F3CEA3
:104E4000C501B4010E94881B6983272E382E9D8BD3
:104E500076CFC301B2010E94881B9B0184CF809151
:104E6000A7119091A811891B877019F490E080E038
:104E700008959091A411992351F0833030F48FEF6D
:104E8000890F19F08093A411F1CF1092A411809191
:104E9000A8112CE5829FC00111248C5C974FFC0166
:104EA000208120FDE3CF2091A8112F5F2770209350
:104EB000A5113091A8112091A611321304C02091A0
:104EC000A5112093A611089590916F0081E091FDA6
:104ED00002C080E0089590916F009D7F90936F00D5
:104EE0000895FC01208131814281538160917C0BC6
:104EF00070917D0B80917E0B90917F0B0F946B2DA9
:104F00000F9442366093B5117093B6118093B71128
:104F10009093B8119091A7118091A81198130C94B7
:104F2000F41D0E94A0230E9464274091B511509166
:104F3000B6116091B7117091B81140933A05509332
:104F40003B0560933C0570933D0581110C94C4F2C0
:104F500008954F925F926F927F928F929F92AF923D
:104F6000BF92CF92DF92EF92FF920F931F93CF9356
:104F7000DF93EC018B015A01F90120917C0B3091F8
:104F80007D0B40917E0B50917F0B608171818281FE
:104F900093810F946B2D0F9442366B017C0120910D
:104FA000780B3091790B40917A0B50917B0BF50186
:104FB00060817181828193810F946B2D0F944236B1
:104FC0004B015C012091740B3091750B4091760B75
:104FD0005091770BF80160817181828193810F94E8
:104FE0006B2D0F9442362B013C012091700B3091B8
:104FF000710B4091720B5091730B688179818A819A
:105000009B810F946B2D0F9442366093A91170937E
:10501000AA118093AB119093AC114092AD115092B4
:10502000AE116092AF117092B0118092B111909256
:10503000B211A092B311B092B411C092B511D09236
:10504000B611E092B711F092B8119091A71180912A
:10505000A811981791F0DF91CF911F910F91FF90B8
:10506000EF90DF90CF90BF90AF909F908F907F9008
:105070006F905F904F900C94F41D0E94A0230E94AB
:1050800064274091B1115091B2116091B3117091A8
:10509000B4110091AD111091AE112091AF1130916A
:1050A000B011C090A911D090AA11E090AB11F0906E
:1050B000AC11C0922E05D0922F05E0923005F092EF
:1050C0003105009332051093330520933405309356
:1050D0003505409336055093370560933805709336
:1050E00039054091B5115091B6116091B711709189
:1050F000B81140933A0550933B0560933C0570937B
:105100003D05882391F0DF91CF911F910F91FF9082
:10511000EF90DF90CF90BF90AF909F908F907F9057
:105120006F905F904F900C94C4F2DF91CF911F91DC
:105130000F91FF90EF90DF90CF90BF90AF909F9036
:105140008F907F906F905F904F900895CF92DF92F5
:10515000EF92FF92CF93DF93C82F0E94642794E0D1
:10516000C99FE0011124FE01E25DFA4FC080D180A9
:10517000E280F38081110E94C4F2CC57DF4EC70158
:10518000B6010F940C2D288139814A815B810F94DF
:105190006B2DDF91CF91FF90EF90DF90CF9008952E
:1051A0003F924F925F926F927F928F929F92AF92B7
:1051B000BF92CF92DF92EF92FF920F931F93CF9304
:1051C000DF93CDB7DEB768970FB6F894DEBF0FBE9A
:1051D000CDBFD82E2A013B01480159013E2C20E0C9
:1051E00030E0A901C501B8010F94052D811110C04F
:1051F00081E08D1508F0B6C060E070E080E793E4D0
:1052000020E030E040E752E40F94CF344B015C01E2
:105210008D8A9E8AAF8AB88E0D2D10E0F801ED5B65
:10522000F04FE491BB24B3941E160CF4B12CCC24A3
:10523000C39420E030E0A901C301B2010F943536D8
:1052400018160CF0C12CBC1471F092E0D9120BC0EE
:10525000332049F081E00E9424C469E170E080E0DD
:1052600090E00E94E1F280E00E94A62869837A83A0
:105270008B839C8381E00E94A6286D837E838F832D
:10528000988782E00E94A62869877A878B879C8707
:1052900083E00E94A6286D877E878F87988B000FFA
:1052A000111F000F111FE1E0F0E0EC0FFD1F0E0FCA
:1052B0001F1FF80110821182128213829E01235F48
:1052C0003F4FAE01475F5F4FBE016B5F7F4FCE0127
:1052D00001960E94A927F80140825182628273825E
:1052E000198A1A8A1B8A1C8A809132089091330885
:1052F000892B91F4CE0141967C018E010B5E1F4FEC
:105300009E01235F3F4FAE01475F5F4FBE016B5F62
:105310007F4F40970E94CEB20E94A023BC1451F050
:1053200092E0D91205C0332019F080E00E9424C415
:105330000E94561F68960FB6F894DEBF0FBECDBF11
:10534000DF91CF911F910F91FF90EF90DF90CF9061
:10535000BF90AF909F908F907F906F905F904F9095
:105360003F90089560E070E88BE395E449CFCF92D9
:10537000DF92EF92FF92CF93DF93C82F0E946427B2
:1053800094E0C99FE0011124FE01EE5DFA4FC08058
:10539000D180E280F38081110E94C4F2CC57DF4EAD
:1053A000C701B6010F940C2D288139814A815B8198
:1053B0000F946B2DDF91CF91FF90EF90DF90CF9006
:1053C00008950E9464279091A8119093A71190933B
:1053D000A6119093A51194E69093A41120ED33E0CB
:1053E000309333082093320881110E94C4F281E087
:1053F00080932105089580FF04C09091560B90FD85
:105400008E7F81FF05C09091560B969590FD8D7F04
:1054100082FF06C09091560B9695969590FD8B7FD6
:1054200008958F929F92AF92BF92CF92DF92EF92A8
:10543000FF92CF93DF9320912E02222309F49EC086
:10544000EC0180919204C82ED12CF12CE12C80FF2C
:105450002CC08090300290903102A0903202B09027
:105460003302288139814A815B81C501B4010F94DF
:105470003536181624F488829982AA82BB828090DD
:105480003C0290903D02A0903E02B0903F022881E5
:1054900039814A815B81C501B4010F94052D87FFD5
:1054A00004C088829982AA82BB82D701C601B695C0
:1054B000A7959795879580FF2CC080903402909097
:1054C0003502A0903602B09037022C813D814E818A
:1054D0005F81C501B4010F943536181624F48C820F
:1054E0009D82AE82BF828090400290904102A09047
:1054F0004202B09043022C813D814E815F81C50103
:10550000B4010F94052D87FF04C08C829D82AE826A
:10551000BF8282E0F694E794D794C7948A95D1F736
:10552000C0FE2CC0C0903802D0903902E0903A0200
:10553000F0903B02288539854A855B85C701B60115
:105540000F943536181624F4C886D986EA86FB8669
:10555000C0904402D0904502E0904602F09047028D
:10556000288539854A855B85C701B6010F94052DCD
:1055700087FF04C0C886D986EA86FB86DF91CF9173
:10558000FF90EF90DF90CF90BF90AF909F908F9063
:1055900008952F923F924F925F926F927F928F92D7
:1055A0009F92AF92BF92CF92DF92EF92FF920F93B2
:1055B0001F93CF93DF93CDB7DEB7A6970FB6F894BE
:1055C000DEBF0FBECDBF82EA96E00E94112A809115
:1055D000140B83FD7EC020915602309157024091FA
:1055E0005802509159026091AE067091AF068091B9
:1055F000B0069091B1060F94052D882309F469C077
:1056000010913108111161C08091480290914902B6
:1056100001972091091130910A11281739073CF49C
:105620000F94A10B8DEC9EE00E94B1F711E0209148
:1056300056023091570240915802509159026091A0
:10564000AE067091AF068091B0069091B1060F94AE
:10565000D4336B017C0120E030E0A9010F94353692
:1056600087FF04C0F7FAF094F7F8F09420915A02FB
:1056700030915B0240915C0250915D02C701B6011E
:105680000F946B2D20E030E84BE354E40F94353653
:105690001816ECF40F94A10B8EEA9EE00E94B1F76D
:1056A0008091AE069091AF06A091B006B091B10680
:1056B0008093560290935702A0935802B0935902D8
:1056C0008EEA96E00E94712704C010E0B0CF11115D
:1056D000E7CF2AE037ED43E25CE360912A02709164
:1056E0002B0280912C0290912D020F946B2D6B0157
:1056F0007C016091600270916102072E000C880BA2
:10570000990B0F940C2D9B01AC01C701B6010F94AE
:105710006B2D698B7A8B8B8B9C8B8091570B88239D
:1057200009F18090FA079090FB07A090FC07B090D9
:10573000FD07C090AA06D090AB06E090AC06F090B2
:10574000AD0620E030E0A901C501B4010F94052D9C
:105750008823D1F1A7019601C501B4010F94353614
:10576000181694F1C12CD12C76018E010F5E1F4FBB
:105770002EEA36E04AEA56E066EA76E082EA96E009
:105780000E9498BF80E1E2EAF6E0AAE4B2E001906C
:105790000D928A95E1F7A6960FB6F894DEBF0FBE7C
:1057A000CDBFDF91CF911F910F91FF90EF90DF90D0
:1057B000CF90BF90AF909F908F907F906F905F90B1
:1057C0004F903F902F90089520914A0230914B02C4
:1057D00040914C0250914D026091A2067091A30637
:1057E0008091A4069091A5060F94D4336D8B7E8B87
:1057F0008F8B988F20914E0230914F024091500232
:10580000509151026091A6067091A7068091A8065A
:105810009091A9060F94D433698F7A8F8B8F9C8FC8
:1058200020915202309153024091540250915502FE
:10583000C701B6010F94D4336D8F7E8F8F8F98A3DD
:1058400020915602309157024091580250915902CE
:105850006091AE067091AF068091B0069091B1064E
:105860000F94D4336B017C0120E030E0A9016D89F5
:105870007E898F89988D0F94052D81110CC020E0B1
:1058800030E0A901698D7A8D8B8D9C8D0F94052D4B
:10589000882309F467CF2D893E894F89588DCA0125
:1058A000B9010F946B2D4B015C01298D3A8D4B8D05
:1058B0005C8DCA01B9010F946B2D9B01AC01C50130
:1058C000B4010F94D5334B015C012D8D3E8D4F8D6E
:1058D00058A1CA01B9010F946B2D9B01AC01C50100
:1058E000B4010F94D5334B015C01A7019601C701A8
:1058F000B6010F946B2D9B01AC01C501B4010F944F
:10590000D5330F9483364B015C012DEB37E346E82A
:1059100055E30F94052D87FF0FC020E030E0A9016B
:10592000C701B6010F9435364601570187FF04C001
:10593000B7FAB094B7F8B0942DEB37E346E855E3E7
:10594000C501B4010F94052D87FD1CCF20E030E088
:1059500040EA51E4C501B4010F94CF340F944835A7
:105960001B01672B19F422242394312CB10190E000
:1059700080E00F940A2D9B01AC0160E070E080E8AC
:105980009FE30F94CF342B013C01AC019B01C50177
:10599000B4010F946B2D4B015C01A30192016D8941
:1059A0007E898F89988D0F946B2D6D8B7E8B8F8B5D
:1059B000988FA3019201698D7A8D8B8D9C8D0F94A8
:1059C0006B2D698F7A8F8B8F9C8FA30192016D8DC8
:1059D0007E8D8F8D98A10F946B2D6D8F7E8F8F8F05
:1059E00098A3A3019201C701B6010F946B2D69A37F
:1059F0007AA38BA39CA380E1EAE4F2E08E010F5F1F
:105A00001F4FD80101900D928A95E1F70E948BC833
:105A10002B013C0128EC420E511C611C711C0DA392
:105A20001EA381E0281A310809F460C00E948BC8C7
:105A30008B019C01041915092609370937FD59C046
:105A40002B013C0128EC420E511C611C711C80E0B2
:105A50000F944C0F2D893E894F89588D69817A8129
:105A60008B819C810F94D53369837A838B839C834C
:105A7000298D3A8D4B8D5C8D6D817E818F819885CE
:105A80000F94D5336D837E838F8398872D8D3E8DC4
:105A90004F8D58A169857A858B859C850F94D53368
:105AA00069877A878B879C8729A13AA14BA15CA142
:105AB0006D857E858F8598890F94D5336D877E8718
:105AC0008F87988B750164018E010F5E1F4F9E01B9
:105AD000235F3F4FAE01475F5F4FBE016B5F7F4F5C
:105AE0008DA19EA10E9498BF81119BCF7501640179
:105AF0003CCE0E94E78CAECF8091BA049091BB045B
:105B0000A091BC04B091BD0480932A0290932B0213
:105B1000A0932C02B0932D028091B8049091B90407
:105B20009093610280936002089580912A0290917F
:105B30002B02A0912C02B0912D028093BA04909375
:105B4000BB04A093BC04B093BD048091600290910B
:105B500061029093B9048093B80484E690E0909336
:105B600061028093600208958F929F92AF92BF92DC
:105B7000CF92DF92EF92FF92CF93DF9380902A0231
:105B800090902B02A0902C02B0902D02FC01C080BE
:105B9000D180E280F38020E030E0A901C701B601A6
:105BA0000F94052D882341F0C0922A02D0922B0237
:105BB000E0922C02F0922D02C0916002D09161021D
:105BC00084E690E09093610280936002C0905A0254
:105BD000D0905B02E0905C02F0905D0280E090E08B
:105BE000A0E8BFE380935A0290935B02A0935C020B
:105BF000B0935D020E94C92A80922A0290922B02E1
:105C0000A0922C02B0922D02D0936102C093600248
:105C1000C0925A02D0925B02E0925C02F0925D0266
:105C2000DF91CF91FF90EF90DF90CF90BF90AF903A
:105C30009F908F9008950F931F93CF93DF9300D081
:105C40001F92CDB7DEB79C0102EA16E090E1EAE4CC
:105C5000F2E0D80101900D929A95E1F7F9012081C7
:105C6000318142815381F8016085718582859385F8
:105C70000F94D533F801608771878287938780E01E
:105C800090E0A0EAB0E489839A83AB83BC83CE0121
:105C900001960E94B42D0F900F900F900F90DF91FE
:105CA000CF911F910F910895AF92BF92CF92DF9243
:105CB000EF92FF920F931F93CF93DF93CDB7DEB791
:105CC00064970FB6F894DEBF0FBECDBF0E94CE2002
:105CD00087FDAFC08AE50E947EEE882309F4BAC032
:105CE00040E050E0BA018AE50E94EBEE7B018C01B6
:105CF000209152023091530240915402509155022A
:105D000060E070E088EC93E40F94D4335B016C01A5
:105D10009701A8010F943536181614F07501860105
:105D200020E030E0A901B701C8010F9435361816FC
:105D300024F4E12CF12C00E010E0B701C8010F942D
:105D40004135072E000C880B990B0F940C2D698B95
:105D50007A8B8B8B9C8B20E030E0A9010F94052D72
:105D6000882321F0CE0141960E941B2E80E090E016
:105D7000A0EAB1E48D879E87AF87B88B19861A8613
:105D80001B861C868CE40E9430EE882309F467C0D1
:105D90000E9406EE6B017C0120E030E0A901C70102
:105DA000B6010F94353687FF04C0F7FAF094F7F880
:105DB000F094CD82DE82EF82F88620910B11309133
:105DC0000C112430310574F08091091190910A1161
:105DD000821B930B97FF03C091958195910901E078
:105DE00004970CF400E080E00F94571C882359F0CE
:105DF00022E0AE01435F5F4FBE016B5F7F4FCE017C
:105E000009960F94741B69897A898B899C898B0107
:105E10009C01305809831A832B833C8320E030E0B7
:105E2000A9010F94052D882321F0CE0101960E942F
:105E30001B2E64960FB6F894DEBF0FBECDBFDF9168
:105E4000CF911F910F91FF90EF90DF90CF90BF9077
:105E5000AF900895E12CF12C00E211E449CFC090FD
:105E6000E404D090E504E090E604F090E70494CFD9
:105E7000CF92DF92EF92FF920F931F93C12CD12C00
:105E800076018C0126E532E042E552E06EE472E0F4
:105E90008AE492E00E9498BF1F910F91FF90EF90CB
:105EA000DF90CF9008954F925F926F927F928F9282
:105EB0009F92AF92BF92CF92DF92EF92FF920F9399
:105EC0001F93CF93DF93CDB7DEB72C970FB6F8941F
:105ED000DEBF0FBECDBF2B013C0129873A874B8720
:105EE0005C8747015801F601E080F180028113814F
:105EF00020E030E0A901B701C8010F94052D8823E7
:105F000009F488C05E2D4F2D302F212F852F942F1F
:105F1000A32FB22F89839A83AB83BC8320E030E028
:105F2000A901B701C8010F94052D811108C0E090A7
:105F30002602F09027020091280210912902C70141
:105F4000D8018D839E83AF83B887A50194016091AA
:105F500052027091530280915402909155020F9415
:105F6000052D87FF0CC08092520290925302A0929E
:105F70005402B0925502CE0101960E94382F4092F1
:105F80004A0250924B0260924C0270924D028985F7
:105F90009A85AB85BC8580934E0290934F02A09367
:105FA0005002B0935102CE0105960E94382FA501F0
:105FB0009401609152027091530280915402909129
:105FC00055020F943536181664F48092520290925E
:105FD0005302A0925402B0925502CE0101960E9443
:105FE000382F0E94A0232C960FB6F894DEBF0FBE68
:105FF000CDBFDF91CF911F910F91FF90EF90DF9078
:10600000CF90BF90AF909F908F907F906F905F9058
:106010004F90089550E040E030E820E477CFCF92F1
:10602000DF92EF92FF920F931F936A01E09052026A
:10603000F09053020091540210915502FB0120810F
:10604000318142815381FC01608171818281938120
:106050000E94532F1F910F91FF90EF90DF90CF90F0
:106060000895CF92DF92EF92FF920F931F936B01EF
:10607000FC01E080F18002811381EAE4F2E02481F6
:1060800035814681578160817181828193810E942F
:10609000532F1F910F91FF90EF90DF90CF900895B5
:1060A000AF92BF92CF92DF92EF92FF920F931F9326
:1060B000CF93DF9300D01F92CDB7DEB7FC01E08015
:1060C000F18002811381611112C0A0905202B09040
:1060D0005302C0905402D09055029501A601B70119
:1060E000C8010F94052D87FF02C07501860120E0CD
:1060F00030E048EC53E4B701C8010F94052D87FD4B
:1061000004C0E12CF12C08EC13E4C701D801898309
:106110009A83AB83BC8366EE72E0CE0101960E9447
:1061200031300F900F900F900F90DF91CF911F9112
:106130000F91FF90EF90DF90CF90BF90AF900895B8
:10614000EF92FF920F931F93CF93DF937C018B010C
:106150000E9495F3CAE4D2E020915A0230915B028A
:1061600040915C0250915D02F701608171818281F2
:1061700093810F94CF342C853D854E855F850F9498
:10618000D5336C877D878E879F87C8010E94382F03
:10619000DF91CF911F910F91FF90EF900C94A0236E
:1061A0008F929F92AF92BF92CF92DF92EF92FF9227
:1061B0001F93CF93DF93CDB7DEB760970FB6F894F8
:1061C000DEBF0FBECDBF182F80E00E94A6284B0176
:1061D0005C018092AC049092AD04A092AE04B092A7
:1061E000AF0481E00E94A6286B017C01C092B0043C
:1061F000D092B104E092B204F092B30482E00E9423
:10620000A6286093B4047093B5048093B604909369
:10621000B7041D861E861F86188A89829A82AB82E1
:10622000BC82CD82DE82EF82F88669877A878B878F
:106230009C8783E00E94A6286D877E878F87988B36
:106240008091570B882321F0CE0101960E943E23B6
:106250001E3FD9F480E1FE013196AAE4B2E001903C
:106260000D928A95E1F760960FB6F894DEBF0FBEE7
:10627000CDBFDF91CF911F91FF90EF90DF90CF9036
:10628000BF90AF909F908F90089584E0189FF00189
:106290001124DF01A65BBD4F81E090E08C0F9D1FB4
:1062A000E80FF91F40815181628173814D935D93A5
:1062B0006D937C931397D7CF0C949CC00F931F932F
:1062C000CF93DF93EC018B0181E00E9424C469E14C
:1062D00070E080E090E00E94E1F2B801CE010E94FF
:1062E0003130C091160680E00E9424C41092160638
:1062F00082E00E94D0300E945C31C2FBCC27C0F902
:1063000081E08C27DF91CF911F910F910895CF935A
:10631000DF93CDB7DEB72C970FB6F894DEBF0FBE74
:10632000CDBF0E947AC10E9464279CE0EEE2F5E0B6
:10633000DE01119601900D929A95E1F781110E946C
:10634000C4F2CE0101960E9427912C960FB6F894C4
:10635000DEBF0FBECDBFDF91CF9108952F923F9248
:106360004F925F926F927F928F929F92AF92BF9265
:10637000CF92DF92EF92FF920F931F93CF93DF9311
:1063800000D0CDB7DEB780904A0290904B02A0902B
:106390004C02B0904D0240904E0250904F026090DF
:1063A000500270905102C0905202D0905302E0907F
:1063B0005402F09055020E94861C0E94F92306E2C6
:1063C00012E180E392E09B838A838AE1282E82E1B6
:1063D000382E198289810E94D41CC8010E9493E83A
:1063E000EA81FB816193719381939193FB83EA83AB
:1063F000C1010E9493E8EA81FB81608771878287EF
:106400009387F981FF5FF9830C5F1F4F84E0280EAB
:10641000311CF330F9F689E095E00E94DFC10E945B
:1064200067F20E947C23A501940160914A02709159
:106430004B0280914C0290914D020F94052D8111D9
:106440001CC0A301920160914E0270914F02809195
:106450005002909151020F94052D81110EC0209190
:106460005202309153024091540250915502C7019B
:10647000B6010F94052D8823B9F00F900F900F905F
:10648000DF91CF911F910F91FF90EF90DF90CF9010
:10649000BF90AF909F908F907F906F905F904F9044
:1064A0003F902F900C9487310F900F900F90DF91B9
:1064B000CF911F910F91FF90EF90DF90CF90BF9001
:1064C000AF909F908F907F906F905F904F903F9094
:1064D0002F9008958091AB04659B6EC0806180937E
:1064E000AB04909103018091AB0491FF67C080627F
:1064F0008093AB048091AB044B9B62C0846080931B
:10650000AB048091AB049091AA04981709F45AC087
:1065100092E09093A9048093AA048091D3058111FD
:1065200005C08091B206882309F459C080912005E6
:1065300080FF10C08091D40580FD0CC08091A8041C
:1065400084FF08C08091160680618093160680E063
:106550000E94479180912005869580FF11C080910F
:10656000D405869580FD0CC08091A80485FF08C0E5
:106570008091160680628093160681E00E94479102
:10658000809120058695869580FF29C08091D4054D
:106590008695869580FF23C08091B2068823F9F006
:1065A0008091A80482FF1BC08091160684608093AE
:1065B000160682E00C9447918F7E91CF8F7D98CF05
:1065C0008B7F9DCF8091A904882309F4A6CF8150A9
:1065D0008093A9048111A1CF9093A8049ECF089520
:1065E0008091D305811104C08091B206882331F0D7
:1065F00062E070E080E090E00C94E1F208953F9258
:106600004F925F926F927F928F929F92AF92BF92C2
:10661000CF92DF92EF92FF920F931F93CF93DF936E
:1066200000D01F92CDB7DEB7382E80E090E0A0E218
:10663000B1E489839A83AB83BC83C0909E11D090D0
:106640009F11E090A011F090A11120E030E0A9018D
:10665000C701B6010F94052D87FF0CC0A701960155
:1066600060E070E080E291E40F94D43369837A8330
:106670008B839C8360E0CE0101960E945030409055
:106680004A0250904B0260904C0270904D028090F4
:106690004E0290904F02A0905002B09051023320D1
:1066A00089F10F94C20D19821A821B821C82E0901C
:1066B0005202F09053020091540210915502CE0103
:1066C00001966C01A5019401C301B2010E94532FF0
:1066D0003092B2060E94F0320F900F900F900F9000
:1066E000DF91CF911F910F91FF90EF90DF90CF90AE
:1066F000BF90AF909F908F907F906F905F904F90E2
:106700003F9008950F947F0DCECF2F923F924F92DE
:106710005F926F927F928F929F92AF92BF92CF9231
:10672000DF92EF92FF920F931F93CF93DF93CDB73A
:10673000DEB766970FB6F894DEBF0FBECDBFF82E5A
:10674000282E312CF101ED5BF04FD49022E0821322
:1067500035C08091B206811103C081E00E94FF32F2
:106760000F94C20D811139C18FE39FE00E9493E81D
:1067700020E030E0A9010F94052D8823F9F06D2D5C
:10678000DD0C770B880B990B0F940C2D2B013C0122
:106790008FE39FE00E9493E84B015C0120E030E032
:1067A00040EA50E40F94052D11E087FF1CC0812CB6
:1067B000912C90EAA92E90E4B92E15C06D2DDD0C18
:1067C000770B880B990B0F940C2D2B013C01C10109
:1067D000880F991F880F991F895C904F0E9493E83A
:1067E0004B015C0110E0A3019201C501B4010F94BB
:1067F0006B2D4B015C016101CC0CDD1CCC0CDD1C54
:10680000C601855D904F0E9493E8EE24E394E12653
:1068100020E030E040EC5FE30F946B2DA301920188
:106820000F946B2DAB01BC0100E010E098018F2D9F
:106830000E94D02820E030E0A901C501B4010F94E6
:10684000052DF601E15EF04FFA8BE98B882309F400
:106850004DC0F2E000E010E020E431E4FF1619F052
:1068600000E010E09801B501A4017058E12C8F2DD3
:106870000E94D028A5019401C501B4010F94D5331D
:106880006B8B7C8B8D8B9E8B22E0F216E9F0F101F5
:10689000E45EF04F6491611107C00F94A10B8AEF81
:1068A0009EE00E94B1F76AE070E090E080E00F9413
:1068B0000A2D9B01AC0160E070E088E492E40F9443
:1068C000CF348B019C0104C000E010E020EC30E4E8
:1068D000EE24E3944B895C896D897E898F2D0E941B
:1068E000D02832E0F312D0C00F947F0D81E090E009
:1068F000A0E0B0E00F2C04C0880F991FAA1FBB1F97
:106900000A94D2F72091560B282B2093560B2091F6
:106910009204822B8093920489899A890E9493E839
:10692000F601E65BFD4F608371838283938382E08F
:10693000F8121AC020919E1130919F114091A01120
:106940005091A111609152027091530280915402B2
:10695000909155020F94D433609352027093530276
:106960008093540290935502F601E85DF84F10822F
:106970001182128213828F2D0E94D41C0E945C31DE
:10698000F601E65BFD4F80819181A281B381F60122
:10699000EE55F94F80839183A283B38392E0F91679
:1069A000A9F18CE0E7E9F2E0DE01119601900D9289
:1069B0008A95E1F7E1E0F0E0EC0FFD1FEC0DFD1D25
:1069C00080809180A280B38020E030E0A901C501E1
:1069D000B4010F94052D81111EC066960FB6F89470
:1069E000DEBF0FBECDBFDF91CF911F910F91FF9002
:1069F000EF90DF90CF90BF90AF909F908F907F905F
:106A00006F905F904F903F902F9008950E9499E86B
:106A10008111E3CFC6CF20E030E0A901C501B40168
:106A20000F94353687FF04C0B7FAB094B7F8B09426
:106A3000F601E65BFD4F6F01A3019201C501B401B0
:106A40000F946B2D9B01AC01F601608171818281F5
:106A500093810F94D433F60160837183828393838F
:106A6000F2E080E090E0A0E4B1E4FF1621F080E0E5
:106A700090E0A8E4B2E48D879E87AF87B88BCE0103
:106A80000D960E94382FA9CF81E090E0A0E0B0E001
:106A90000F2C04C0880F991FAA1FBB1F0A94D2F79E
:106AA0002091560B282B2093560B20919204822B79
:106AB0008093920489899A890E9493E8F601E65BA3
:106AC000FD4F60837183828393834ECF0F931F9317
:106AD00080914210813019F50E948BC80091C60444
:106AE0001091C7042091C8043091C904601B710B38
:106AF000820B930B28EE33E040E050E00F944933D3
:106B00006091CA047091CB048091CC049091CD0423
:106B1000620F731F841F951F1F910F91089560913D
:106B2000CE047091CF048091D0049091D104D6CF3F
:106B3000109242101092C6041092C7041092C8041A
:106B40001092C9041092CE041092CF041092D00477
:106B50001092D1041092CA041092CB041092CC046B
:106B60001092CD0408958F929F92AF92BF92CF92D0
:106B7000DF92EF92FF920F931F93CF93DF93CDB7E6
:106B8000DEB72C970FB6F894DEBF0FBECDBF8B01DA
:106B900040E050E068E472E44D835E836F83788761
:106BA00040E050E060EA70E449875A876B877C8751
:106BB0008130B9F1823009F459C020E030E040E082
:106BC00050E460915202709153028091540290916E
:106BD00055020F94D5334B017C0120E030E048ECA6
:106BE00053E40F943536181634F4812C912C88EC2C
:106BF000E82E93E4F92EF801A084B184C284D384F2
:106C00009401A701B501C6010F943536181614F08A
:106C100054016701C501D60189839A83AB83BC8384
:106C200048C0BE01675F7F4FC80108960E9431309F
:106C3000B8016C5F7F4FAE014B5F5F4FC8010E9490
:106C40000F300E9487312C960FB6F894DEBF0FBE2E
:106C5000CDBFDF91CF911F910F91FF90EF90DF900B
:106C6000CF90BF90AF909F908F900895F8012085AE
:106C70003185428553856091520270915302809113
:106C80005402909155020F94D5336B017C0120E0A2
:106C900030E048EC53E40F94052D87FD06C0C12C6D
:106CA000D12C28ECE22E23E4F22EC982DA82EB8288
:106CB000FC82BE01675F7F4FCE010196B7CFCF92B6
:106CC000DF92EF92FF92CF93DF93C62FFC01C0803B
:106CD000D180E280F38020E030E0A901C701B60155
:106CE0000F94052D20E030E0A90187FD14C020E0BD
:106CF00030E048EC52E4C701B6010F94353624E683
:106D000030E040E050E0181634F0C701B6010F94AF
:106D100041359B01AC01C230A0F4D0E0C15DD74F3A
:106D2000AFEFB0E00F948A3324E630E040E050E06B
:106D30000F946B332F3F310519F010F02FEF30E037
:106D40002883DF91CF91FF90EF90DF90CF9008954F
:106D5000E0E4F5E0108211821282138214820C9416
:106D600097C8EF92FF920F931F93CF93DF93CDB706
:106D7000DEB78C01EDB6FEB60F94522C01962DB7FE
:106D80003EB7281B390B0FB6F8943EBF0FBE2DBF80
:106D90008DB79EB70196B8010F944B2C0E9484C406
:106DA0000FB6F894FEBE0FBEEDBEDF91CF911F91DE
:106DB0000F91FF90EF9008958091090180FD06C02A
:106DC00080914F1383FB882780F9089580E0089510
:106DD000CF92DF92EF92FF92FC01C080D180E280DF
:106DE000F380663019F51092450510924605109211
:106DF000470510924805109249050E946D8920E0D0
:106E000030E0A901C701B6010F94052D87FF1DC011
:106E1000C12CD12C7601C701B6010F944236CB01AB
:106E2000FF90EF90DF90CF900C9482ED0E94A836F7
:106E300020E030E0A901C701B6010F94052D87FFBE
:106E400015C0C12CD12C760122C020E030E04CE0EE
:106E500053E4C701B6010F9435361816E4F6C12C79
:106E6000D12C9CE0E92E93E4F92ED5CF20E030E838
:106E700049ED53E4C701B6010F94353618163CF4BA
:106E8000C12C80E8D82E89EDE82E83E4F82EC701C6
:106E9000B6010F944236CB01FF90EF90DF90CF9078
:106EA0000C9470239091560B977081E0973009F005
:106EB00080E008952091910420FF14C020E83EE373
:106EC000629FA001639F500D729F500D1124CA0153
:106ED0009695879596958795009731F08A9500004D
:106EE000E9F708950C94E1F20895CF93DF9310929F
:106EF000150B1092A80B1092AA0B1092A90B1092CE
:106F0000A6041092A504CFEFDFEF80914F1385FD0B
:106F100007C00E948675D093CE11C093CD11F5CFD6
:106F20008FEF9FEF9093CE118093CD11DF91CF9192
:106F300008958F929F92AF92BF92CF92DF92EF927D
:106F4000FF920F931F93CF93DF937C0121E5E20E15
:106F5000F11CD7014C914A3509F0A4C06C01B2E58F
:106F6000CB0ED11CF6013081353A09F09BC0EC0103
:106F7000C05BDF4F2881233008F494C08C01005699
:106F80001F4FD8014C93E15BFF4F30833196208334
:106F9000EF54F1093081E05BFF4F30833038B1F4BA
:106FA0003196AC54B1093C913083E854F109AF5AA1
:106FB000BF4F50E040E02250330B42175307CCF450
:106FC000808132968D934F5F5F4FF7CF233031F53D
:106FD000313809F074C0FC01EC55FF4FDC01AC5AAC
:106FE000BF4F2C9120833196885A9F4FDC018C91A2
:106FF00080834801B12CA12C888190E002968A15EB
:107000009B050CF43FC0F40181914F010E941AF6D8
:107010000E9413ACFFEFAF1ABF0AEECF323821F552
:10702000FC01EC5AFF4F30814181E05BFF4F408310
:1070300031963083DC01AA55BF4F50E040E0235029
:10704000330B42175307ACF6FA01EE7FE45AFF4FB9
:10705000E80FF91F608171817C9311966C931197F1
:107060004E5F5F4F1296EDCF243019F6333809F694
:10707000FC01EC5AFF4F20813181E05BFF4F3083F0
:107080003196B0CF80E5DE011D928A95E9F78AE15D
:10709000F80111928A95E9F78AE5D7018C9385EA80
:1070A000F6018083DF91CF911F910F91FF90EF90B8
:1070B000DF90CF90BF90AF909F908F90089532381F
:1070C00009F097CFADCFCF93DF93D091421082E0FC
:1070D00092E10E94B1F78AE00E9489F78091C10B8A
:1070E000873009F449C083E08093BF0B81E080932F
:1070F000670280E190E09093E6128093E51285E0CC
:107100008093D912C2E8C093DC1284E190E1A0E040
:10711000B0E08093DD129093DE12A093DF12B09363
:10712000E01289E892E10E94993761E070E080E026
:1071300090E00E945A3781E09AE59093E61280939E
:10714000E51285E390E09093E8128093E71287E0E0
:107150008093D912C093DC1284E890E0A0E0B0E004
:107160008093DD129093DE12A093DF12B093E012B1
:1071700089E892E10E94993780914210813089F12B
:10718000823061F50E9466356093CA047093CB0427
:107190008093CC049093CD0481E0809342100E94B0
:1071A0008BC86093C6047093C7048093C8049093FF
:1071B000C904D23089F08091C2059091C30501962F
:1071C0009093C3058093C205109293041092940487
:1071D000109295041092960481E004C00E949835A4
:1071E000DBCF80E0DF91CF9108950E94ADAF109288
:1071F000550B109225020E94E0F3882351F08091F4
:107200004F1382FD06C08DE29EE09093A50B809304
:10721000A40B61E086E29EE00E94C0F80C94633803
:10722000809142108130C1F582E49EE00E94B1F766
:107230008AE00E9489F781E09AE59093E6128093B4
:10724000E51287E590E09093E8128093E71287E0DB
:107250008093D91282E88093DC1284E890E0A0E069
:10726000B0E08093DD129093DE12A093DF12B09312
:10727000E01289E892E10E94993782E080934210FF
:107280000E948BC86093CE047093CF048093D00487
:107290009093D10481E0089580E008950F931F93A7
:1072A0000E948BC80091BD051091BE052091BF05BD
:1072B0003091C005011511052105310509F067C0A0
:1072C0002091BB11222309F45FC0E091B911215034
:1072D0002093BB1121E02E0F2093B9113091BC11E6
:1072E000231302C01092B91124E0E29FF00111248F
:1072F000E354FE4E00811181228133810093B90550
:107300001093BA052093BB053093BC05600F711F25
:10731000811D911D6093BD057093BE058093BF05CF
:107320009093C0058091BB059091BC05892B61F1BC
:107330001FB7F89481E39EE00E94B1F78AE00E94B3
:1073400089F784E096E09093E6128093E51280EA54
:1073500090E89093E8128093E71287E08093D91227
:1073600082E88093DC1280EA90E0A0E0B0E08093B5
:10737000DD129093DE12A093DF12B093E01289E841
:1073800092E10E9499371FBF1F910F910895601BD2
:10739000710B820B930B97FDF7CF40981092BD05B0
:1073A0001092BE051092BF051092C005EDCF0F934D
:1073B0001F93CF93DF938C01EB019091BB11209130
:1073C000BC11921305C00E944E390E94E78CF5CF84
:1073D0008091BA1134E0839FF0011124E354FE4EF2
:1073E00011830083D383C2839F5F9093BB118F5F10
:1073F000281739F08093BA11DF91CF911F910F9127
:1074000008951092BA11F8CF2F923F924F925F9247
:107410006F927F928F929F92AF92BF92CF92DF92A4
:10742000EF92FF920F931F93CF93DF93009709F092
:10743000AAC11092AA0B1092A90B9093A604809354
:10744000A504BAE0CB2EB0E2DB2EE12CF12C15E046
:1074500002E846015701C4E1D0E010922C121092CC
:107460002B1210931F1200932212809223129092DB
:107470002412A0922512B09226128FEC91E10E9464
:10748000993721972FEF821A920AA20AB20A2097FF
:1074900021F744E1C40ED11CE11CF11C8AE5C81699
:1074A00080E2D806E104F104A1F6C12CA0E2DA2EB4
:1074B000E12CF12CD5E0C2E810922C1210922B1284
:1074C000D0931F12C0932212C0922312D092241282
:1074D000E0922512F09226128FEC91E10E949937EA
:1074E00010922C1210922B12D0931F12C0932212C2
:1074F000D701C6018C529F4FAF4FBF4F80932312CD
:1075000090932412A0932512B09326128FEC91E150
:107510000E949937EFEFCE1ADE0AEE0AFE0AFAE071
:10752000CF16F0E2DF06E104F10431F6FEEDCF2ED6
:10753000F0E2DF2EE12CF12CD5E0C2E810922C1203
:1075400010922B12D0931F12C0932212C0922312BA
:10755000D0922412E0922512F09226128FEC91E143
:107560000E9499372FEFC21AD20AE20AF20A46EEB7
:10757000C41640E2D406E104F10401F7CC24C3941C
:10758000E2E1DE2EE12CF12C0AE010E0D5E0C2E8C9
:1075900010932C1200932B12D0931F12C09322121F
:1075A000C0922312D0922412E0922512F092261259
:1075B0008FEC91E10E94993710932C1200932B12BB
:1075C000D0931F12C0932212D701C6018096A11D2D
:1075D000B11D8093231290932412A0932512B0938F
:1075E00026128FEC91E10E9499378FEFC81AD80AC2
:1075F000E80AF80AE5E0CE16E2E1DE06E104F1046D
:1076000039F60091A90B1091AA0B0115110509F08B
:10761000D6C08091A80B882309F4E1C02AE030E2AB
:1076200040E050E061EB73E08FEC91E10E9418AC18
:10763000C1E0D0E003E010E0E090A90BF090AA0BCD
:1076400035E0332E42E8242E44244A94542C64E03E
:10765000662E712C7FE1C72E74E0D72E8091A90B86
:107660009091AA0B800F911FE816F90608F0D5C07B
:10767000C7010E942FAD882309F481C08091BD10FD
:1076800060EB70E1882311F06DEB70E1FB0101907C
:107690000020E9F7CF010197861B970BF4E1FC9FCF
:1076A0009001FD9F300D1124265F3F4D50E040E0DA
:1076B000459710F0FB01128A8FEC91E10E9418AC03
:1076C000CE018F5F9D4EB0E0A0E021964E0124E0F8
:1076D000880C991C2A95E1F7FDEF8F1AFFE99F0AA4
:1076E000B12CA12C20914F1324FF7EC070922C123C
:1076F00060922B1230921F1220922212809323123A
:1077000090932412A0932512B09326128FEC91E14E
:107710000E949937D0922C12C0922B1230921F12D5
:10772000209222128092231290922412A09225126B
:10773000B09226128FEC91E10E949937B7018EEE3C
:107740009DE00E94D0F98091BD106DEB70E1811138
:1077500002C060EB70E18BEE9DE00F94930B65E14E
:107760007BE087EE9DE00F94930B60EB70E186EE7B
:107770009DE00F94930B82EE9DE00E94B1F72FEFF6
:10778000E21AF20A6BCF2091A90B3091AA0BA90142
:10779000415051096091A5047091A60468177907BA
:1077A00038F42C5F3F4F3093AA0B2093A90B45CEA2
:1077B0004430510508F43DCE24503109F4CF043053
:1077C000110569F48091A80B882331F083E090E0E3
:1077D0009093AA0B8093A90BD0E0C0E02DCFD0E00E
:1077E000C0E004E010E028CF10922C1210922B126F
:1077F00030921F122092221280932312909324120F
:10780000A0932512B09326128FEC91E10E94993734
:1078100050922C1240922B1281CFDF91CF911F9169
:107820000F91FF90EF90DF90CF90BF90AF909F901F
:107830008F907F906F905F904F903F902F90089522
:10784000AF92BF92CF92DF92EF92FF920F931F936E
:10785000CF93DF93EC0184E6C82E80E2D82EE12C92
:10786000F12C02E8A12C90E2B92E15E00093DC1275
:10787000C092DD12D092DE12E092DF12F092E0129E
:10788000B092E612A092E5121093D91289E892E123
:107890000E9499378FEFC81AD80AE80AF80A88E7D1
:1078A000C81680E2D806E104F10401F724E630E2CC
:1078B00040E050E0BE0189E892E1DF91CF911F9155
:1078C0000F91FF90EF90DF90CF90BF90AF900C940E
:1078D00018AC0F931F93CF93DF938C016F3F19F474
:1078E0001092831060E020918310862F062E000CEA
:1078F000990B2817190609F08CF56093831060E046
:1079000080EF9DE00E94C0F8C8010E94B1F78AE0B4
:107910000E9489F7C8010F94522C800F911FEC012F
:10792000C01BD10BC034D1053CF00197FC01249160
:10793000207C2038D1F3F3CFDD27AE01B80183E4FA
:1079400090E10F94732CCD5BDF4E188283E490E1BD
:10795000DF91CF911F910F910C94203CDF91CF913B
:107960001F910F910895DF92EF92FF920F931F9353
:10797000CF93DF93CDB7DEB7CA5AD1090FB6F894CB
:10798000DEBF0FBECDBFCF55DF4F188219821A82DE
:107990001B82C15AD0408091BE039091BF03A09139
:1079A000C003B091C103CB55DF4F88839983AA836D
:1079B000BB83C55AD04084E690E09093DF04809367
:1079C000DE0410920F0510920E05109210052EE0A5
:1079D00035E044E050E0BE016B557F4F8EED94E002
:1079E0000F940B0E8091DE049091DF040296909329
:1079F000DF048093DE0410920F0510920E0581E0E3
:107A0000C655DF4F8883CA5AD040CE0186559F4F56
:107A10000E94F29C2EE035E048E450E06CE57BE00B
:107A20008EED94E00F940B0E2EE035E040E150E037
:107A30006BE078E08EED94E00F940B0E8AE097ED0A
:107A4000A3EABCE3CF55DF4F88839983AA83BB8326
:107A5000C15AD040CE018F559F4F0E94E99C84E3CC
:107A600097E00E94049D8FE092E00E94FB9C8BE0D7
:107A700092E00E94E99C8091FA079091FB07A09107
:107A8000FC07B091FD0789839A83AB83BC838E0189
:107A90000F5F1F4FC8010E94E99CCF55DF4F18822E
:107AA00019821A821B82C15AD0407E018DE6E80EEF
:107AB000F11C83E0D7018C938983CE018F559F4FB2
:107AC0000E94E99CC7010E94F29CC8010E94F29C9E
:107AD0004AE0D42EDA94DD2031F0CE018F559F4F4D
:107AE0000E94E99CF7CF86E991E10E94049DCF5561
:107AF000DF4F188219821A821B82C15AD0403AE0A5
:107B0000D32EDA94DD2031F0CE018F559F4F0E94A5
:107B1000E99CF7CF85E0D82ED982F701D082C80141
:107B20000E94F29CC7010E94F29C2EE035E048E0E2
:107B300050E061E075E08EED94E00F940B0E2EE0C6
:107B400035E048E050E069EF74E08EED94E00F948A
:107B50000B0E2EE035E044E650E06EEB76E08EED65
:107B600094E00F940B0E19828FEFD7018C93C8010C
:107B70000E94FB9CC7010E94F29C2EE035E044E08D
:107B800050E06AEE72E08EED94E00F940B0E80915F
:107B9000D5058983C8010E94FB9C2EE035E040E1B9
:107BA00050E069EE74E08EED94E00F940B0E198AAC
:107BB0001A8A1B8A1C8A80E090E0A0E8BFE38D87C8
:107BC0009E87AF87B88B80910E1190910F11A09175
:107BD0001011B091111189839A83AB83BC832CEA75
:107BE00035EC47E25EE360911211709113118091C0
:107BF0001411909115110F94CF346D837E838F8370
:107C000098872CEA35EC47E25EE36091161170919B
:107C1000171180911811909119110F946B2D69878C
:107C20007A878B879C872EE035E044E150E0B801ED
:107C30008EED94E00F940B0E84E190E09A8389839B
:107C4000C8010E94D79C8091A3109091A410A0918C
:107C5000A510B091A61089839A83AB83BC832CEACC
:107C600035EC47E25EE36091A7107091A810809117
:107C7000A9109091AA100F94CF346D837E838F83C7
:107C800098872CEA35EC47E25EE36091AB10709187
:107C9000AC108091AD109091AE100F946B2D698750
:107CA0007A878B879C87C8010E94E09C8CE0E3EA7E
:107CB000F2E0D80101900D928A95E1F7C8010E9487
:107CC000E09C1982C8010E94F29C8FE790E09A83A1
:107CD0008983C8010E94D79CEFEAF2E0D8010190A5
:107CE0000D92DA94E1F72EE035E045E050E0B8017E
:107CF0008EED94E00F940B0E8091E8048983C80107
:107D00000E94FB9C80E2E4EBF2E0D80101900D922E
:107D10008A95E1F72EE035E040E250E0B8018EEDC3
:107D200094E00F940B0EF7011082C7010E94FB9C98
:107D300087E297E00E94FB9C83E297E00E94E99C27
:107D4000CF55DF4F188219821A821B82C15AD04048
:107D5000CE018F559F4F0E94E99C80E2D8011D9271
:107D60008A95E9F72EE035E040E250E0B8018EED6B
:107D700094E00F940B0EFE01F99688E0DF011D924E
:107D80008A95E9F744E650E060E070E049835A8361
:107D90006B837C834D835E836F83788783E090E081
:107DA000A0E0B0E089879A87AB87BC874D875E8764
:107DB0006F87788B498B5A8B6B8B7C8B8D8B9E8BD3
:107DC000AF8BB88F898F9A8FAB8FBC8F8D8F9E8F23
:107DD000AF8FB8A38EE190E0A0E0B0E089A39AA3B2
:107DE000ABA3BCA38DA39EA3AFA3B8A789A79AA753
:107DF000ABA7BCA78DA79EA7AFA7B8AB89AB9AAB23
:107E0000ABABBCAB8DAB9EABAFABB8AF2EE035E050
:107E100040E450E0B8018EED94E00F940B0E90E139
:107E2000D92EF8018D2D11928A95E9F72EE035E0D3
:107E300040E150E0B8018EED94E00F940B0ED801B4
:107E40001D92DA94E9F72EE035E040E150E0B80108
:107E50008EED94E00F940B0ECF55DF4F18821982F0
:107E60001A821B82C15AD040CE018F559F4F0E946B
:107E7000E99C2CE0D22EF8018D2D11928A95E9F71C
:107E80002EE035E04CE050E0B8018EED94E00F9428
:107E90000B0E8CE6D8011D928A95E9F72EE035E0AD
:107EA0004CE650E0B8018EED94E00F940B0E82ED9D
:107EB00094E00E94E09C2EE035E048E050E060EE67
:107EC00074E08EED94E00F940B0EF7011192DA94AA
:107ED000E9F7C755DF4F1882C95AD04080E090E0DB
:107EE000A0E4B0E4C356DF4F88839983AA83BB83A1
:107EF000CD59D040C7010E94049DCE0187559F4FA8
:107F00000E94F29CCE0183569F4F0E94E99C80E321
:107F1000D7011D928A95E9F782E392E10E94B1F7B9
:107F20008AE00E9489F72EE035E040E350E0B70197
:107F30008EED94E00F940B0E80911005811128C0F6
:107F40000091DE041091DF0480910E0590910F05E1
:107F5000F7019183808384E690E09093DF0480931F
:107F6000DE042EE035E044E050E06AEF72E08EED92
:107F700094E00F940B0EC7010E94D79C91E0053747
:107F8000134009F490E080911005892B809310052F
:107F900080911005811105C060E086E692E10E94A3
:107FA000693C86E492E10E94B1F78AE00E9489F779
:107FB0009091100581E08927C655DF4F0FB6F894E0
:107FC000DEBF0FBECDBFDF91CF911F910F91FF900C
:107FD000EF90DF9008951092550B1092250280913A
:107FE0004F13806480934F1361E08EEF9DE00E94F9
:107FF000C0F843E15EE06BE17EE085E00E9432AED6
:1080000060E085E09EE00C94693CCF92DF92EF92B5
:10801000FF920F931F93CF93DF93CDB7DEB77C0111
:10802000CDB6DEB60F94522C01962DB73EB7281B65
:10803000390B0FB6F8943EBF0FBE2DBF0DB71EB75C
:108040000F5F1F4FB701C8010F944B2CF80101902F
:108050000020E9F73197E01BF10B759720F084EDD4
:1080600092E0F801848BC8010E94203C0FB6F8947E
:10807000DEBE0FBECDBEDF91CF911F910F91FF905D
:10808000EF90DF90CF900895CF93DF9300D01F92B1
:10809000CDB7DEB787EB9DE00E94B1F78AE00E9482
:1080A00089F78091C10B8330D9F119821A821B8222
:1080B0001C8260E0CE0101960E945F3619821A820E
:1080C0001B821C8261E0CE0101960E945F3681E036
:1080D000809366021092BE0B8093670281E09AE55E
:1080E0009093E6128093E51283E390E09093E81278
:1080F0008093E71287E08093D91282E88093DC12A4
:1081000084E890E0A0E0B0E08093DD129093DE126E
:10811000A093DF12B093E01289E892E10E949937B0
:108120000F900F900F900F90DF91CF910895CF9205
:10813000DF92EF92FF92CF93C82F8091421081502F
:10814000823008F069C00E944440109242100E94A0
:108150008BC86093CE047093CF048093D004909327
:10816000D104C0909304D0909404E0909504F090D2
:1081700096040E946635AB01BC0140939304509372
:10818000940460939504709396048091C605909131
:10819000C705A091C805B091C9058C199D09AE0904
:1081A000BF09840F951FA61FB71F8093C605909324
:1081B000C705A093C805B093C905C1110AC0C1E0A5
:1081C0000E94E6228C2FCF91FF90EF90DF90CF900E
:1081D00008958091C4059091C50501969093C505B9
:1081E0008093C4050E946635C090CA05D090CB0527
:1081F000E090CC05F090CD05C616D706E806F90646
:10820000F0F60E9466356093CA057093CB058093A3
:10821000CC059093CD05D3CFC0E0D2CF8F929F9263
:10822000AF92BF92CF92DF92EF92FF920F931F9384
:10823000CF93DF930E9475373AE0C32E30E2D32EFE
:10824000E12CF12C15E002E846015701CAE0D0E02C
:108250001092E6121092E5121093D9120093DC12DC
:108260008092DD129092DE12A092DF12B092E012A4
:1082700089E892E10E94993721978FEF881A980A2E
:10828000A80AB80A209721F78AE0C80ED11CE11C81
:10829000F11C82EDC81680E2D806E104F104A1F6D3
:1082A000C12C20E2D22EE12CF12CD5E0C2E81092B4
:1082B000E6121092E512D093D912C093DC12C0924C
:1082C000DD12D092DE12E092DF12F092E01289E825
:1082D00092E10E9499371092E6121092E512D09323
:1082E000D912C093DC12D701C6018C529F4FAF4FF9
:1082F000BF4F8093DD129093DE12A093DF12B093F4
:10830000E01289E892E10E9499378FEFC81AD80AE3
:10831000E80AF80A8AE0C81680E2D806E104F10407
:1083200031F69EEDC92E90E2D92EE12CF12CD5E04C
:10833000C2E81092E6121092E512D093D912C093BF
:10834000DC12C092DD12D092DE12E092DF12F092C7
:10835000E01289E892E10E9499378FEFC81AD80A93
:10836000E80AF80A86EEC81680E2D806E104F104AD
:1083700001F7CC24C39482E1D82EE12CF12C0AE041
:1083800010E0D5E0C2E81093E6120093E512D09316
:10839000D912C093DC12C092DD12D092DE12E092AC
:1083A000DF12F092E01289E892E10E94993710936F
:1083B000E6120093E512D093D912C093DC12D701D4
:1083C000C6018096A11DB11D8093DD129093DE122F
:1083D000A093DF12B093E01289E892E10E949937EE
:1083E0008FEFC81AD80AE80AF80A85E1C81682E1B0
:1083F000D806E104F10439F682E190E09093E612A8
:108400008093E512D093D912C093DC1284E190E1FD
:10841000A0E0B0E08093DD129093DE12A093DF1213
:10842000B093E01289E892E1DF91CF911F910F9113
:10843000FF90EF90DF90CF90BF90AF909F908F9084
:108440000C9499374F925F926F927F928F929F9286
:10845000AF92BF92CF92DF92EF92FF920F931F9352
:10846000CF93DF9300D000D01F921F92CDB7DEB71D
:108470008091A30481110AC48091A1049091A20467
:108480009C012F5F3F4F3093A2042093A1048E3EA6
:10849000924008F4FBC38091091190910A119093C6
:1084A000E6128093E51205E00093D91212E81093CA
:1084B000DC1286E390E1A0E0B0E08093DD129093BF
:1084C000DE12A093DF12B093E01289E892E10E94DD
:1084D000993780919E1090919F109093E61280930F
:1084E000E5120093D9121093DC128CE390E1A0E026
:1084F000B0E08093DD129093DE12A093DF12B09370
:10850000E01289E892E10E94993780910B119091D5
:108510000C119093E6128093E5120093D9121093F8
:10852000DC1284E390E1A0E0B0E08093DD12909350
:10853000DE12A093DF12B093E01289E892E10E946C
:1085400099378091A0109091A1109093E61280939A
:10855000E5120093D9121093DC128AE390E1A0E0B7
:10856000B0E08093DD129093DE12A093DF12B093FF
:10857000E01289E892E10E94993781E08093A30498
:108580001092A2041092A1048091C10B882339F1AA
:108590000E94F41C811123C08091A0048F5F8093FE
:1085A000A0048091A004853620F01092A0041092BF
:1085B000C10BE091C10BE150E73008F06AC00E2E0C
:1085C000000CFF0B8827E851FD4B8F4F0D94CC33E7
:1085D000F24241430D4539457A45B2454543109233
:1085E000A004DFCF0E945237882309F452C081E0F3
:1085F0008093670289EA9DE00E94B1F78AE00E94B9
:1086000089F780E190E09093E6128093E51285E08F
:108610008093D91212E81093DC1284E190E1A0E07B
:10862000B0E08093DD129093DE12A093DF12B0933E
:10863000E01289E892E10E94993781E09AE59093EF
:10864000E6128093E51286E390E09093E81280931F
:10865000E71287E08093D9121093DC1284E890E04F
:10866000A0E0B0E08093DD129093DE12A093DF12C1
:10867000B093E01289E892E10E9499371092C10B01
:1086800008C00E945237882321F00E94F41C8823DE
:10869000A9F380916702882309F433C78091A40469
:1086A0008111C0C284E096E09093E6128093E512B7
:1086B00080EA90E89093E8128093E71217E0109315
:1086C000D91202E80093DC1280EA90E0A0E0B0E06A
:1086D0008093DD129093DE12A093DF12B093E0122C
:1086E00089E892E10E949937809162029091630239
:1086F000A0916402B09165020097A105B10509F04F
:108700003FC21092E6121092E51215E01093D912B2
:108710000093DC128AE890E1A0E0B0E08093DD12E3
:108720009093DE12A093DF12B093E01289E892E1F9
:108730000E94993789E090E09093E6128093E512C9
:108740001093D9120093DC128CE890E1A0E0B0E025
:108750008093DD129093DE12A093DF12B093E012AB
:1087600089E892E10E9499378091620290916302B8
:10877000A0916402B09165020097F1E0AF07B105E6
:1087800008F441C2B093E612A093E5129093E81268
:108790008093E71287E08093D91282E88093DC12FD
:1087A00088E890E1A0E0B0E08093DD129093DE12C3
:1087B000A093DF12B093E01289E892E10E9499370A
:1087C0008091620290916302A0916402B09165026F
:1087D000BA2FA92F982F8827009721E0A207B1056B
:1087E00008F417C2B093E612A093E5129093E81232
:1087F0008093E71287E08093D91212E81093DC127D
:1088000081EA90E0A0E0B0E08093DD129093DE1268
:10881000A093DF12B093E01289E892E10E949937A9
:108820008091570B882309F4FAC183E090E090937C
:10883000E6128093E51285E08093D9121093DC1242
:1088400085E490E1A0E0B0E08093DD129093DE1229
:10885000A093DF12B093E01289E892E10E94993769
:108860008091A404875E8093A4042091A404822FA5
:1088700090E0253608F021C29093E6128093E5122D
:1088800085E08093D91282E88093DC1280E090E149
:10889000A0E0B0E08093DD129093DE12A093DF128F
:1088A000B093E01289E892E10E9499370E94F41C8B
:1088B000811114C20E94E0F3811105C090919104CE
:1088C00091FD0E94F41C9091910480FB91F990938A
:1088D000910491FD03C280914F1382FDFFC18091ED
:1088E00042108150823008F4F9C16091A01070915B
:1088F000A110072E000C880B990B0F940C2D6B0107
:108900007C0120E030E0A9010F94052D882309F4B3
:10891000BBC660919E1070919F10072E000C880BB3
:10892000990B0F940C2D2B013C0120E030E040E02E
:1089300050E4C701B6010F94D433A30192010F9400
:10894000353618160CF4C2C66091091170910A11DF
:10895000072E000C880B990B0F940C2D6D837E83D2
:108960008F83988760910B1170910C11072E000C6A
:10897000880B990B0F940C2D4B015C0120E030E02B
:1089800040E251E40F94D4332D813E814F815885CC
:108990000F94353618160CF499C620E030E040E00C
:1089A00050E4C701B6010F94D533A30192010F948F
:1089B000052D87FD10C020E030E040E251E4C50104
:1089C000B4010F94D5332D813E814F8158850F948A
:1089D000052D87FF6AC684E190E09093E6128093AC
:1089E000E51285E08093D91282E88093DC1284E15D
:1089F00090E1A0E0B0E08093DD129093DE12A093AE
:108A0000DF12B093E01289E892E10E9499378091D9
:108A1000BF0B81117CC682E07AC68BE99DE00E9483
:108A2000B1F78AE00E9489F781E09AE59093E61217
:108A30008093E51280E490E09093E8128093E7122F
:108A400017E01093D91282E88093DC1284E890E05A
:108A5000A0E0B0E08093DD129093DE12A093DF12CD
:108A6000B093E01289E892E10E9499371093C10B0C
:108A700010CE8091AE0B882309F40BCE0E945237A2
:108A8000882309F406CE0E94F41C811102CE8DE8E1
:108A90009DE00E94B1F78AE00E9489F78091AF0BB8
:108AA00090E0B0E0A0E0895B9F4FAE4FB54A21E077
:108AB0003AE53093E6122093E5129093E812809302
:108AC000E71287E08093D91282E88093DC1284E871
:108AD00090E0A0E0B0E08093DD129093DE12A093CE
:108AE000DF12B093E01289E892E10E949937109268
:108AF000AE0BC4CD0E945237882309F4CACD0E9420
:108B0000F41C8111C6CD81E0809367021092C10BE5
:108B10008FE79DE00E94B1F78AE00E9489F781E02B
:108B20009AE59093E6128093E5128EE490E090939C
:108B3000E8128093E71287E08093D91282E880934D
:108B4000DC1284E890E0A0E0B0E08093DD12909326
:108B5000DE12A093DF12B093E01289E892E10E9446
:108B6000993797CD0E94F41C811193CD19821A82F6
:108B70001B821C8262E0CE0101960E94FABF7ECD6C
:108B80000196A11DB11D35E0B695A79597958795DE
:108B90003A95D1F70197A109B1090097E1E0AE0735
:108BA000B10548F1B093E612A093E5129093E81254
:108BB0008093E7121093D91212E81093DC128AE81E
:108BC00090E1A0E0B0E08093DD129093DE12A093DC
:108BD000DF12B093E01289E892E10E94993788E0B1
:108BE00090E09093E6128093E51285E08093D9128D
:108BF0001093DC12A9CD9093E6128093E51285E0E4
:108C00008093D912D9CF9093E6128093E51285E034
:108C1000C2CD9093E6128093E51285E0ECCD82E020
:108C200090E005CE8A3F08F020CE8EEF8093A4041A
:108C30008EE69DE00E94B1F78AE00E9489F781E00C
:108C40008093670281E09AE59093E6128093E512A3
:108C50008DE290E09093E8128093E71287E0809392
:108C6000D91282E88093DC1284E890E0A0E0B0E0C2
:108C70008093DD129093DE12A093DF12B093E01286
:108C800089E892E10E9499371092A30428960FB6C2
:108C9000F894DEBF0FBECDBFDF91CF911F910F9132
:108CA000FF90EF90DF90CF90BF90AF909F908F900C
:108CB0007F906F905F904F900895845691099093A4
:108CC000E6128093E51285E08093D91282E88093C2
:108CD000DC1281E090E1A0E0B0E0DCCD8CE090E03F
:108CE0009093E6128093E51215E01093D91282E872
:108CF0008093DC1284E190E1A0E0B0E08093DD128B
:108D00009093DE12A093DF12B093E01289E892E113
:108D10000E9499370E94663520E13EE040E050E035
:108D20000F9449332115310581E04807510508F4B6
:108D300070C05093E6124093E5123093E8122093EE
:108D4000E71287E08093D91212E81093DC1280E1D9
:108D500090E1A0E0B0E08093DD129093DE12A0934A
:108D6000DF12B093E01289E892E10E9499370E94E5
:108D7000663520E13EE040E050E00F9449332CE3BB
:108D800030E040E050E00F9449333093E6122093F6
:108D9000E51205E00093D9121093DC1282E190E114
:108DA000A0E0B0E08093DD129093DE12A093DF127A
:108DB000B093E01289E892E10E9499370E94641F03
:108DC000882309F45CC48F5F80939F04E82EF12C04
:108DD000833330F5EE0CFF1CF092E612E092E512C0
:108DE0000093D9121093DC128EE090E1A0E0B0E085
:108DF0008093DD129093DE12A093DF12B093E01205
:108E000089E892E10E9499371092E6121092E512D9
:108E10002BC03093E6122093E5121093D91294CF11
:108E200084E690E09093E6128093E5120093D912C5
:108E30001093DC128EE090E1A0E0B0E08093DD12B0
:108E40009093DE12A093DF12B093E01289E892E1D2
:108E50000E949937A2E3EA1AA0E8FA0AEE0CFF1C76
:108E6000F092E612E092E5120093D9121093DC1210
:108E70008FE090E1A0E0B0E08093DD129093DE12ED
:108E8000A093DF12B093E01289E892E10E94993733
:108E90000E94641F90E09093E6128093E51285E0B3
:108EA0008093D91282E88093DC1286E190E1A0E001
:108EB000B0E08093DD129093DE12A093DF12B093A6
:108EC000E01289E892E10E94993720E030E0A901A0
:108ED00060919E1170919F118091A0119091A111AC
:108EE0000F94D53320E030E048EC52E40F946B2D22
:108EF0000F9441357093E6126093E51205E00093FC
:108F0000D91212E81093DC1286E290E1A0E0B0E002
:108F10008093DD129093DE12A093DF12B093E012E3
:108F200089E892E10E94993780915E0290915F02F8
:108F30009093E6128093E5120093D9121093DC12FD
:108F400080E093E1A0E0B0E08093DD129093DE1228
:108F5000A093DF12B093E01289E892E10E94993762
:108F600020E030E040E251E46091700B7091710BB1
:108F70008091720B9091730B0F946B2D0F94483569
:108F80007093E6126093E5120093D9121093DC12ED
:108F900082E492E1A0E0B0E08093DD129093DE12D3
:108FA000A093DF12B093E01289E892E10E94993712
:108FB00020E030E040E251E46091740B7091750B59
:108FC0008091760B9091770B0F946B2D0F94483511
:108FD0007093E6126093E5120093D9121093DC129D
:108FE00086E492E1A0E0B0E08093DD129093DE127F
:108FF000A093DF12B093E01289E892E10E949937C2
:1090000020E030E040E251E46091780B7091790B00
:1090100080917A0B90917B0B0F946B2D0F944835B8
:109020007093E6126093E5120093D9121093DC124C
:109030008AE492E1A0E0B0E08093DD129093DE122A
:10904000A093DF12B093E01289E892E10E94993771
:1090500020E030E040E251E460917C0B70917D0BA8
:1090600080917E0B90917F0B0F946B2D0F94483560
:109070007093E6126093E5120093D9121093DC12FC
:109080008EE492E1A0E0B0E08093DD129093DE12D6
:10909000A093DF12B093E01289E892E10E94993721
:1090A00020E030E048EC52E4609196117091971105
:1090B00080919811909199110F946B2D0F944135D7
:1090C0007093E6126093E5120093D9121093DC12AC
:1090D00086E392E1A0E0B0E08093DD129093DE128F
:1090E000A093DF12B093E01289E892E10E949937D1
:1090F00020E030E048EC52E460919A1170919B11AD
:1091000080919C1190919D110F946B2D0F9441357E
:109110007093E6126093E5120093D9121093DC125B
:109120008AE392E1A0E0B0E08093DD129093DE123A
:10913000A093DF12B093E01289E892E10E94993780
:1091400080916E0290916F029093E6128093E512E7
:109150000093D9121093DC1282E592E1A0E0B0E016
:109160008093DD129093DE12A093DF12B093E01291
:1091700089E892E10E94993780916C0290916D028A
:109180009093E6128093E5120093D9121093DC12AB
:1091900084E592E1A0E0B0E08093DD129093DE12CE
:1091A000A093DF12B093E01289E892E10E94993710
:1091B00020E030E040E251E460910E1170910F1117
:1091C00080911011909111110F946B2D0F944835CF
:1091D0007093E6126093E5120093D9121093DC129B
:1091E00086E592E1A0E0B0E08093DD129093DE127C
:1091F000A093DF12B093E01289E892E10E949937C0
:109200002CEA35EC47E25EE3609112117091131184
:1092100080911411909115110F94CF3420E030E01B
:1092200040E251E40F946B2D0F9448357093E61291
:109230006093E5120093D9121093DC128AE592E153
:10924000A0E0B0E08093DD129093DE12A093DF12D5
:10925000B093E01289E892E10E9499372CEA35EC4C
:1092600047E25EE360911611709117118091181119
:10927000909119110F946B2D20E030E040E251E401
:109280000F946B2D0F9448357093E6126093E5129E
:109290000093D9121093DC128EE592E1A0E0B0E0C9
:1092A0008093DD129093DE12A093DF12B093E01250
:1092B00089E892E10E94993720E030E040E251E4F1
:1092C0006091A3107091A4108091A5109091A610A8
:1092D0000F946B2D0F9448357093E6126093E5124E
:1092E0000093D9121093DC1282E692E1A0E0B0E084
:1092F0008093DD129093DE12A093DF12B093E01200
:1093000089E892E10E9499372CEA35EC47E25EE366
:109310006091A7107091A8108091A9109091AA1047
:109320000F94CF3420E030E040E251E40F946B2DF5
:109330000F9448357093E6126093E5120093D912AA
:109340001093DC1286E692E1A0E0B0E08093DD129B
:109350009093DE12A093DF12B093E01289E892E1BD
:109360000E9499372CEA35EC47E25EE36091AB103E
:109370007091AC108091AD109091AE100F946B2D48
:1093800020E030E040E251E40F946B2D0F9448351B
:109390007093E6126093E5120093D9121093DC12D9
:1093A0008AE692E1A0E0B0E08093DD129093DE12B5
:1093B000A093DF12B093E01289E892E10E949937FE
:1093C0008091B80B811105C08091BA0B882309F4F4
:1093D0006DC06091091170910A11072E000C880B65
:1093E000990B0F940C2D20E030E048EC52E40F94E0
:1093F0006B2D6B017C0160910B1170910C11072E8C
:10940000000C880B990B0F940C2D9B01AC01C7012C
:10941000B6010F94CF340F9448356536710510F0BE
:1094200064E670E07093E6126093E51205E0009345
:10943000D91212E81093DC1284E290E1A0E0B0E0CF
:109440008093DD129093DE12A093DF12B093E012AE
:1094500089E892E10E9499376091091170910A118F
:10946000072E000C880B990B0F940C2D6B017C01BF
:1094700020E030E04AE253E40F943536181624F425
:109480008091B80B811146C160910B1170910C1144
:10949000072E000C880B990B0F940C2D9B01AC012F
:1094A000C701B6010F94353687FFAFC18091AE0B6F
:1094B000882339F18091AD0B91E0980F9093AD0B1B
:1094C00090E09093E6128093E51285E08093D912A4
:1094D00082E88093DC1282E490E1A0E0B0E0809327
:1094E000DD129093DE12A093DF12B093E01289E8B0
:1094F00092E10E9499378091AD0B8A3010F0109262
:10950000AD0B0E94DC36882309F4B5C16091A60B2F
:109510007091A70BEE24E394F12C61157105A9F06D
:1095200090E080E00F940A2D20E030E040E85EE318
:109530000F946B2D0F94B33420E030E040E85FE3EC
:109540000F94D5330F9448357B0101E010E08091F2
:10955000A80B811102C010E000E08091CD11909124
:10956000CE118F3F980711F40E947C7E9093CE110C
:109570008093CD11080F191FB80190E080E00F947F
:109580000A2D20E030E040E85EE30F946B2D0F944D
:10959000B3344B015C01F092E612E092E51205E073
:1095A0000093D91212E81093DC1280E193E1A0E05D
:1095B000B0E08093DD129093DE12A093DF12B0939F
:1095C000E01289E892E10E949937C501B4010F9435
:1095D00048357093E6126093E5120093D912109308
:1095E000DC1282E193E1A0E0B0E08093DD12909381
:1095F000DE12A093DF12B093E01289E892E10E949C
:10960000993709E213E1AAE1FA2E80914F04909173
:10961000500420919D0430919E04891B8F7309F49E
:1096200049C12A3131050CF0DBC190914F04809182
:1096300050044FEF5FEF981749F0E82FF0E0E15B3F
:10964000FB4F42818F5F8F7380935004F901E75D78
:10965000FC4E4083809129138A3509F0B3C162E042
:1096600070E080E090E00E945A3780919D049091D4
:109670009E04019690939E0480939D04C6CF109201
:10968000E6121092E512ACCB60910B1170910C11A7
:10969000072E000C880B990B0F940C2D20E030E066
:1096A000A9010F94052D811134C98CE090E09093AD
:1096B000E6128093E51285E08093D91282E88093C8
:1096C000DC1284E190E1A0E0B0E0F3CB8DE090E02B
:1096D0009093E6128093E51285E08093D91282E898
:1096E0008093DC1284E190E1A0E0B0E08093DD1291
:1096F0009093DE12A093DF12B093E01289E892E11A
:109700000E9499378091BF0B811101C081E0809345
:10971000BF0BDBCB1092B80B20E030E040E251E40D
:109720006091B00B7091B10B8091B20B9091B30B23
:109730000F946B2D0F9441357093E6126093E512F0
:109740000093D9121093DC1284E590E1A0E0B0E020
:109750008093DD129093DE12A093DF12B093E0129B
:1097600089E892E10E94993720E030E040E251E43C
:109770006091B40B7091B50B8091B60B9091B70BC3
:109780000F946B2D0F9441357093E6126093E512A0
:109790000093D9121093DC1288E590E1A0E0B0E0CC
:1097A0008093DD129093DE12A093DF12B093E0124B
:1097B00089E892E10E9499378DE49DE00E94B1F71B
:1097C0008AE00E9489F781E09AE59093E6128093FF
:1097D000E51281E490E09093E8128093E71287E02D
:1097E0008093D9121093DC1284E890E0A0E0B0E0FE
:1097F0008093DD129093DE12A093DF12B093E012FB
:1098000089E892E10E94993751CE6091BA0B6623A4
:1098100009F44CCE062E000C770B84E39DE00E94E9
:1098200004FA8AE00E9489F71092BA0B84E090E073
:109830009093E6128093E51285E08093D91212E8A6
:109840001093DC128EE890E1A0E0B0E08093DD128E
:109850009093DE12A093DF12B093E01289E892E1B8
:109860000E94993781E09AE59093E6128093E51281
:1098700083E590E0B0CF1092E6121092E51205E079
:109880000093D91212E81093DC1280E193E1A0E07A
:10989000B0E08093DD129093DE12A093DF12B093BC
:1098A000E01289E892E10E9499371092E612109234
:1098B000E51293CE121613060CF492C080918D120D
:1098C00090918E12A0918F12B09190128C34E0E1A1
:1098D0009E07A105B10509F4D7C98A349041A105B5
:1098E000B10509F4D1C920E030E040E251E46091D3
:1098F0004A0270914B0280914C0290914D020F945C
:109900006B2D0F9441357093E6126093E51205E0DC
:109910000093D91212E81093DC1288E490E1A0E0E1
:10992000B0E08093DD129093DE12A093DF12B0932B
:10993000E01289E892E10E94993720E030E040E2AD
:1099400051E460914E0270914F02809150029091CB
:1099500051020F946B2D0F9441357093E612609372
:10996000E5120093D9121093DC128AE490E1A0E092
:10997000B0E08093DD129093DE12A093DF12B093DB
:10998000E01289E892E10E94993720E030E040E25D
:1099900051E460915202709153028091540290916F
:1099A00055020F946B2D0F9441357093E61260931E
:1099B000E5120093D9121093DC128CE490E1A0E040
:1099C000B0E056C9121613060CF01FCEF8012F2D69
:1099D00011922A95E9F710929E0410929D0415CEDB
:1099E00090918A1280912913981321C090918B1223
:1099F00080912A1398131BC023303105C4F0909135
:109A00002B139093891280912C1380938C12933096
:109A1000D1F4982F9D7F9038B1F490912D139F34FD
:109A200009F059C090912E139B3409F054C0E9E21B
:109A3000F3E18AE1DF011D928A95E9F710929E0415
:109A400010929D043BCF833809F045C080912D13BF
:109A500090912E13982789279827B0E0A0E0809353
:109A60008D1290938E12A0938F12B0939012C0908B
:109A70002F13D12CF12CE12CC0929112D092921282
:109A8000E0929312F092941220E333E140E050E030
:109A9000BA014C155D056E057F0508F04AC0DB0173
:109AA000CA01B695A795979587950696880F991F31
:109AB000FC01E757FD4ED9018C9111969C918927A5
:109AC00098278927918380834E5F5F4F6F4F7F4F29
:109AD0002E5F3F4FDECF813861F580912D1390E0EE
:109AE000B0E0A0E080938D1290938E12A0938F121D
:109AF000B093901280912E13482F50E070E060E0F8
:109B00004093911250939212609393127093941217
:109B1000AFE2B3E1E5E9F2E190E030E020E0821766
:109B2000930739F04D9150E0419351932F5F3F4F90
:109B3000F6CFE9E2F3E18AE1DF011D928A95E9F7C8
:109B400010929E0410929D040E943BC9B7CE6F9262
:109B50007F928F929F92AF92BF92CF92DF92EF92BD
:109B6000FF920F931F93CF93DF93CDB7DEB7649728
:109B70000FB6F894DEBF0FBECDBF1092D00080911B
:109B8000D00082608093D0001092D50080E1809355
:109B9000D4008091D10080618093D1008091D10068
:109BA00088608093D1008091D10080688093D1003B
:109BB0008091D1008F7D8093D1008AE58093DA1265
:109BC00080938A1285EA8093DB1280938B12E9E2FC
:109BD000F3E18AE1DF011D928A95E9F78091BD0BDF
:109BE000882309F473C283E090E09093E612809397
:109BF000E51285E08093D91282E88093DC128FE130
:109C000090E1A0E0B0E08093DD129093DE12A0938B
:109C1000DF12B093E01289E892E10E94993784E65E
:109C200090E09093E6128093E51205E00093D9123C
:109C300012E81093DC1286E090E1A0E0B0E080939F
:109C4000DD129093DE12A093DF12B093E01289E848
:109C500092E10E9499378BE090E09093E612809316
:109C6000E5120093D9121093DC1280E092E1A0E09B
:109C7000B0E08093DD129093DE12A093DF12B093D8
:109C8000E01289E892E10E9499371092E612109250
:109C9000E5120093D9121093DC1284E390E1A0E066
:109CA000B0E08093DD129093DE12A093DF12B093A8
:109CB000E01289E892E10E9499371092E612109220
:109CC000E5120093D9121093DC128AE390E1A0E030
:109CD000B0E08093DD129093DE12A093DF12B09378
:109CE000E01289E892E10E949937809109119091E0
:109CF0000A119093E6128093E5120093D912109303
:109D0000DC1286E390E1A0E0B0E08093DD12909356
:109D1000DE12A093DF12B093E01289E892E10E9474
:109D2000993780919E1090919F109093E6128093A6
:109D3000E5120093D9121093DC128CE390E1A0E0BD
:109D4000B0E08093DD129093DE12A093DF12B09307
:109D5000E01289E892E10E94993782E090E09093C6
:109D6000E6128093E5120093D9121093DC128EE173
:109D700090E1A0E0B0E08093DD129093DE12A0931A
:109D8000DF12B093E01289E892E10E94993781E0F6
:109D90008093660270E6C72E70E1D72EE12CF12C7D
:109DA0001092E6121092E5120093D9121093DC1271
:109DB000C092DD12D092DE12E092DF12F092E01239
:109DC00089E892E10E949937BFEFCB1ADB0AEB0AD0
:109DD000FB0AE4E7CE16E0E1DE06E104F10401F758
:109DE000CE0101967C0184E1D7011D928A95E9F7A5
:109DF00081E08F9390E99F938F9398E69F938F9341
:109E00009F9382EC93E09F938F93FF92EF920F9436
:109E10005D3720E630E140E050E06FEC73E089E828
:109E200092E10E9418AC2AE630E140E050E06CED8F
:109E300073E089E892E10E9418AC24E730E140E049
:109E400050E0B70189E892E10E9418AC2EE730E1BA
:109E500040E050E068EE73E089E892E10E9418ACBF
:109E60001092E6121092E5120093D9121093DC12B0
:109E70008EE090E1A0E0B0E08093DD129093DE12DE
:109E8000A093DF12B093E01289E892E10E94993723
:109E90001092E6121092E5120093D9121093DC1280
:109EA0008FE090E1A0E0B0E08093DD129093DE12AD
:109EB000A093DF12B093E01289E892E10E949937F3
:109EC0000FB6F894DEBF0FBECDBF4AE0C42E40E20D
:109ED000D42EE12CF12C55E0752E62E8662E460159
:109EE00057010AE010E01092E6121092E51270920B
:109EF000D9126092DC128092DD129092DE12A09252
:109F0000DF12B092E01289E892E10E949937015085
:109F10001109FFEF8F1A9F0AAF0ABF0A0115110539
:109F200011F78AE0C80ED11CE11CF11C92EDC91694
:109F300090E2D906E104F10491F6C12C30E2D32E6F
:109F4000E12CF12C05E012E81092E6121092E512D5
:109F50000093D9121093DC12C092DD12D092DE125F
:109F6000E092DF12F092E01289E892E10E949937C4
:109F70001092E6121092E5120093D9121093DC129F
:109F8000D701C6018C529F4FAF4FBF4F8093DD1258
:109F90009093DE12A093DF12B093E01289E892E171
:109FA0000E949937AFEFCA1ADA0AEA0AFA0ABAE047
:109FB000CB16B0E2DB06E104F10431F62EEDC22E41
:109FC00020E2D22EE12CF12C05E012E81092E612EC
:109FD0001092E5120093D9121093DC12C092DD1298
:109FE000D092DE12E092DF12F092E01289E892E164
:109FF0000E949937EFEFCE1ADE0AEE0AFE0AF6EE5D
:10A00000CF16F0E2DF06E104F10401F7CC24C3949B
:10A0100082E1D82EE12CF12C9AE0A92EB12C05E09A
:10A0200012E8B092E612A092E5120093D9121093B2
:10A03000DC12C092DD12D092DE12E092DF12F092BA
:10A04000E01289E892E10E949937B092E612A0925C
:10A05000E5120093D9121093DC12D701C601809645
:10A06000A11DB11D8093DD129093DE12A093DF122B
:10A07000B093E01289E892E10E9499378FEFC81AF5
:10A08000D80AE80AF80A95E1C91692E1D906E1046E
:10A09000F10439F68DE19DE00E94B1F78AE00E945B
:10A0A00089F764960FB6F894DEBF0FBECDBFDF917F
:10A0B000CF911F910F91FF90EF90DF90CF90BF90C5
:10A0C000AF909F908F907F906F90089582E090E086
:10A0D0008CCD0E94A74D1092A40481E0809367026A
:10A0E0008FEC9DE00E94B1F78AE00C9489F7AB01F8
:10A0F000BC0140934B1350934C1360934D137093DA
:10A100004E1383EB94E10C94257ACF93DF93DB011C
:10A11000F9019C919130C1F0943080F094509C935F
:10A120008830D1F480819181009771F001979183FB
:10A130008083480F591FEA01188206C08C3539F414
:10A140009C5F9C93943041F4DF91CF9108958B33C1
:10A1500039F781E08C93F8CF20813181B9016F5FAD
:10A160007F4F71836083420F531FEA018883808190
:10A1700091818F3591056CF7E7CF0F931F9381E0A5
:10A1800000914B1310914C1320914D1330914E13AD
:10A1900040914713509148136091491370914A13AD
:10A1A000041715072607370708F480E01F910F9161
:10A1B00008954F925F926F927F928F929F92AF928B
:10A1C000BF92CF92DF92EF92FF920F931F93CF93A4
:10A1D00010929C0410929B042FE320939A041092F7
:10A1E0009904109298041092970410924A041092C5
:10A1F0004B0410924C0410924D049C01F901908183
:10A200002F5F3F4F9032D1F39E34C9F4818190ED9E
:10A21000980F9A3020F08D3211F08B3281F4329603
:10A220009F012F5F3F4F808180538A3008F47EC0AA
:10A230009F012F5F3F4F8081803209F479C0F093F6
:10A24000B506E093B4068F010F5F1F4FC0816AE22D
:10A2500070E0C8010F942337009731F0FC0131976B
:10A2600080818032E1F31182CD3429F0C43519F0B8
:10A27000C73409F04BC0F80180810F5F1F4F803257
:10A28000D1F380538A3008F041C0C0939A0490E023
:10A2900080E04AE0DF011196489F9001499F300D10
:10A2A0001124C901C0972081820F911D27FD9A9525
:10A2B000218130ED320F3A30E8F190939904809388
:10A2C00098042E3261F4329630E04AE0DF01319694
:10A2D0002C9150ED520F5A3078F1309397049D0134
:10A2E000D9012F5F3F4F4C914032D1F3CD34A1F5CE
:10A2F0008E31910539F030F58731910519F08C31A7
:10A30000910551F5B0939C04A0939B04CF911F91AC
:10A310000F91FF90EF90DF90CF90BF90AF909F9004
:10A320008F907F906F905F904F900895F90178CF54
:10A33000F9017ECFFD01AECF349F200D112430ED09
:10A34000320FC4CF8537910538F087379105D0F2A9
:10A35000803A23E09207B1F25091B40670E060E0D9
:10A36000C12CD12C7601C394FD0131964C9144232C
:10A3700009F492C04132A1F4CD3491F480329105B8
:10A3800079F4F0939C04E0939B0463E270E0CF01C6
:10A390000F942337009709F4B9CFFC011082B6CF90
:10A3A00041544A3108F073C0DF012D91203209F485
:10A3B00059C030ED320F3A3008F465C02E3209F042
:10A3C00053C0218120532A3008F45DC030E020E0E2
:10A3D0006115710519F4BF0161507109A42FB0E036
:10A3E0002601370104C0440C551C661C771C4A9595
:10A3F000D2F780904A0490904B04A0904C04B09007
:10A400004D0484289528A628B72880924A04909263
:10A410004B04A0924C04B0924D0421153105A9F1D2
:10A42000251BA05DBB4F2C9320812154DF012A31D5
:10A4300008F49ACFDF012191222309F495CF30ED62
:10A44000320F3A30B8F333ED320F323098F32B320B
:10A4500089F39D012F5F3F4F4C91403209F084CF2B
:10A46000D901F7CFFD01A0CF2D3219F02B3209F021
:10A47000ADCF218130ED320F3A3028F02E3209F085
:10A48000A5CF22819FCF9F01A9CF20E0CACF611520
:10A49000710551F6BD01C8CF70939C0460939B0475
:10A4A00035CFCF93DF93EC018991882319F00E9477
:10A4B00089F7FACF8DE00E9489F78AE0DF91CF918A
:10A4C0000C9489F7EF92FF920F931F93CF93DF9332
:10A4D000CDB7DEB762970FB6F894DEBF0FBECDBF23
:10A4E0000E94FB29882309F43FC046E054E082FF24
:10A4F00002C04BEF53E026E034E081FF02C02DEFB5
:10A5000033E080FD2EC086E094E05F934F933F934D
:10A510002F939F938F9388EE9EE09F938F938E014E
:10A520000F5F1F4F1F930F930F949C2C0F94A10B41
:10A53000C8010E945152C8010E9475AF0FB6F8942D
:10A54000DEBF0FBECDBF81E062960FB6F894DEBFCE
:10A550000FBECDBFDF91CF911F910F91FF90EF9074
:10A5600008958FEF93E0D1CF80E0EECFAF92BF920E
:10A57000CF92DF92EF92FF920F931F93CF93DF93CF
:10A58000CDB7DEB7E6970FB6F894DEBF0FBECDBFEE
:10A5900000919B0410919C04F80101900020E9F7C0
:10A5A00031976F01C01AD10AF801CF01801B910BBE
:10A5B0008C159D053CF481918F32B9F7DF0111971D
:10A5C0001C92F3CF8BE1EFE6F3E1DE015C960190A4
:10A5D0000D928A95E1F7F12CE12CEC14FD040CF0BE
:10A5E0005DC0F801EE0DFF1D8081811103C08FEF6A
:10A5F000E81AF80A5801AE0CBF1CF50180818823C7
:10A6000009F44CC0FFEFEF1AFF0AF801EE0DFF1D31
:10A610007F01E01AF10A81918111FACFCE014C96A7
:10A620000E94777E8BE1FE017C96DE0111960190FF
:10A630000D928A95E1F7B501CE0101960E948576CB
:10A64000CE0101960E94D1EF8FE20E9489F780919E
:10A65000BD1081113BC081E094E00E94E4798091BB
:10A660004F1384FF1BC019821C8221E0A501BE018B
:10A67000645E7F4FCE0101960E94B980811129C08E
:10A680008AE00E9489F70F94A10BB5018DEC9CE044
:10A690000F94930BCE0101960E94D1EF8AE00E94A5
:10A6A00089F7CE014C960E94D1EFE6960FB6F8944A
:10A6B000DEBF0FBECDBFDF91CF911F910F91FF90F5
:10A6C000EF90DF90CF90BF90AF9008958DEB90E129
:10A6D000C4CFCE014C960E94E67D8BE1FE013196FF
:10A6E000DE015C9601900D928A95E1F7CE0101960C
:10A6F0000E94D1EF72CF3F924F925F926F927F9202
:10A700008F929F92AF92BF92CF92DF92EF92FF9281
:10A710000F931F93CF93DF9380914C0487FD38C034
:10A7200080914D048370A1F5C091A211D091A31125
:10A73000488159816A817B818EEB9CE00E94E2F91D
:10A740004C815D816E817F8182ED94E20E94E2F90D
:10A7500040919E1150919F116091A0117091A11193
:10A760008FEC94E20E94E2F98AE0DF91CF911F9191
:10A770000F91FF90EF90DF90CF90BF90AF909F90A0
:10A780008F907F906F905F904F903F900C9489F7DF
:10A7900060909611709097118090981190909911F7
:10A7A000A0909A11B0909B1100919C1110919D1155
:10A7B000C0909E11D0909F11E090A011F090A11137
:10A7C00088E50E947EEEC82F882309F49AC00E9473
:10A7D00006EE362E472E582ED92F20E030E044EBDF
:10A7E00053EC0F94353687FD0DC020E030E044EB8C
:10A7F00053E4632D742D852D9D2F0F94052D181670
:10A800000CF081C068E671E08BEA9CE00E9404FADB
:10A8100068E671E086EA9CE00E9404FA83EA9CE024
:10A820000E94B1F7C0E089E50E947EEE882361F1C5
:10A830000E9406EE362E472E582ED92F20E030E00B
:10A8400044EB53EC0F94353687FD0DC020E030E02B
:10A8500044EB53E4632D742D852D9D2F0F94052D0E
:10A8600018160CF055C068E671E080E99CE00E9483
:10A8700004FA68E671E08BE89CE00E9404FA88E83C
:10A880009CE00E94B1F7C0E08AE50E947EEE88233A
:10A8900009F443C00E9406EE6B017C0120E030E029
:10A8A00040E151EC0F94353687FD0AC020E030E0DE
:10A8B00040E151E4C701B6010F94052D18166CF55F
:10A8C00067EF7FEF86E79CE00E9404FA69E070E0A2
:10A8D00081E79CE00E9404FA8EE69CE0DF91CF9134
:10A8E0001F910F91FF90EF90DF90CF90BF90AF90AE
:10A8F0009F908F907F906F905F904F903F900C94BF
:10A90000B1F7C1E090CF632C742C852C9D2E8BCF9A
:10A91000A32CB42C052D1D2FB7CFCC23E1F0C30100
:10A92000D4018093961190939711A0939811B093AE
:10A930009911C501D80180939A1190939B11A0930E
:10A940009C11B0939D11C0929E11D0929F11E092E4
:10A95000A011F092A111DF91CF911F910F91FF9063
:10A96000EF90DF90CF90BF90AF909F908F907F90AF
:10A970006F905F904F903F900895CF92DF92EF924B
:10A98000FF928AE50E947EEE882309F45AC00E9455
:10A9900006EE20E030E040E050EC0F94052DC12C95
:10A9A000D12CE12C90ECF92E87FD0FC00E9406EE11
:10A9B00020E030E040E050E40F94353618160CF4F7
:10A9C00062C00E9406EE6B017C012091780B3091F1
:10A9D000790B40917A0B50917B0BC701B6010F9414
:10A9E0006B2D0F944135CB010E94C4C880E50E94B5
:10A9F00030EE81114EC0A701960160919E117091B9
:10AA00009F118091A0119091A1110F94D533609363
:10AA10009E1170939F118093A0119093A1110F9498
:10AA2000A10B40919E1150919F116091A0117091C6
:10AA3000A1118FE59CE00E94E2F98AE00E9489F76B
:10AA400005C083E50E947EEE8111A1CF80914C0468
:10AA500087FD24C080914D04837001F50F94A10BF4
:10AA600040919E1150919F116091A0117091A11180
:10AA700080E59CE00E94E2F98AE0FF90EF90DF9091
:10AA8000CF900C9489F7C12CD12CE12C80E4F82EC6
:10AA90009CCF0E94F2ED8111AECFD8CF82E50E940B
:10AAA00030EE8111DBCFFF90EF90DF90CF900895D3
:10AAB0004F925F926F927F928F929F92AF92BF92CE
:10AAC000CF92DF92EF92FF92CF93DF93CDB7DEB7B5
:10AAD0002C970FB6F894DEBF0FBECDBF4090FE0797
:10AAE0005090FF076090000870900108209130029C
:10AAF000309131024091320250913302C301B201D0
:10AB00000F94D53369837A838B839C83809002086A
:10AB100090900308A0900408B0900508209134029A
:10AB2000309135024091360250913702C501B4018F
:10AB30000F94D5336D837E838F839887C0900608EA
:10AB4000D0900708E0900808F0900908209138029A
:10AB50003091390240913A0250913B02C701B6014F
:10AB60000F94D53369877A878B879C8720913C0225
:10AB700030913D0240913E0250913F02C301B2012B
:10AB80000F94D5332B013C012091400230914102BA
:10AB90004091420250914302C501B4010F94D53354
:10ABA0004B015C01209144023091450240914602E4
:10ABB00050914702C701B6010F94D5336B017C0158
:10ABC0000F94A10B88E894E00E94B1F783E50E94FE
:10ABD00030EE882321F00E94F2ED80932E028091C6
:10ABE0002E02811151C08FE694E00E94B1F780E8F7
:10ABF00094E00E94B1F749815A816B817C8186EB98
:10AC000093E10E94E2F94D815E816F81788582ED4A
:10AC100094E20E94E2F949855A856B857C858FEC28
:10AC200094E20E94E2F98EE794E00E94B1F786E791
:10AC300094E00E94B1F7B301A20186EB93E10E9478
:10AC4000E2F9B501A40182ED94E20E94E2F9B701B4
:10AC5000A6018FEC94E20E94E2F98AE02C960FB6EE
:10AC6000F894DEBF0FBECDBFDF91CF91FF90EF9084
:10AC7000DF90CF90BF90AF909F908F907F906F901C
:10AC80005F904F900C9489F783E794E0AECF2F92BA
:10AC90003F924F925F926F927F928F929F92AF926C
:10ACA000BF92CF92DF92EF92FF920F931F93CF93B9
:10ACB000DF93CDB7DEB7E5970FB6F894DEBF0FBED2
:10ACC000CDBF8DAB20912F042CAB21E020932F041E
:10ACD00080919A048D3409F4CBC4843511F40C941A
:10ACE000726A873409F091C1809198049091990417
:10ACF0008B31910509F430C208F079C18430910597
:10AD000008F030C1209117068230910508F4E1C1A6
:10AD1000213009F0E4C111E0029709F010E00E942F
:10AD2000A11F19821A821B821C821D821E821F8211
:10AD3000188682E50E947EEE882309F4E3C10E9412
:10AD400006EE6B017C0120E030E0A9010F94052D97
:10AD5000882309F4EAC040904A0250904B02609068
:10AD60004C0270904D0280914E0290914F02A09142
:10AD70005002B09151028CA79DA7AEA7BFA78090AB
:10AD8000A2069090A306A090A406B090A50680917C
:10AD9000A6069091A706A091A806B091A90688AB37
:10ADA00099ABAAABBBABA5019401C301B2010F944F
:10ADB000052D81110DC028A939A94AA95BA96CA547
:10ADC0007DA58EA59FA50F94052D882309F4ADC000
:10ADD000A3019201C501B4010F94D43320E030E007
:10ADE00040E05FE30F946B2D68A779A78AA79BA724
:10ADF0002CA53DA54EA55FA568A979A98AA99BA9FF
:10AE00000F94D43320E030E040E05FE30F946B2DEB
:10AE10002B013C0120E030E0A901C701B6010F94ED
:10AE2000052D881F8827881F181709F462C180E044
:10AE300090E0A0E8BFEB8CA79DA7AEA7BFA728A571
:10AE400039A54AA55BA5CA01B9010F946B2D4B0129
:10AE50005C01A3019201C301B2010F946B2D9B0110
:10AE6000AC01C501B4010F94D5330F9483364B0167
:10AE70005C01AC019B01C701B6010F94D43368ABF0
:10AE800079AB8AAB9BABA5019401C701B6010F94C6
:10AE9000D5339B01AC0168A979A98AA99BA90F9414
:10AEA0006B2D6B017C0120E030E0A9010F94353659
:10AEB00087FD24C1C701B6010F9483366B017C0165
:10AEC000C301B2019058A50194010F94CF342CA571
:10AED0003DA54EA55FA50F946B2DA70196010F947C
:10AEE0006B2D28A539A54AA55BA50F94D533698399
:10AEF0007A838B839C83A501940168A579A58AA593
:10AF00009BA50F94CF342CA53DA54EA55FA50F940E
:10AF10006B2DA70196010F946B2DA30192010F9445
:10AF2000D5336D837E838F83988720E030E0A9013D
:10AF300069817A818B819C810F94052D8111F6C0E6
:10AF400020E030E0A9016D817E818F8198850F948A
:10AF5000052D8111EBC00F949D0B80E695E00E94BA
:10AF6000B1F7BDC08531910509F4B9C08A319105A9
:10AF700009F4EFC0049709F048C080E50E947EEE16
:10AF8000C12CD12C7601882321F00E9483E86B012B
:10AF90007C0183E50E947EEE882361F00E9406EE2C
:10AFA00020E030E04AE754E40F946B2D0F944835CD
:10AFB0006B017C010E94A02380914310811105C088
:10AFC00060E086E795E00E94693C0E948BC8C60E4F
:10AFD000D71EE81EF91E0E948BC86C197D098E09C8
:10AFE0009F0997FF7CC080E00F944C0FF4CF823212
:10AFF000910509F401C260F48D31910509F429C16C
:10B0000008F4C3C04E9709F47CC10E9476C467C09F
:10B010008A35910509F4B5C208F58A97B1F7809190
:10B020001706813009F05BC089E40E947EEE082F8C
:10B03000F12C882319F00E9402EEF82E8AE40E9477
:10B040007EEEE82E882309F4DAC10E9402EE182F62
:10B050000111D8C1153008F4DFC1D7C18B35910576
:10B0600009F492C28C35910581F68091970488236A
:10B0700009F48EC2893099F562EEA62E62E0B62EF2
:10B080007AE4C72E72E0D72EE12C00E010E0D50163
:10B090008D915D010E947EEEF82E882361F01330C1
:10B0A00011F4082FFE2C0E9406EEF60160837183D6
:10B0B00082839383EF2C1F5FF4E0CF0ED11C1430FA
:10B0C00031F7EE2009F4B6C20E945C310E9487314C
:10B0D00006C0213021F40E94A11F0E94C92A3DA967
:10B0E000311102C00E9496DF8CA980932F040C942A
:10B0F000316380E090E0A0E8BFE39DCEC12CD12C6D
:10B100007601DECE89E40E947EEE882331F00E9433
:10B1100006EE69837A838B839C838AE40E947EEEA9
:10B12000882309F402CF0E9406EEFBCE412FBE0118
:10B130006F5F7F4F82EA96E00E94E9DF0E948BC832
:10B14000609394107093951080939610909397103D
:10B15000C6CF0F946403C3CF87E00E94625281116F
:10B16000BECF8CE0E6EDF2E0DE01119601900D928B
:10B170008A95E1F770E060E080E50E94931FBE01D0
:10B180006F5F7F4F0E94B335AACF87E00E94FB29F3
:10B19000811106C060E08FE40E941DEF81119FCFF6
:10B1A0000E94A02310922F026091570B8CE40E9402
:10B1B0001DEFE82E80E00E94C4F10E948BC86093CE
:10B1C00094107093951080939610909397100E940E
:10B1D000952D81E08093D3050E94F0328AE50E948C
:10B1E00030EEF82E882369F081E00E94FB29182FA9
:10B1F00082E00E94FB2911110C94E06B11E0811197
:10B2000001C010E088E50E9430EE81110C94876A3D
:10B21000112311F40C948A6A012F10E00C94976AA0
:10B2200060E070E080E890E40C94A06AA3019201D1
:10B23000C501B4010C94ED6A60E081E995E00E94DB
:10B24000693C0F94A10B8FE795E00E94B1F70C9435
:10B25000C96B14E00E948BC8609394107093951092
:10B2600080939610909397108091570B811127C06F
:10B270008EE40E9430EE882321F082EA95E00E945D
:10B28000126C87E00E94625281111FC00F947816E1
:10B290008823D9F0115001F130E020E043E15EE075
:10B2A0006DEC75E085E00E9419F961E080EC95E0B5
:10B2B0000E94C0F888EA95E00E94126CCBCF60E053
:10B2C0008FE40E941DEF882399F20E94F1F88BE62B
:10B2D00096E00E94126C03CF61E08EE596E00E943A
:10B2E000C0F889EE95E00E94126C61E08EEF9DE05F
:10B2F0000E94C0F840E070E060E08AED95E00F94B5
:10B300007B0E0091A2111091A311D8012D913D91B6
:10B310004D915C9160914A0270914B0280914C0278
:10B3200090914D020F94D533AB01BC0188E50E948A
:10B33000EBEE69837A838B839C83F80124813581CA
:10B340004681578160914E0270914F028091500268
:10B35000909151020F94D533AB01BC0189E50E9455
:10B36000EBEE6D837E838F839887BE016B5F7F4F8B
:10B37000CE0101960E94BCE8882309F4B0CE80E09B
:10B380000E94C4F10E94952D61E085E40E941DEFAA
:10B39000182F01E021E0482FBE016B5F7F4FCE01E7
:10B3A00001960E94B3C46B017C01AC019B010F9418
:10B3B000C736811119C049815A816B817C818DE822
:10B3C00096E00E94E2F94D815E816F81788588E880
:10B3D00096E00E94E2F9B701A60183E896E00E9498
:10B3E000E2F98AE00E9489F70E947C2D11110E94E7
:10B3F000A2E80E94873173CE0E94CBFE70CE10E08F
:10B40000002351F0F4E0FF1528F485E996E00E944E
:10B41000B1F765CEE1101ECE80E1EAE4F2E0A2EAE7
:10B42000B6E001900D928A95E1F7002319F16F2D96
:10B43000FF0C770B880B990B0F940C2D20910105B5
:10B440003091020540910305509104050F946B2D36
:10B450002091F9043091FA044091FB045091FC04CE
:10B460000F94D5336093A2067093A3068093A4062D
:10B470009093A506EE2019F1612F110F770B880B21
:10B48000990B0F940C2D20910505309106054091E4
:10B490000705509108050F946B2D2091FD04309104
:10B4A000FE044091FF04509100050F94D533609342
:10B4B000A6067093A7068093A8069093A90660E05D
:10B4C00080E50E941DEF8823C1F10023D1F0E091B7
:10B4D000A211F091A31120813181428153816091A9
:10B4E000A2067091A3068091A4069091A5060F94E0
:10B4F000D4336093A2067093A3068093A40690931E
:10B50000A506EE20D1F0E091A211F091A3112481C3
:10B510003581468157816091A6067091A70680917A
:10B52000A8069091A9060F94D4336093A606709351
:10B53000A7068093A8069093A90640E050E0BA01C0
:10B5400086E40E94EBEE6B017C0120E030E0A90173
:10B550000F94353618168CF420E030E040E752E4C2
:10B56000C701B6010F94CF3469837A838B839C83A0
:10B57000CE0101960E94B42DB2CD60E070E0CB0107
:10B58000F3CF10922207ABCD8FE080932207A7CD97
:10B5900052EEC52E52E0D52EF12CE12C00E010E049
:10B5A000D6018D916D010E947EEE382E8823D9F14F
:10B5B0000E9406EE4B015C01133059F0F701E25096
:10B5C000F84F20813181428153810F94D4334B0154
:10B5D0005C01F701E65BFD4F20813181428153819F
:10B5E000C501B4010F94D4332B013C012DEB37E39B
:10B5F00046E855EB0F94353687FD0AC02DEB37E34F
:10B6000046E855E3C301B2010F94052D18165CF40A
:10B610001330C1F48092560290925702A0925802C1
:10B62000B0925902032D1F5FB4E0EB0EF11C1430F1
:10B6300009F0B6CF002309F449CD86E592E00E94D7
:10B64000712744CDF701E85DF84F5F01A301920136
:10B6500060817181828193810F94D533D5016D937F
:10B660007D938D939C931397812F0E94D41CDBCFE5
:10B6700080919804909199048937910511F40C9464
:10B68000326508F0B7C18D34910509F4F7C608F0AA
:10B69000CEC08A31910509F42CC608F071C08431FE
:10B6A000910509F472C508F04EC08131910509F485
:10B6B00031C508F042C0029708F0A7CC80E50E948F
:10B6C0007EEEC12CD12C7601882321F00E9483E8E4
:10B6D0006B017C0183E50E947EEE882361F00E946D
:10B6E00006EE20E030E04AE754E40F946B2D0F940F
:10B6F00048356B017C010E94A02380919B049091AE
:10B700009C04892B09F401C50E9484C4809198048B
:10B710009091990466EB76E0892B11F46EEA76E05D
:10B7200030E020E04EEB56E082E00E9419F940E064
:10B73000C701B6010F94911ED2CC429709F065CC97
:10B740000E948BEECCCC8731910509F453C570F47F
:10B750008531910509F44AC5469709F056CC809188
:10B760004F1382FDBCCC0E94007EB9CC883191057C
:10B7700009F455C5499709F048CC0E94FE21AFCC89
:10B780008032910509F439C6C0F58D31910509F46F
:10B790001DC670F48B31910509F4BEC54C9709F0B4
:10B7A00034CC80919B0490919C040E94F28297CCAF
:10B7B0008E31910509F411C64F9709F026CC0E94ED
:10B7C00066356C8F7D8F8E8F9F8FBE016F5F7F4F31
:10B7D000CE014C960E942C1ECE0101960E9475AFA0
:10B7E0000F94A10BBE016F5F7F4F82E397E00F9430
:10B7F000930B8AE00E9489F772CC8934910509F491
:10B8000029C650F48132910509F420C6C09709F089
:10B81000FCCB0E940EFA63CC8B34910509F42AC646
:10B820008C34910509F0F1CB0E94103958CC8C363C
:10B83000910509F454CC08F072C08535910511F4D6
:10B840000C941F6490F58235910509F4E8C720F542
:10B850008E34910509F416C68135910509F0D5CBD2
:10B860000E949A890E94B1230E94EEF30E94F1F394
:10B870001092BD061092BC061092BB0668EE73E0F3
:10B8800080E090E00E94E1F20E94F6F360E08DEF2C
:10B8900097E00E94693C23CC8335910509F4C7C722
:10B8A0008435910509F44CCFB0CB8936910509F464
:10B8B000C6C600F58C35910509F4E6C788369105B2
:10B8C00009F0A3CB8091140B83FD09CC0E94CE20FC
:10B8D00087FD05CC83E50E947EEE882341F00E941F
:10B8E00002EE0E94702361E080E00F9425210F9406
:10B8F0008420F5CB8A36910509F4CCC68B369105A8
:10B9000009F083CB60E080E50E9411EF823008F0FF
:10B91000E6CBE82FF0E0E15DF74F1082E0CB823715
:10B92000910511F40C94E564A0F58F36910509F4A6
:10B93000DAC6C8F48D36910509F436C68E369105FF
:10B9400009F063CB8EE40E947EEE882309F4C7CB16
:10B950000E94CEED6093440C7093450C8093460C8E
:10B960009093470CBCCB8037910509F4B8CB813755
:10B97000910509F04ACB83E50E947EEE882309F405
:10B98000F9C60E94DEED8D3308F0EFC68093000209
:10B99000A6CB8637910511F40C94F564D0F4833767
:10B9A000910511F40C94ED648537910509F02DCBC8
:10B9B00080919B0490919C04009711F40C94F16485
:10B9C000DC012C91222311F40C94F1640E9475AFD8
:10B9D00086CB8737910511F40C942E658837910535
:10B9E00009F013CB81E08093D3058093D2050E94A8
:10B9F000F03275CB8239E1E09E0711F40C94856832
:10BA000008F078C1833D910511F40C94126608F09A
:10BA1000C4C0883C910511F40C943A65D0F58C387B
:10BA2000910509F4B4C628F48D37910509F4A5CE23
:10BA3000ECCA8B39910509F4CBC68E3B910509F010
:10BA4000E4CA8091140B83FD4ACB83E50E947EEE0D
:10BA5000182F882309F4B2C60E9402EE0E9482EDDC
:10BA600060E081E00F9425212091A0103091A11079
:10BA700080919E1090919F10821793070CF4A5C699
:10BA80008FED97E060E00E94693C812F0E943E8626
:10BA900026CB8C3C910511F40C94956548F5893CB6
:10BAA000910511F40C946B658B3C910509F0ADCABE
:10BAB0000E94CE2087FD13CB12EEE12E12E0F12E74
:10BAC00010E000E0D7018D917D010E9430EE8823C7
:10BAD00049F00E9406EEF801E45AF44F64A375A3FE
:10BAE00086A397A30C5F1F4F0031110559F7F7CAC2
:10BAF0008D3C910511F40C940E66B4E3EB2EB7E087
:10BB0000FB2E10E08E3C910509F07FCA88E5810F7D
:10BB10000E9430EE882351F00E9406EEF701608308
:10BB2000718382839383812F0E94D41C1F5FF4E072
:10BB3000EF0EF11C133051F780914C0487FDC6CAFB
:10BB400080914D04837009F0C1CA4091340750912F
:10BB50003507609136077091370785E298E00E94BB
:10BB6000E2F9409138075091390760913A07709196
:10BB70003B0782ED94E20E94E2F940913C0750912C
:10BB80003D0760913E0770913F078FEC94E20E9461
:10BB9000E2F98AE00E9489F7A2CA8D3221E0920779
:10BBA00011F40C94136708F06CC08831A1E09A0777
:10BBB00011F40C94736608F045C08C3D910511F4A6
:10BBC0000C9416668D3D910509F01FCA0E94CE2087
:10BBD000082F87FD84CA83E50E947EEE002E000CAC
:10BBE000110B7801EE0CFF1C882311F40C9459669C
:10BBF0000E9402EEF701E25AFD4F91838083000F0D
:10BC0000111F000F111F9801265A3D4F7901BC01E9
:10BC1000990F880B990B0F940C2D2AE037ED43E216
:10BC20005CE30F946B2D085A144FD8012D913D9170
:10BC30004D915C910F946B2DF7016083718382832A
:10BC400093834DCA8232E1E09E0711F40C940F6792
:10BC50008C32914009F0D9C964E071E083E50E941B
:10BC6000931F8C0168EE73E080E50E94931F893872
:10BC700023E1920710F088E893E1B8010E94D739D8
:10BC80002ECA803321E0920711F40C94956700F5D9
:10BC90008E32A1E09A0711F40C9409688F3291401A
:10BCA00009F0B3C970E060E085E40E9402EFF82E6D
:10BCB0003FEF831711F40C947E68882311F40C94E1
:10BCC0004F688FEB98E00E94B1F70E943BAE07CA25
:10BCD0008039E1E09E0711F40C948168813991402C
:10BCE00009F093C98091B2068111F0C981E00E94E8
:10BCF000FF32ECC9883F31E0930711F40C9483695B
:10BD000008F0E2C0863AB1E09B0711F40C943A6A5D
:10BD100008F0B3C08D39F1E09F0711F40C944E6A1E
:10BD200078F58A3931E0930709F4D9C98C39914003
:10BD300009F06BC980914A04887811F00C948D68E1
:10BD400080914C04867011F00C948D680F94A10BB7
:10BD500083E099E00E94B1F780910F020E94C4F93C
:10BD600040910B0250910C0260910D0270910E02F5
:10BD700083EE98E00E94E2F98AE00E9489F7AFC959
:10BD8000843AB1E09B0711F40C94BD68853A914068
:10BD900009F03BC96FEF7FEF89E40E9402EF082FA3
:10BDA0006FEF7FEF8AE40E9402EF182F8AE50E946E
:10BDB0007EEED12C811108C081E50E947EEED82E46
:10BDC000882311F40C94D86BC02E81E0800F86304C
:10BDD00010F00C94C468912E81E0810F863010F031
:10BDE0000C94C4680E9406EE2B013C01F02E07FD66
:10BDF000F12C07FF02C004E0C02E812E17FD812C1C
:10BE000017FF02C014E0912EB5E03B2ECF1408F4CA
:10BE100066C9E82C3F9C500111249E1410F40C9428
:10BE2000C1680E2D10E020E030E0A901DD2069F0AE
:10BE3000F501E00FF11FEE0FFF1FEE0FFF1FE254A1
:10BE4000F94F20813181428153810A0D1B1D000F62
:10BE5000111F000F111F0254194FC301B2010F949B
:10BE6000D533D8016D937D938D939C9313976E2D4D
:10BE70008F2D0E9417C3E394D0CF853FF1E09F0739
:10BE800011F40C947B6968F48C3A31E0930711F457
:10BE90000C94CC68843F914009F0B7C80E94B33C31
:10BEA0001EC9863FB1E09B0711F40C947F69873F60
:10BEB000914009F0AAC861E083E50E941DEF91E07E
:10BEC00089270E94B2A30BC98335F3E09F0711F4C1
:10BED0000C94366A08F0CBC08B3532E0930711F42E
:10BEE0000C94A66968F48C30B2E09B0711F40C94B2
:10BEF00095698835924009F088C80E94F320EFC800
:10BF00008D3BF2E09F0711F40C94266A8E3B924021
:10BF100009F07BC80E94CE20182F87FDE0C88AE573
:10BF20000E947EEE812C912C90E2A92E91E4B92EF4
:10BF3000882379F040E050E0BA018AE50E94EBEEF8
:10BF40004B015C0120E030E0A9010F943536181652
:10BF50007CF580E090E0A0EAB0E489839A83AB832B
:10BF6000BC8320915202309153024091540250916F
:10BF70005502C501B4010F94D5336B017C0120E05B
:10BF800030E048EC53E40F94052D87FD06C0C12C2A
:10BF9000D12C88ECE82E83E4F82ECC8EDD8EEE8E4C
:10BFA000FF8EBE016F5F7F4FCE014C960E943130F5
:10BFB00085E50E9430EE882311F40C942A6A0E94D1
:10BFC00006EE6B017C0120E030E0A901C701B6015B
:10BFD0000F94353687FF04C0F7FAF094F7F8F09421
:10BFE000F7FAF094F7F8F094C982DA82EB82FC82D7
:10BFF00080E00F94571C882321F0CE0101960E9407
:10C0000005F320E030E0A901C501B4010F943536F5
:10C0100018160CF064C880E090E0A0EAB0E48983D0
:10C020009A83AB83BC83A501940160915202709105
:10C03000530280915402909155020F94D4336B01B6
:10C040007C0120E030E0A9010F94353618161CF071
:10C05000C12CD12C7601CC8EDD8EEE8EFF8EBE01F2
:10C060006F5F7F4FCE014C960E94313038C8873EBB
:10C0700033E0930711F40C943E6AB8F48C36B3E0C5
:10C080009B0709F42CC8803A934011F00C94055892
:10C0900020919B0430919C0490914F139260909357
:10C0A0004F13C9010E94F2821AC8883EF3E09F072D
:10C0B00011F40C94676A893E934011F00C94055872
:10C0C0008091451381110C946B6A0E94A9EF0E9424
:10C0D000E7820E9466356D3371058105910520F078
:10C0E00085EC99E00E94126C81EC99E00E94126C40
:10C0F00084EE8093A7048DEA99E00E94B1F789EA63
:10C1000099E00E94126C0C946F5887EC96E00E94A4
:10C11000B136FCCA80914A0484FD18C080914C0459
:10C1200087FD14C080914D04837081F460E08AED36
:10C1300096E00E94693C5F988A988091080181701E
:10C1400080930601479812980C946F5888E50E94D6
:10C1500030EE81115F9889E50E9430EE81118A9856
:10C160008AE50E9430EE882331F0809108018170C9
:10C1700080930601479885E40E9430EE882311F4ED
:10C180000C946F5812980C946F5880914F1383FF42
:10C1900025C082EF96E00E94B1F780914F1383FF94
:10C1A00017C08FE693E10E94777E8BE1EFE6F3E123
:10C1B000DE01119601900D928A95E1F770E060E042
:10C1C000CE0101960E942E84CE0101960E94D1EFED
:10C1D00083EE96E00E94B1F70C946F580F94A10B78
:10C1E00083E097E00E94B1F70C946F580E94117E93
:10C1F0000C946F5880919B0490919C04FC012191B8
:10C20000222331F02032D9F7DF0111971C92F7CFAA
:10C2100060E00E943B831092A7040C946F5883E562
:10C220000E947EEE882321F00E94CEED0E9477507E
:10C2300084E50E947EEE8823A9F00E94CEED6B017A
:10C240007C010E949835C092CA04D092CB04E0923F
:10C25000CC04F092CD04CD28CE28CF2819F081E06F
:10C2600080934210809141108823F9F080E090E0A3
:10C27000A0EAB1E489839A83AB83BC831C8E1D8EB4
:10C280001E8E1F8E18A219A21AA21BA210E000E097
:10C2900020E0AE014F5F5F4FBE01645E7F4FCE0175
:10C2A00080960F94B81C0C946F580E94E0F388237A
:10C2B00081F00E94EE750E9463388EE797E00E943D
:10C2C0009F7D1092AB0C1092AC0C1092AD0C1092A2
:10C2D000AE0C61E086E29EE00E94C0F843E15EE0C1
:10C2E0006DE077E085E00E9432AE0E94ADAF0C9425
:10C2F0006F5880914F1383FD02C00C946F5883E5F3
:10C300000E947EEE882311F40C946F580E94CEEDAB
:10C310000E9477500C946F5883E40E9430EE88237B
:10C3200061F183E297E00E94B1F78091B61488230F
:10C33000F9F0BE016F5F7F4F83EB94E10E94327D85
:10C34000CE0101960E94E479CE0101960E94BD7E45
:10C350008091BD10882339F080E20E9489F78DEB2F
:10C3600090E10E94E4798AE00E9489F70C946F586A
:10C3700089E197E00E94B1F7F6CF83E50E947EEE57
:10C38000882301F10E94DEED182F8C3308F08CE336
:10C39000809324040E948BC86B017C01212F30E024
:10C3A000A8EEB3E00F949D33C60ED71EE81EF91E0B
:10C3B000C0922004D0922104E0922204F09223043F
:10C3C0000C946F580E94AC750C946F5880914F1369
:10C3D0008E7F80934F130C946F5880914F1383FD81
:10C3E00002C00C946F580E945CC480919B04909191
:10C3F0009C040E947F820C946F5880914F1382FDA1
:10C400000E94A02380914F1383FD02C00C946F58AB
:10C4100060E080E50E941DEF182F682F80919B043B
:10C4200090919C040E943B8383E50E947EEE8823CA
:10C4300021F00E94CEED0E9477500E94EE751111FE
:10C440000C946F580E9463380C946F580E94B65237
:10C450000C946F5880E50E9430EE882311F40C9400
:10C460006F580E94DEED853608F084E68093A704BD
:10C470000C946F580E9463380C946F580E94EEF32E
:10C480000C946F5870E060E083E50E9402EF8E34F8
:10C49000910531F40E940F230E94ADAF0C946F58A8
:10C4A0008DE997E00E94B1F76091C2057091C305D4
:10C4B00084E997E00E94D0F96091C4057091C505A8
:10C4C00087E897E00E94D0F96091C2057091C3059A
:10C4D0008091C4059091C505681B790B809142102D
:10C4E000815021E030E0823010F030E020E0621B2B
:10C4F000730B8CE797E00E94D0F98AE00E9489F7DD
:10C5000084E797E00E94B1F78091C6059091C70536
:10C51000A091C805B091C9058C8F9D8FAE8FBF8F3C
:10C52000BE016F5F7F4FCE014C960E942C1EBE0154
:10C530006F5F7F4F87E697E00F94930B8091CA055A
:10C540009091CB05A091CC05B091CD058C8F9D8F9E
:10C55000AE8FBF8FBE016F5F7F4FCE014C960E94A2
:10C560002C1EBE016F5F7F4F87E597E00F94930B02
:10C5700020E030E04AE754E46091CE057091CF05A9
:10C580008091D0059091D1050F94CF34AB01BC01BF
:10C590008FE397E00E94E2F98DE60E9489F78AE036
:10C5A0000E9489F70C946F588091140B83FF02C08E
:10C5B0000C946F580E94CE20082F87FF02C00C9465
:10C5C0006F5883E50E947EEE182F882359F10E9450
:10C5D00002EE0E94702361E081E00F9425212091FA
:10C5E0000B1130910C118091091190910A11821751
:10C5F0009307F4F480EB97E09F938F938BEB97E096
:10C600009F938F931F920E9442C40F9484200F9097
:10C610000F900F900F900F90612F802F0E94B58781
:10C620000C946F5882E50E947EEE8111D0CF5FC9D5
:10C6300085EA97E0112301F30F948420EDCF0E9447
:10C64000CE20182F87FD0AC080EC97E00E94B1F73A
:10C65000812F0E94CB858AE00E9489F73CA9309304
:10C660002F04E5960FB6F894DEBF0FBECDBFDF9165
:10C67000CF911F910F91FF90EF90DF90CF90BF90DF
:10C68000AF909F908F907F906F905F904F903F9072
:10C690002F90089560E080E50E9411EFF82E81E070
:10C6A0008F1510F40C946F5881E40E9430EE609165
:10C6B0002F08062F811102C00FEF10E083E50E94C2
:10C6C0007EEE882349F00E94CEED8B016F3F71050D
:10C6D00019F010F00FEF10E0EF2DF0E0E15DF74FF3
:10C6E00000830C946F5883E50E9430EE882331F06C
:10C6F00060E083E50E9411EF8093140B0F94A10B6F
:10C7000081ED97E00E94B1F78091140B882351F1DD
:10C7100010E000E020E08091140B90E0B0E0A0E099
:10C72000002E04C0B695A795979587950A94D2F7E1
:10C7300080FF12C0FF24F394F20E222319F08CE242
:10C740000E9489F7F801EE0FFF1FE953F84F85911A
:10C7500094910E94B1F72F2D0F5F1F4F05301105E7
:10C76000D1F601CE83EC97E005CE8CE380930002F6
:10C770000C946F580F94A10B6091000288ED97E024
:10C780000E94DAF98AE00E9489F70C946F58809130
:10C79000140B83FF02C00C946F5883E50E947EEE59
:10C7A000882311F40C946F580E9402EE0E9482EDCF
:10C7B00061E080E00F9425210C946F5882E50E947F
:10C7C0007EEE811149C90C946F588EEE97E05AC9DC
:10C7D00083E50E947EEE882311F40C946F580E942A
:10C7E000DEED182F8C3308F08CE3809329040E942F
:10C7F0008BC86B017C01212F30E0A8EEB3E00F94D1
:10C800009D33C60ED71EE81EF91EC0922504D09295
:10C810002604E0922704F09228040C946F5880912B
:10C8200022078F7D8061809322070C946F5880913E
:10C8300022078F7E8062809322070C946F5883E5D5
:10C840000E9430EE882311F40C946F580E948BC81C
:10C850006093941070939510809396109093971016
:10C860000E9406EE20E030E04AE754E40F946B2D7E
:10C870000F94483560932A0470932B0480932C0402
:10C8800090932D040C946F580E94CE2087FF02C015
:10C890000C946F5880914A0484FD09C080914C0427
:10C8A00087FD05C080914D04837009F489C022EE94
:10C8B000C22E22E0D22E3CE5E32E3BE0F32E10E028
:10C8C000D6018D916D010E947EEE882309F465C02A
:10C8D000133009F06DC00E9406EE4B015C0120E0B0
:10C8E00030E040EA51E40F94052D87FF4EC0A501CA
:10C8F000940160917C0B70917D0B80917E0B9091E7
:10C900007F0B0F94CF342B013C01AC019B01609154
:10C910001708709118088091190890911A080F94BF
:10C920006B2D6093170870931808809319089093E3
:10C930001A08A301920160918C0B70918D0B80916C
:10C940008E0B90918F0B0F946B2D60938C0B7093CB
:10C950008D0B80938E0B90938F0B609127087091B5
:10C9600028088091290890912A080F940A2DA30184
:10C9700092010F946B2D0F944835609327087093A4
:10C9800028088093290890932A0880927C0B909223
:10C990007D0BA0927E0BB0927F0B1F5FF4E0EF0E39
:10C9A000F11C143009F08CCF0E947C230C946F583A
:10C9B0000E9406EEF701648B758B868B978BEDCF0B
:10C9C00081E00E94E9C30C946F580E947AC189EA01
:10C9D00091E10E9427910C946F580E94591D0C946C
:10C9E0006F580E94ADAF0C946F5800919B0410914A
:10C9F0009C0494E0F12C40E09150F9F0F801808122
:10CA0000282F2B7F213499F421812133B1F48134F3
:10CA100011F1853409F441E098012E5F3F4F8901FF
:10CA20002F5F3F4FF80180818032C9F3E5CF803519
:10CA300021F4818180538A3078F341110F94A10B46
:10CA4000FF2021F08FE098E00E94B1F7C8010E941A
:10CA500051520C946F58FF24F394DECF0E940B1FA9
:10CA60000C946F581092D3051092D2050E94F032A8
:10CA70000C946F580E94CE20182F87FF02C00C9490
:10CA80006F580091270784E40E947EEEF82E8823D9
:10CA9000B1F00E9406EE4B015C0120E030E0A901FC
:10CAA0000F94052D8823A9F024E01202F00111242F
:10CAB000ED5DF84F80829182A282B3820F2D602FAC
:10CAC00083E50E941DEF809327070E94F9230C94B1
:10CAD0006F5880E0F8CF0E94CE2087FF02C00C94F0
:10CAE0006F5802EE12E08CE5E82E8BE0F82E96EE01
:10CAF000C92E92E0D92ED8018D918D010E9430EE81
:10CB0000882359F00E9406EE0F944835F7016083A0
:10CB10007183828393830E94861CF4E0EF0EF11CE4
:10CB2000C016D10641F70C946F5880914B0487FDD5
:10CB30002DC080914C048E7049F54091900B50911E
:10CB4000910B6091920B7091930B85E198E00E949C
:10CB5000E2F94091940B5091950B6091960B709176
:10CB6000970B82E198E00E94E2F94091980B509176
:10CB7000990B60919A0B70919B0B85E494E10E9454
:10CB8000E2F98AE00E9489F70C946F5883E50E94CD
:10CB90007EEE882391F00E9406EE6093900B7093D6
:10CBA000910B8093920B9093930B6093980B7093DF
:10CBB000990B80939A0B90939B0B80E50E947EEEDD
:10CBC000882351F00E9406EE6093900B7093910BB6
:10CBD0008093920B9093930B82E50E947EEE8823C4
:10CBE00051F00E9406EE6093940B7093950B809326
:10CBF000960B9093970B84E50E947EEE882311F4A8
:10CC00000C946F580E9406EE6093980B7093990BEA
:10CC100080939A0B90939B0B0C946F580E94BFF7D4
:10CC20000C946F580E9458550C946F5882E40E94DF
:10CC300030EE882341F080916002909161029093E0
:10CC400002028093010282E50E9430EE882341F0C7
:10CC500080910102909102029093610280936002A0
:10CC600083E50E947EEE882331F00E9402EE9093CD
:10CC700061028093600280914A0490914B04A091DC
:10CC80004C04B0914D04892B8A2B8B2B11F00C9402
:10CC90006F5860916002709161028CE298E00E948E
:10CCA00004FA85E20E9489F78AE00E9489F70C94D1
:10CCB0006F580F94A10B85E40E9489F780E3800FE1
:10CCC0000E9489F7F701E25AFD4F6081718180E38C
:10CCD00098E00E9404FA85E20E9489F78AE00E94A7
:10CCE00089F70C946F5880E50E9430EE882311F488
:10CCF0000C946F580E9402EE8C01892B09F082C0BF
:10CD000083E50E9430EE882391F00E9402EE8F3F6F
:10CD1000980731F483E991E10E94FBF30C946F587A
:10CD2000BC0183E991E10E9469F40C946F580F945F
:10CD3000A10B70E060E08BE398E00E9404FA809120
:10CD4000951158E5C52E52E0D52EC81AD10887FD99
:10CD5000D394CC0CDD1CCC0CDD1C0D2C000CEE088F
:10CD6000FF088091941178E8872E912C881A9108F9
:10CD700087FD9394880C991C880C991C092C000C35
:10CD8000AA08BB088091931190E08F3FC9F1FC0184
:10CD9000EE0FFF1FE80FF91FE65BFE4E81819281C7
:10CDA00033E0880F991F3A95E1F7B0E0A0E044E046
:10CDB000B595A795979587954A95D1F702969C01C9
:10CDC0002F5F3F4F032E000C440B550B28193909D8
:10CDD0004A095B09A4EBB0E00F948A33A7019601DE
:10CDE000281939094A095B090F946B33B90188E3A3
:10CDF00098E00E9404FA8AE00E9489F70C946F5828
:10CE000080E0DDCF0F949D0BB80182E598E00E9491
:10CE100004FA83E498E00E94B1F70C946F580E94E2
:10CE2000BD540C946F5860E085E40E9411EF8111AD
:10CE300074C080E50E9430EE882351F00E9406EE17
:10CE400060930E1170930F11809310119093111134
:10CE500089E40E9430EE882381F00E9406EE2CEADD
:10CE600035EC47E25EE30F946B2D609312117093E3
:10CE70001311809314119093151184E40E9430EEE5
:10CE8000882381F00E9406EE2CEA35EC47E25EE34F
:10CE90000F94CF346093161170931711809318116B
:10CEA000909319110F94A10B40910E1150910F11F5
:10CEB000609110117091111181E698E00E94E2F9E1
:10CEC0002CEA35EC47E25EE3609112117091131188
:10CED00080911411909115110F94CF34AB01BC01C6
:10CEE0008DE598E00E94E2F92CEA35EC47E25EE33A
:10CEF000609116117091171180911811909119116C
:10CF00000F946B2DAB01BC0189E598E00E94E2F91A
:10CF10008AE00E9489F70C946F580F949D0B85E668
:10CF200098E00E94B1F70C946F5880E50E9430EEB3
:10CF3000882351F00E9406EE6093A3107093A41012
:10CF40008093A5109093A61089E40E9430EE882368
:10CF500081F00E9406EE2CEA35EC47E25EE30F9486
:10CF60006B2D6093A7107093A8108093A9109093D5
:10CF7000AA1084E40E9430EE882381F00E9406EE1D
:10CF80002CEA35EC47E25EE30F94CF346093AB10AC
:10CF90007093AC108093AD109093AE100F94A10BD2
:10CFA0004091A3105091A4106091A5107091A6100B
:10CFB0008FE798E00E94E2F92CEA35EC47E25EE365
:10CFC0006091A7107091A8108091A9109091AA105B
:10CFD0000F94CF34AB01BC018BE798E00E94E2F9DB
:10CFE0002CEA35EC47E25EE36091AB107091AC1037
:10CFF0008091AD109091AE100F946B2DAB01BC01E0
:10D0000087E798E00E94E2F98AE00E9489F70C9491
:10D010006F5883E50E9430EE182F882369F00E9434
:10D0200002EE9C01909349028093480291E0232BE9
:10D0300009F090E09093310880E50E9430EE88235B
:10D0400061F02091480230914902232B11F00E9497
:10D05000F2ED809331080C946F5811110C946F58B5
:10D060000F94A10B8FE998E00E94B1F780913108ED
:10D07000882391F087E898E00E94B1F76091480218
:10D08000709149028EE898E00E9404FA8AE898E0DC
:10D090000E94B1F70C946F5883E898E0EDCF04EB51
:10D0A00010E083E50E947EEE882319F00E9402EED4
:10D0B0008C0165E070E083E40E9402EFE82E60E0FE
:10D0C00085E50E941DEFD82E60E082EB98E00E947B
:10D0D000693CB801110F880B990B0F940C2D6983D3
:10D0E0007A838B839C832D2D4E2D6F2DCE0101963F
:10D0F0000E949E9E0E94ADAF0C946F5806E410E013
:10D10000D0CF0E94A0230C946F580E9499E80E94EF
:10D11000A2E80E9487310C946F5888E40E9430EE98
:10D12000882321F00E94F2ED80932E0482E50E9474
:10D1300030EE082F83E50E9430EE182F011102C057
:10D14000882341F00E9495F3112321F00E94F2ED13
:10D1500080930F0284E40E9430EE882311F40C9433
:10D160006F580E9406EE60930B0270930C0280933E
:10D170000D0290930E020C946F580F94A50B0C9413
:10D180006F58F3940C94065F0F949D0B84E399E021
:10D190000E94B1F70C946F5887E00E94625281118F
:10D1A0000C946F587FE1C72E7FE0D72EEAE4F2E0BF
:10D1B000F9A7E8A79E012F5F3F4F1901790110E001
:10D1C00000E0C6010E9493E8A8A5B9A58D909D90A6
:10D1D000AD90BD90B9A7A8A7A50194010F94D43331
:10D1E0002B013C01F701408251826282738220E070
:10D1F00030E040EA51EC0F94353687FD0AC020E05C
:10D2000030E040EA51E4C301B2010F94052D181635
:10D2100084F4F801ED5BF04FE4911E1654F4B7FA74
:10D22000B094B7F8B094D7018D929D92AD92BC9214
:10D230001397F70181909190A190B1907F0120E028
:10D2400030E040EA51ECC501B4010F94353687FD5A
:10D250003FC020E030E040EA51E4C501B4010F9442
:10D26000052D1816ACF10F5F1F4FF4E0CF0ED11C47
:10D270000330110509F0A5CF64E3E62E67E0F62E32
:10D2800010E0F10181919191A191B1911F01F701FC
:10D2900081939193A193B1937F01812F0E94D41C1C
:10D2A0001F5F133071F70E94873160E08DE499E0D1
:10D2B0000E94693C63E972E084E690E00E94D739FD
:10D2C0006AEB72E084E690E00E94D7390C946F58C4
:10D2D0000F949D0B8BE699E00E94B1F761E08DE51C
:10D2E00099E00E94693C68E270E088EC90E00E945E
:10D2F000D7390C946F580E94C0AA0C946F580E94A2
:10D300000D9D0C946F5820930D050E94CB22109216
:10D310000D05882311F40C946F580F94A10B89E824
:10D3200099E00E94B1F70C946F5880914F1382FFDF
:10D3300005C0806480934F130C946F5883FD02C026
:10D340000C946F580E945CC40C946F580E94CE20BD
:10D35000082F87FF02C00C946F5885E50E9430EEBD
:10D36000882359F10E9406EE4B015C01E02E002E4D
:10D37000000CFF0820E030E0A9010F94353687FF4C
:10D3800004C0B7FAB094B7F8B09420E030E84BE3AB
:10D3900054E4C501B4010F943536970153E0220FD0
:10D3A000331F5A95E1F720523B4F1816D4F1D9019B
:10D3B0008D929D92AD92BC9213978CE40E9430EEB8
:10D3C000882311F40C946F580E9406EE6B017C01C7
:10D3D000002E000C110B20E030E0A9010F9435362F
:10D3E00087FF04C0F7FAF094F7F8F09420E030E8F3
:10D3F0004BE354E4C701B6010F943536980143E07E
:10D40000220F331F4A95E1F720523B4F18169CF02C
:10D41000D9011496CD92DD92ED92FC9217970C945F
:10D420006F5880E090E8ABE3B4E4F9018083918326
:10D43000A283B383C2CF80E090E8ABE3B4E4F90108
:10D4400084839583A683B7830C946F580E94542ECF
:10D450000C946F5828E01202F0011124E052FB4FA7
:10D46000C080D180E280F3800C94E35F0E947B5304
:10D470000C946F580E94E6FD0C946F5881E08093E5
:10D4800017061092831060E083E50E941DEF811162
:10D490000C946F580E948DB20C946F5883E50E94D3
:10D4A00030EE882341F00E94F2ED8093E8040E9460
:10D4B000B1EF0C946F580F94A10B84E999E00E948E
:10D4C000B1F78091E8040E94C4F90C946F580E944F
:10D4D000846C0C946F580E94E88181110C946F58F1
:10D4E0000C946560109198040E948BC8609394100E
:10D4F000709395108093961090939710112311F4C8
:10D500000C946F58812F0E9415850C946F5811113F
:10D5100007C011E089E50E9430EE082F811307C093
:10D52000012FF11204C011E001E0FF24F39482E521
:10D530000E947EEE882311F40C9410590E9406EE8E
:10D540006CA37DA38EA39FA320E030E0A9010F94DC
:10D55000052D882381F0111105C0011103C0FF20A2
:10D5600009F417C160E0CE0184960E9450300E94F9
:10D57000A3F50E946DF5112309F47EC0002309F480
:10D5800078C010924A0210924B0210924C021092F4
:10D590004D0210924E0210924F02109250021092C1
:10D5A00051020E945C318BE29FE00E9493E84B01A4
:10D5B0005C018FE29FE00E9493E82B013C01AC01EB
:10D5C0009B01C501B4010F943536181614F00C9464
:10D5D0001659A5019401C301B2010F94CF349B01E8
:10D5E000AC010F946B2D20E030E040E85FE30F9436
:10D5F000D5330F94833620E030E048E452E40F94B2
:10D600006B2D68A379A38AA39BA320E030E040ECB4
:10D610005FE3C301B2010F946B2D69837A838B831F
:10D620009C8320E030E040EC5FE3C501B4010F943F
:10D630006B2D6C8F7D8F8E8F9F8FAE01405E5F4F05
:10D64000BE016F5F7F4FCE014C960E940F300E944B
:10D65000561F10924A0210924B0210924C021092E6
:10D660004D0210924E0210924F02109250021092F0
:10D67000510280E00E948533002319F081E00E946E
:10D680008533FF2009F485C0109216051092150508
:10D690001092170583E00E94625281117AC00E94A5
:10D6A0005C31209134073091350740913607509115
:10D6B000370760E070E084E393E40F94D4332B01E8
:10D6C0003C01209138073091390740913A07509139
:10D6D0003B0760E070E084E393E40F94D4334B01A4
:10D6E0005C018091520290915302A0915402B0913A
:10D6F00055028093AA069093AB06A093AC06B09314
:10D70000AD060091A2111091A311D8012D913D9168
:10D710004D915C91C301B2010F94D4336093A20682
:10D720007093A3068093A4069093A506F801248124
:10D73000358146815781C501B4010F94D43360937C
:10D74000A6067093A7068093A8069093A90682EA7E
:10D7500096E00E948DED882311F40C941C591C8EC8
:10D760001D8E1E8E1F8E88E0E2EAF6E0DE01119625
:10D7700001900D928A95E1F7AE01445E5F4FBE01C4
:10D780006B5F7F4FCE0101960E940F3082E00E94B6
:10D7900085330E945C318091D2058093D3058E2D14
:10D7A0000E94C4F10E947C2D0E9487310C946F5816
:10D7B0000F949D0B84E199E00E94B1F70C946F588F
:10D7C000882309F4A6CEAFCEDF92EF92FF920F939B
:10D7D0001F93CF93DF93EC01E090B406F090B50671
:10D7E0008AE0D82E6AE070E0CE010F9423378C01D6
:10D7F000009711F0FC011082CE010E94D95081E007
:10D800000E9447560115110519F0E801D992EACF97
:10D81000C701DF91CF911F910F91FF90EF90DF90A3
:10D820000C94D9504F925F926F927F928F929F92F9
:10D83000AF92BF92CF92DF92EF92FF920F931F931E
:10D84000CF93DF93CDB7DEB77C014DB65EB6609067
:10D85000B4067090B5068DB69EB66AE070E0C7015A
:10D860000F94402C6C018C010E191F09892B21F497
:10D87000C7010F94522C8C01C80101962DB73EB7F9
:10D88000281B390B0FB6F8943EBF0FBE2DBF8DB7C6
:10D890009EB701965C01A801B7010F94732CF501A6
:10D8A000E00FF11F1082C5010E94D95081E00E9453
:10D8B0004756C114D10451F076019FEFE91AF90AD5
:10D8C0000FB6F8949EBE0FBE8DBEC5CF0FB6F894AE
:10D8D0009EBE0FBE8DBEC3010E94D9500FB6F894F4
:10D8E0005EBE0FBE4DBEDF91CF911F910F91FF9095
:10D8F000EF90DF90CF90BF90AF909F908F907F90F0
:10D900006F905F904F9008954F925F926F927F92C9
:10D910008F929F92AF92BF92CF92DF92EF92FF923F
:10D920000F931F93CF93DF93CDB7DEB7C059D109C3
:10D930000FB6F894DEBF0FBECDBF0E94BFEF8823A5
:10D94000B9F183E50E9430EE882309F449C088E9E3
:10D9500094E00E94B1F78AE00E9489F78EEF8093ED
:10D96000A40481E0809367021092A30481E09AE509
:10D970009093E6128093E5128CE490E09093E81285
:10D980008093E71287E08093D91282E88093DC12BB
:10D9900084E890E0A0E0B0E08093DD129093DE1286
:10D9A000A093DF12B093E01289E892E10E949937C8
:10D9B000C057DF4F0FB6F894DEBF0FBECDBFDF916B
:10D9C000CF911F910F91FF90EF90DF90CF90BF907C
:10D9D000AF909F908F907F906F905F904F90089541
:10D9E00083E40E9430EE882349F00E94A9EF0E9450
:10D9F000E7820E943C820E944440DACF8090E70791
:10DA00009090E807A090E907B090EA078091F007AE
:10DA100080FF05C09091140B98609093140B86952D
:10DA200081708093310882E495E00E94126C8091AD
:10DA30007607909177079E012F5F3F4F79010097FE
:10DA400099F09F938F9389E395E09F938F933F93F2
:10DA50002F930F949C2CC7010E94E46B0F900F90A2
:10DA60000F900F900F900F90809174079091750711
:10DA7000009799F09F938F9380E395E09F938F9306
:10DA8000FF92EF920F949C2CC7010E94E46B0F90C1
:10DA90000F900F900F900F900F906E0131E8C30E12
:10DAA000D11C609153077091540780915507909154
:10DAB0005607860123E041E00F94D2279F938F936E
:10DAC0008EE195E09F938F93FF92EF920F949C2CA1
:10DAD000C7010E94E46B86E195E00E94126C87E02A
:10DAE0008093560B809392040F900F900F900F909D
:10DAF0000F900F9080916F078823F9F06091700765
:10DB000070917107809172079091730723E041E053
:10DB10000F94D2279F938F938DE095E09F938F93DF
:10DB2000FF92EF920F949C2CC7010E94E46B0F9020
:10DB30000F900F900F900F900F908091780788238F
:10DB4000A1F01F928F931F921F9280E095E09F9308
:10DB50008F93FF92EF920F949C2CC7010E94E46B6D
:10DB60000FB6F894DEBF0FBECDBF80917907882332
:10DB7000A9F01F928F931F9281E08F9380E095E030
:10DB80009F938F93FF92EF920F949C2CC7010E945A
:10DB9000E46B0FB6F894DEBF0FBECDBF40907A079E
:10DBA00050907B0760907C0770907D0720E030E00C
:10DBB000A901C301B2010F94052D811104C0809108
:10DBC000F00782FF20C0860121E041E0C301B201DD
:10DBD0000F94D2279F938F938091F00782FB882721
:10DBE00080F91F928F9383EF94E09F938F93FF921E
:10DBF000EF920F949C2CC7010E94E46B0FB6F8942F
:10DC0000DEBF0FBECDBF6091450770914607809182
:10DC10004707909148078E010F581F4F23E041E0BE
:10DC20000F94D227782E692E609141077091420798
:10DC30008091430790914407860123E041E00F94CF
:10DC4000D2276F927F929F938F9382EE94E09F935F
:10DC50008F93FF92EF920F949C2CC7010E94E46B6C
:10DC60006091490770914A0780914B0790914C074A
:10DC700023E041E00F94D22787ED94E00E94126CDC
:10DC8000DF92CF928DEC94E09F938F93FF92EF926F
:10DC90000F949C2CC7010E94E46B809152078F93D4
:10DCA000809151078F9386EC94E09F938F93FF921E
:10DCB000EF920F949C2CC7010E94E46B60914D077A
:10DCC00070914E0780914F079091500723E041E0FB
:10DCD0000F94D2279F938F938CEB94E09F938F9315
:10DCE000FF92EF920F949C2CC7010E94E46B8CE092
:10DCF000E7E5F7E0A4E3B7E001900D928A95E1F73C
:10DD00008CE0E3E6F7E0A8E2B7E001900D928A9597
:10DD1000E1F780E00E94D41C81E00E94D41C82E0E4
:10DD20000E94D41C8091EF078093220781E08093AA
:10DD3000E8040E94B1EF8EE797E09F938F938BEDFD
:10DD400090E29F938F93FF92EF920F949C2C0FB6CB
:10DD5000F894DEBF0FBECDBFC7010E94E46B809177
:10DD6000EE078F938091ED078F938091EC078F934F
:10DD70008091EB078F93BF92AF929F928F928EEA22
:10DD800094E09F938F93FF92EF920F949C2CC70186
:10DD90000E94E46B0FB6F894DEBF0FBECDBF08CE75
:10DDA000CF93DF93C091B00CC0930A0881E6C89F5F
:10DDB000E0011124CE54D34F8091140B80FF05C095
:10DDC0000F94A10BCE010E945152CE010E94D95056
:10DDD00080E0DF91CF910C9447568BE1EFE6F3E1C1
:10DDE000AAE8B3E101900D928A95E1F780914F1373
:10DDF000806280934F130895CF9380913E10C1E0CD
:10DE00008823C9F080913F109091401040913610C6
:10DE1000509137106091381070913910DC01ED91FC
:10DE2000FC910288F389E02D26E33EE01995C82F86
:10DE3000811104C0C0E08C2FCF91089540913A1019
:10DE400050913B1060913C1070913D10411551056F
:10DE500061057105B9F080913F1090914010DC018F
:10DE6000ED91FC910288F389E02D26E33EE01995BF
:10DE7000882301F310923A1010923B1010923C103C
:10DE800010923D1010923E10D6CF0F931F93CF9358
:10DE9000DF93CDB7DEB760970FB6F894DEBF0FBE45
:10DEA000CDBF8C01DC01ED91FC910280F381E02D6E
:10DEB000BE016F5F7F4F1995882309F464C0898183
:10DEC000807CC9F56F81637070E0762F6627770FCD
:10DED000770F8885B4E08B9FC0011124682B792BC4
:10DEE00089858295869586958370682B6F5F7F4FB5
:10DEF00090E080E02A852370220F3B8537FB332793
:10DF000030F9232B3E813F70230F3327331F2750D7
:10DF1000310904C0660F771F881F991F2A95D2F711
:10DF200060960FB6F894DEBF0FBECDBFDF91CF91E4
:10DF30001F910F910895803419F56885669566954F
:10DF400070E090E080E0CB01772766272A85622B7E
:10DF5000098510E0102F0027012E000C220B330B37
:10DF6000602B712B822B932B6F5F7F4F8F4F9F4FB7
:10DF70004AE0660F771F881F991F4A95D1F7D0CFC7
:10DF80008BE0F801848360E070E0CB01C9CF089595
:10DF9000FC01828108954F925F926F927F928F92DF
:10DFA0009F92AF92BF92EF92FF920F931F93CF93E6
:10DFB000DF93B0E2A0E06A2F70E0AB014B0F511D80
:10DFC00055954795411117C0E6E6FFE1859194917B
:10DFD000282F822FDF91CF911F910F91FF90EF900B
:10DFE000BF90AF909F908F907F906F905F904F9079
:10DFF0000895B42FE2CFA41711F0B41303C0E2EEDA
:10E00000FFE1E4CF9A0121503109220F331F220F83
:10E01000331FF901EC59F04EE590F490F901E859FD
:10E02000F04E059114918E159F051CF3A42F08172F
:10E0300019070CF4C0CFBC01F901EA59F04EC591A3
:10E04000D491F901E659F04EA590B4906E197F096C
:10E05000072E000C880B990B0F940C2D2B013C0103
:10E06000B5016C1B7D0B072E000C880B990B0F94D0
:10E070000C2D9B01AC01C301B2010F946B2D4B0120
:10E080005C01B8016E197F09072E000C880B990BF3
:10E090000F940C2D9B01AC01C501B4010F94CF343A
:10E0A0004B015C01BE01DD0F880B990B0F940C2D09
:10E0B0009B01AC01C501B4010F94D5330F944135D8
:10E0C000262F972F86CFEF92FF920F931F93E09208
:10E0D0001105F09212050093130510931405609337
:10E0E0001C0570931D0580931E059FEFFF27621B83
:10E0F000730B840B30F4809570956195790B890BC7
:10E10000992790935415A6E06A9F00924815512DC7
:10E11000EE277A9F500DE11D8A9FE00D509349151F
:10E12000E0934A15AFE06A9F00924C15512DEE27FF
:10E130007A9F500DE11D8A9FE00D50934D15E0939D
:10E140004E15AAE06A9F00925015512DEE277A9F36
:10E15000500DE11D8A9FE00D50935115E09352152B
:10E160001F910F91FF90EF90089500008091D405CA
:10E1700080FF29C089988FEF809318068091D4057D
:10E18000869580FF23C08F988FEF8093190680912A
:10E19000D4058695869580FF1CC080910B01827006
:10E1A0008093090143988FEF80931A068091D405DC
:10E1B00086958695869580FF15C016988FEF80937B
:10E1C0001B0600000895899A81E0D6CF8F9A81E0DE
:10E1D000DCCF80910B018095827080930901439A76
:10E1E00081E0E2CF169A81E0EACF0F931F93CF939D
:10E1F000811113C0C42F8B010F94A10B80EC92E10D
:10E200000E94B1F7C8010E94B1F7CC2331F08AE037
:10E21000CF911F910F910C9489F7CF911F910F917E
:10E2200008950F9300910D0521E002272EE035E0BF
:10E230004CE050E0BC018EED94E00E940AF40F9196
:10E2400008950F9300910D0521E002272EE035E09F
:10E2500044E050E0BC018EED94E00E940AF40F917E
:10E2600008950F9300910D0521E002272EE035E07F
:10E2700041E050E0BC018EED94E00E940AF40F9161
:10E2800008950F9300910D0521E002272EE035E05F
:10E2900042E050E0BC018EED94E00E940AF40F9140
:10E2A00008950F9300910D0521E002272EE035E03F
:10E2B00041E050E0BC018EED94E00E940AF40F9121
:10E2C00008950F9300910D0521E002272EE035E01F
:10E2D00048E050E0BC018EED94E00E940AF40F91FA
:10E2E00008950F9300910D0521E002272EE035E0FF
:10E2F0004CE050E0BC018EED94E00E940AF40F91D6
:10E3000008950F9301E02EE035E041E050E0BC01BC
:10E310008EED94E00E940AF40F910895CF93DF935D
:10E32000C5E0D1E18A819B810E94E2C09D838C83FC
:10E33000CAE9D0E18A819B810E94CB6F9D838C8347
:10E34000A89510929006DF91CF9108951F93CF93D7
:10E35000DF93182FEB010F94A10B8AEF91E20E943B
:10E36000B1F786EE91E2113011F48CEE91E20E9449
:10E37000B1F7BE0182EF91E20F94930B8AE0DF9137
:10E38000CF911F910C9489F7CF93DF93EC018D818E
:10E390000F94732060E08B81DF91CF910C94F6C6CF
:10E3A000DF92EF92FF920F931F93CF93DF938C0135
:10E3B000C62FD22FF32EE42ED52E0E94C4710E94B8
:10E3C00013E48C2F80640F9467208D2D0F946720A9
:10E3D0008E2D0F9467208F2D0F9467208D2F0F9413
:10E3E000672087E8C11101C085E90F946720CC3010
:10E3F00011F40F946C20C0E00F946C20F801868318
:10E4000087FF04C0CF3F11F0CF5FF6CFDF91CF91F0
:10E410001F910F91FF90EF90DF90089561E0FC0154
:10E4200083810E94F6C68FEF0D9467200F931F9390
:10E43000CF938C010E94C4710E9413E4C82F8823DB
:10E4400071F08DEF0F9467200E9413E4C82FC8016C
:10E450000E940E728C2FCF911F910F91089582E12F
:10E46000F8018483F4CF8F929F92AF92BF92CF92A4
:10E47000DF92EF92FF920F931F93CF93DF93EC0104
:10E480006A017B01590120E030E0A90167E30E94A5
:10E49000D071A501980167E1CE010E94D071811170
:10E4A00027C08F81833039F089E0CC0CDD1CEE1C55
:10E4B000FF1C8A95D1F7A701960169E1CE010E9460
:10E4C000D07111E0882319F010E087E08C83CE0131
:10E4D0000E940E72812FDF91CF911F910F91FF90BB
:10E4E000EF90DF90CF90BF90AF909F908F90089566
:10E4F00089E08C8310E0EBCFCF93DF93EC016EBD0E
:10E50000FA01CA019E5F0DB407FEFDCF20812EBD2A
:10E510000DB407FEFDCF21812EBD3296E817F90715
:10E5200091F70DB407FEFDCF8FEF0F9467208FEFAB
:10E530000F9467200F946C208E838F71853049F083
:10E5400083E18C83CE010E940E7280E0DF91CF9137
:10E55000089581E0FBCF0F931F93CF93DF93EC01DE
:10E560008B010E94C4710E9413E481110CC085E1EB
:10E570008C8310E0CE010E940E72812FDF91CF912B
:10E580001F910F910895A8016CEFCE010E947C723B
:10E59000182F882361F3EECF0F931F93CF93DF9350
:10E5A000EC0189018F81833039F089E0440F551FD8
:10E5B000661F771F8A95D1F79A01AB0168E1CE01FA
:10E5C0000E94D07181112AC0A8016EEFCE010E9475
:10E5D0007C72182F8823B1F00E9413E4182F88232F
:10E5E000D1F020E030E0A9016DE0CE010E94D071B1
:10E5F000882321F086E18C8310E004C00F946C2006
:10E600008111F8CFCE010E940E72812FDF91CF9140
:10E610001F910F91089587E18C83F4CF86E0EBCFB3
:10E620001F93CF93DF93EC010E94C47120E030E090
:10E63000A9016CE0CE010E94D07111E0882319F08D
:10E6400010E083E08C83CE010E940E72812FDF9157
:10E65000CF911F9108951F93CF93DF93EC018F818A
:10E66000833039F089E0440F551F661F771F8A9564
:10E67000D1F79A01AB0162E1CE010E94D07111E0A5
:10E68000882319F010E085E08C83CE010E940E7281
:10E69000812FDF91CF911F9108958F929F92AF921A
:10E6A000BF92EF92FF920F931F93CF93DF938C0152
:10E6B000EB017A010E948BC84B015C012CE2820EB7
:10E6C00021E0921EA11CB11C0F946C20F8018683DE
:10E6D0008F3F69F40E948BC8681979098A099B09E0
:10E6E00097FDF2CF81E1F8018483C0E021C08E3F25
:10E6F00071F5F1E0EF1AF1088FEF8EBDFE012FEFFB
:10E700000DB407FEFDCF8EB581932EBDCF018C1BBE
:10E710009D0B8E159F05A0F30DB407FEFDCF8EB5A2
:10E72000CE0DDF1D88830F946C200F946C20C1E008
:10E73000C8010E940E728C2FDF91CF911F910F9113
:10E74000FF90EF90BF90AF909F908F9008958FE0D3
:10E75000CACF0F931F93CF93DF93EC018B010E94DD
:10E76000C47140E052E0B801CE01DF91CF911F911A
:10E770000F910C944D730F931F93CF93DF93EC0184
:10E7800089018F81833039F089E0440F551F661F5E
:10E79000771F8A95D1F79A01AB0161E1CE010E9402
:10E7A000D07181110AC040E052E0B801CE01DF9182
:10E7B000CF911F910F910C944D7384E08C83CE0107
:10E7C0000E940E7280E0DF91CF911F910F9108950A
:10E7D0008F929F92AF92BF92CF92DF92EF92FF9271
:10E7E0000F931F93CF93DF93EC01162F1F821C8290
:10E7F0004B830E948BC86B017C0120EDC20E27E089
:10E80000D21EE11CF11CA89561E08B810E94F6C626
:10E810008B810E9445B2209A289A219A2398229AA5
:10E8200081E00F94732085E08D830F9473200AE0BC
:10E830008FEF0F9467200150D9F7A89520E030E0C2
:10E84000A90160E0CE010E94D0718E83813081F0F9
:10E850000E948BC86C197D098E099F0997FDEECF28
:10E8600081E08C83CE010E940E721A8280E06AC021
:10E87000A8952AEA31E040E050E068E0CE010E942D
:10E88000D071853041F581E08F83A8958F81812CEF
:10E89000912C5401823029F4812C912CA12C80E4FC
:10E8A000B82E20E030E0A90167E3CE010E94D071CC
:10E8B000A501940169E2CE010E94D0718E83882364
:10E8C000F1F00E948BC86C197D098E099F0997FD94
:10E8D000E8CF8AE0C6CF04E00F946C208E8301500D
:10E8E000D9F78A3A11F482E0CFCF0E948BC86C1915
:10E8F0007D098E099F0997FDBCCF82E0B2CF8F8141
:10E900008230C1F420E030E0A9016AE3CE010E9428
:10E91000D071882311F088E0A4CF0F946C20807C04
:10E92000803C11F483E08F830F946C200F946C2053
:10E930000F946C20CE010E940E7281E08A83173002
:10E9400070F41D83DF91CF911F910F91FF90EF9095
:10E95000DF90CF90BF90AF909F908F90089588E107
:10E960008C8384CF0F931F93CF93DF93EC018B01A4
:10E9700020E030E0A90169E00E94D07181110AC055
:10E9800040E150E0B801CE01DF91CF911F910F918E
:10E990000C944D7380E18C83CE010E940E7280E056
:10E9A000DF91CF911F910F9108951F920F920FB693
:10E9B0000F9211242F933F938F939F93AF93BF9305
:10E9C00080919A0690919B06A0919C06B0919D061D
:10E9D0003091990623E0230F2D3758F50196A11D9C
:10E9E000B11D2093990680939A0690939B06A0935D
:10E9F0009C06B0939D0680919E0690919F06A091E3
:10EA0000A006B091A1060196A11DB11D80939E069E
:10EA100090939F06A093A006B093A106BF91AF91DB
:10EA20009F918F913F912F910F900FBE0F901F904C
:10EA3000189526E8230F0296A11DB11DD2CFCF92C3
:10EA4000DF92EF92FF920F931F93CF93DF93CDB797
:10EA5000DEB7A0970FB6F894DEBF0FBECDBF44233C
:10EA600009F445C0611571058105910579F100E052
:10EA7000C42ED12CF12CE12CA70196010F9449331F
:10EA800011E0100FE1E0F0E0EC0FFD1FE00FF11DD1
:10EA900007FDFA956083B901CA01012F611571055F
:10EAA0008105910549F7115010F1E1E0F0E0EC0F1C
:10EAB000FD1FE10FF11D17FDFA95908187E39A3054
:10EAC00008F480E3890F0E9489F7EDCF80E3A096D8
:10EAD0000FB6F894DEBF0FBECDBFDF91CF911F916F
:10EAE0000F91FF90EF90DF90CF900C9489F7A09654
:10EAF0000FB6F894DEBF0FBECDBFDF91CF911F914F
:10EB00000F91FF90EF90DF90CF9008958091441384
:10EB10008823C1F0815080934413EFE6F3E188230A
:10EB200051F08150990B2BE1289FF001299FF00DA6
:10EB30001124EB55FC4E8BE1AAE8B3E101900D9254
:10EB40008A95E1F780914413811105C090914F138C
:10EB5000906290934F130895CF92DF92EF92FF92BD
:10EB600080914F1382FF29C0C0904B13D0904C135B
:10EB7000E0904D13F0904E1381EB91E20E94B1F7BB
:10EB80004AE0C701B6010E941F758FE20E9489F713
:10EB900060914713709148138091491390914A13E3
:10EBA0004AE00E941F758DE00E9489F78AE0FF907D
:10EBB000EF90DF90CF900C9489F783EC91E2FF9077
:10EBC000EF90DF90CF900C94B1F7BC0185EE90E20E
:10EBD0000F94930B82EE90E20C94B1F780914F1357
:10EBE00083FF03C0846080934F130895CF92DF9218
:10EBF000EF92FF920F931F93CF93DF93CDB7DEB7C2
:10EC0000EDB6FEB6DC010D900020E9F79D01281B52
:10EC1000390B285F3F4FEDB7FEB7E21BF30B0FB682
:10EC2000F894FEBF0FBEEDBF0DB71EB70F5F1F4FAD
:10EC30009F938F938BED90E29F938F931F930F93EE
:10EC40000F949C2C6801F4E0CF0ED11C0F900F9014
:10EC50000F900F900F900F90D6018D916D0188232A
:10EC600049F0082E000C990B0F94E736F601319706
:10EC70008083F2CF66ED70E2C8010F94352C4FE32C
:10EC800050E0B80186ED95E00F9443370FB6F89445
:10EC9000FEBE0FBEEDBEDF91CF911F910F91FF9091
:10ECA000EF90DF90CF900895FC01938591FD13C004
:10ECB000987121E0903109F020E080914F1320FB02
:10ECC00084F980934F13903141F08085873419F493
:10ECD00081858E3711F480E0089581E00895FC016C
:10ECE00020E03EE2DB014D91BD01403249F0283089
:10ECF00011F430833196DB0111974C9140833196AA
:10ED00002F5F2B3079F710820895EF92FF920F93C7
:10ED10001F93CF93DF93CDB7DEB7A0970FB6F894CC
:10ED2000DEBF0FBECDBF7C018B01BE016F5F7F4F89
:10ED3000C7010E9479AC1816A4F4CE0101960E9476
:10ED40005476882391F3BE016F5F7F4F80EB90E193
:10ED50000E946F7660EB70E1C8010F940537892B34
:10ED600021F7A0960FB6F894DEBF0FBECDBFDF919E
:10ED7000CF911F910F91FF90EF900895CF92DF9266
:10ED8000EF92FF92CF936B017C01C42F80913610DC
:10ED900090913710A0913810B09139108C159D05C5
:10EDA000AE05BF0529F10E94FC6E811108C0C0E0CC
:10EDB0008C2FCF91FF90EF90DF90CF9008958091AE
:10EDC0003F1090914010DC01ED91FC910088F18999
:10EDD000E02D26E33EE0B701A6011995882339F31B
:10EDE000C0923610D0923710E0923810F09239105D
:10EDF000CC2321F081E080933E10DACFC1E0D8CF60
:10EE00004F925F926F927F928F929F92AF92BF923A
:10EE1000CF92DF92EF92FF920F931F93CF93DF93E6
:10EE2000EC01423051056105710590F480E0DF91FD
:10EE3000CF911F910F91FF90EF90DF90CF90BF90F7
:10EE4000AF909F908F907F906F905F904F900895BC
:10EE500089859A85AB85BC850196A11DB11D841756
:10EE60009507A607B70710F38F898031C9F5852E5E
:10EE7000962EA72EBB248B899C89AD89BE89880ECE
:10EE8000991EAA1EBB1E280139016A017B0141E0BF
:10EE9000C501B4010E94BE76882341F29F8990315A
:10EEA00081F5DD24EE24FF24F601EE0FFF1FEA5C5E
:10EEB000F14F118300839A89923008F4B8CF4D81C5
:10EEC0005E816F817885840E951EA61EB71E809286
:10EED0003A1090923B10A0923C10B0923D10A7CFF8
:10EEE000803209F0A3CF8B899C89AD89BE894A0104
:10EEF0005B01E7E0B694A79497948794EA95D1F7DD
:10EF0000BECFE894C7F8DD24EE24FF24F601EE0F0F
:10EF1000FF1FEE0FFF1FEA5CF14F408251826282B9
:10EF20007382C9CFCF92DF92EF92FF920F931F931C
:10EF3000CF93DF93FC0181859285A385B4850196EB
:10EF4000A11DB11D84179507A607B70750F480E0EF
:10EF5000DF91CF911F910F91FF90EF90DF90CF90B5
:10EF6000089587898031A9F5BB27A72F962F852F74
:10EF7000C388D488E588F6888C0D9D1DAE1DBF1D05
:10EF8000E9016A017B018F014091361050913710E1
:10EF9000609138107091391084179507A607B7074C
:10EFA00049F5F8018789803169F5B701A601552730
:10EFB00066277727440F551F4A5C514FFA0180811D
:10EFC0009181B0E0A0E088839983AA83BB8381E02C
:10EFD000BFCF803209F0BBCFC388D488E588F688DC
:10EFE000DB01CA01C7E0B695A79597958795CA95A5
:10EFF000D1F7C2CF40E0BC01CD010E94BE768111A5
:10F00000D0CFA5CFB701A6014F7755276627772721
:10F01000440F551F440F551F4A5C514FFA01808120
:10F020009181A281B381BF70CECF4F925F926F92D8
:10F030007F92AF92BF92CF92DF92EF92FF920F93A7
:10F040001F93CF93DF9300D01F92CDB7DEB78C0113
:10F0500049835A836B837C835901C12CD12C76015F
:10F06000412C82E0582E612C712C49815A816B8190
:10F070007C819E012F5F3F4FC8010E9492778823B9
:10F0800019F1F8018585A301920104C0220F331FF5
:10F09000441F551F8A95D2F7DA01C901C80ED91E3F
:10F0A000EA1EFB1E49815A816B817C8187898031F0
:10F0B000F1F481E0483F5F4F61057105B0F2F50161
:10F0C000C082D182E282F3820F900F900F900F9056
:10F0D000DF91CF911F910F91FF90EF90DF90CF9034
:10F0E000BF90AF907F906F905F904F90089581E0B8
:10F0F000483F5F4F6F4F7F4008F4B7CFE0CF0F938B
:10F100001F93CF93DF93FC012381222331F080E012
:10F11000DF91CF911F910F9108958B01EC01FB01BD
:10F120008789803139F582E08B831D8A1E8A1F8A88
:10F13000188E808D918DB0E0A0E025E0880F991F9A
:10F14000AA1FBB1F2A95D1F7898B9A8BAB8BBC8BDF
:10F150001A8F098F81E08983188619861A861B8683
:10F160001C821D821E821F82188A1C861D861E8696
:10F170001F86CECF803259F683E08B83428D538D2C
:10F18000648D758D4D8B5E8B6F8B788F9E012F5E9E
:10F190003F4FC8010E9415788111DACFB8CF3F9256
:10F1A0004F925F926F927F928F929F92AF92BF9297
:10F1B000CF92DF92EF92FF920F931F93CF93DF9343
:10F1C000CDB7DEB72C970FB6F894DEBF0FBECDBF1C
:10F1D0005C01DC0159968D909C90F40181859285AB
:10F1E000A385B4859C01AD012F5F3F4F4F4F5F4F0B
:10F1F00029873A874B875C87D50114964D905D909F
:10F200006D907C901797411451046104710409F4C6
:10F2100059C0BFEF4B1A5B0A6B0A7B0A312C730192
:10F2200062011D821E821F821886F40181859285EB
:10F23000A385B4852D813E814F81588528173907D4
:10F240004A075B0708F056C089859A85AB85BC855F
:10F250008C159D05AE05BF0550F482E0C82ED12C5B
:10F26000E12CF12C92E0492E512C612C712C9E0145
:10F270002F5F3F4FB701A601C4010E9492778823F8
:10F28000C9F189819A81AB81BC81892B8A2B8B2B17
:10F2900001F1260137019FEF491A590A690A790AD3
:10F2A0002D813E814F8158852F5F3F4F4F4F5F4FDC
:10F2B0002D833E834F8358873FEFC31AD30AE30A57
:10F2C000F30AB3CF4080518062807380332433943B
:10F2D000A6CFC414D504E604F70411F70FEF1FEF0F
:10F2E0002FEF3FE0B701A601C4010E940077782EFE
:10F2F00081111AC0712C872D2C960FB6F894DEBFA1
:10F300000FBECDBFDF91CF911F910F91FF90EF9076
:10F31000DF90CF90BF90AF909F908F907F906F9035
:10F320005F904F903F900895F5014481558166812B
:10F330007781411551056105710539F09701860105
:10F34000C4010E9400778823A9F2D5011496CD92BA
:10F35000DD92ED92FC921797332051F0D701C60150
:10F360000196A11DB11DF40180839183A283B38313
:10F37000F50185899689A789B08D892B8A2B8B2BDE
:10F3800009F0B9CFC58AD68AE78AF08E8181806874
:10F390008183B1CFCF93DF93EC01462F41706C8511
:10F3A0007D858E859F850E94BE76882351F0888951
:10F3B00020E2829FC00111248A5C914FDF91CF919E
:10F3C000089590E080E0FACFCF93DF93EC0189912C
:10F3D000882319F00E9489F7FACFDF91CF91089521
:10F3E000CF93DF93EC018B81882349F1898187FFDB
:10F3F00022C061E0CE010E94CA79FC01892BF9F09C
:10F400008081853EE1F08B81823040F489899A8940
:10F41000AB89BC89848F958FA68FB78F8D899E8984
:10F42000938F828F8D899E89AF89B88DB58BA48B80
:10F4300089818F778983DF91CF910C94FC6E81E075
:10F44000888380E0DF91CF9108958F929F92AF9251
:10F45000BF92CF92DF92EF92FF920F931F93CF93C1
:10F46000DF93EC018B8181110EC080E0DF91CF91A1
:10F470001F910F91FF90EF90DF90CF90BF90AF90D2
:10F480009F908F90089509891A892B893C890417C8
:10F4900015072607370748F34A015B01823031F42C
:10F4A00088869986AA86BB8681E0E0CF8114910484
:10F4B000A104B10449F4188619861A861B861C8299
:10F4C0001D821E821F82F0CF088519852A853B8503
:10F4D000E98DFA8D858590E00996B901A801415022
:10F4E000510961097109082E04C0769567955795F1
:10F4F00047950A94D2F775016401E1E0CE1AD1086C
:10F50000E108F10804C0F694E794D794C7948A956B
:10F51000D2F7C416D506E606F70620F0012B022B1B
:10F52000032B11F58D899E89AF89B88D8C839D83BE
:10F53000AE83BF838E010C5F1F4FC114D104E10461
:10F54000F10409F4ADCF4C815D816E817F8198011A
:10F55000898D9A8D0E94927791E0C91AD108E108AD
:10F56000F1088111EACF81CFC41AD50AE60AF70A59
:10F57000E1CF2F923F924F925F926F927F928F9244
:10F580009F92AF92BF92CF92DF92EF92FF920F9332
:10F590001F93CF93DF9300D01F92CDB7DEB78C01BE
:10F5A0004B011A01DC0113968C911397813009F0FD
:10F5B000CFC011968C9181FFCBC082FDB5C0610197
:10F5C000D80118964D915D916D917C911B97C11456
:10F5D000D10409F41BC159968D919C915A97FC0155
:10F5E00074802FEF270D2A013B0139E07694679450
:10F5F000579447943A95D1F7722E74207A01F1E02E
:10F60000FF22711020C0E114F104E9F414964D9129
:10F610005D916D917C9117974115510561057105BB
:10F6200009F09CC055968D919D910D90BC91A02D97
:10F630000097A105B10509F0AAC0C8010E94CF78C2
:10F64000882309F485C0A12C82E0B82EAE18BF082B
:10F65000CA14DB0408F45601D80159964D915C9107
:10F660005A9714968D919D910D90BC91A02D029763
:10F67000A109B109FA01258504C0880F991FAA1FA5
:10F68000BB1F2A95D2F74685578560897189840FFB
:10F69000951FA61FB71F9C01AD01270D311D411DF0
:10F6A000511D29013A01A11432E0B30609F07DC0D1
:10F6B0008091361090913710A0913810B091391088
:10F6C000481659066A067B0669F410923E108FEFC1
:10F6D0009FEFDC018093361090933710A093381081
:10F6E000B093391080913F1090914010DC01ED9162
:10F6F000FC910288F389E02D9401B301A2011995D0
:10F70000882331F1F80180859185A285B3858A0D22
:10F710009B1DA11DB11D80879187A287B3878A0C8D
:10F720009B1CCA18DB084CCFF801418952896389B8
:10F73000748980859185A285B385481759076A0722
:10F740007B0709F43CCFC8010E94257A811137CF8D
:10F7500081E0D8018C938FEF9FEF6EC09E012F5FE9
:10F760003F4F0E949277882399F389819A81AB81D8
:10F77000BC81F801218D328DF9012789203169F48E
:10F78000883FFFEF9F07A105B10508F056CFF801AC
:10F7900084839583A683B78356CF883F2FEF920744
:10F7A000A2072FE0B20798F348CFE114F10431F536
:10F7B000F801408551856285738581899289A38985
:10F7C000B489481759076A077B07C0F00E94FC6E8E
:10F7D000882309F4BDCF81E080933E10409236101B
:10F7E000509237106092381070923910A501B40110
:10F7F000C7018A5C914F0F94FC3684CF41E0C3016E
:10F80000B2010E94BE768111F1CFA2CFF8018189A9
:10F810009289A389B48984179507A607B70738F496
:10F820008181418B528B638B748B80688183F8015B
:10F83000818183FD18C0C1010F900F900F900F9030
:10F84000DF91CF911F910F91FF90EF90DF90CF90BC
:10F85000BF90AF909F908F907F906F905F904F90F0
:10F860003F902F900895C8010E94F0798111E3CF55
:10F870006FCF2F923F924F925F926F927F928F92B3
:10F880009F92AF92BF92CF92DF92EF92FF920F932F
:10F890001F93CF93DF93EC014B017A018B81811190
:10F8A00015C08FEF9FEFDF91CF911F910F91FF90C8
:10F8B000EF90DF90CF90BF90AF909F908F907F9010
:10F8C0006F905F904F903F902F900895898180FFB7
:10F8D000E8CF89899A89AB89BC89488559856A8529
:10F8E0007B85841B950BA60BB70BA70170E060E02E
:10F8F00084179507A607B70708F47C0167011E0166
:10F9000024E0220E311CC114D10409F4A9C0488599
:10F9100059856A857B855A0181E0B822898D9A8D47
:10F920002A013B0129E076946794579447942A95DD
:10F93000D1F72B81FC01223081F5628D738D848D8E
:10F94000958D640D751D861D971D00E012E00A1946
:10F950001B09C016D10608F486010115E2E01E0756
:10F9600071F44090361050903710609038107090BD
:10F970003910641575058605970509F04EC040E0FD
:10F980000E94BE76882309F48CCFB5016A5C714F62
:10F99000A801C4010F94FC3652C0148111501421E7
:10F9A000A114B10471F411110CC0452B462B472B47
:10F9B00051F58D899E89AF89B88D8C839D83AE83E7
:10F9C000BF83E98DFA8D4C805D806E807F8022E060
:10F9D000421A510861087108858504C0440C551C01
:10F9E000661C771C8A95D2F786859785A089B18990
:10F9F000480E591E6A1E7B1EC301B201610F711DA4
:10FA0000811D911DA2CF4C815D816E817F8191010D
:10FA10000E9492778111D5CF44CFA0913F10B09131
:10FA20004010ED91FC9111970088F189E02D94012F
:10FA3000AB01BC01CD011995882309F432CF800EAA
:10FA4000911E88859985AA85BB85800F911FA11D70
:10FA5000B11D88879987AA87BB87C01AD10A53CF5F
:10FA6000C70121CFCF93DF93EB01FC01238121114B
:10FA700004C080E0DF91CF9108952250223028F415
:10FA80008FE28883198281E0F5CF60E00E94CA7915
:10FA9000009779F3DC0160E080E09EE22D91203256
:10FAA00099F0883031F49E01260F311DF9019083C1
:10FAB0006F5F9E01260F311DAD0141505109FA01C2
:10FAC0004081F90140836F5F8F5F8B3039F7FE0112
:10FAD000E60FF11D1082D7CFCF93DF93EC01CB015E
:10FAE000E881F981608171810E94327D28813981AC
:10FAF000D901ED91FC91AA81BB818C9190819923D0
:10FB000059F08936C8F4CF010196F90191838083B9
:10FB10008C918F5F8C93EACF893670F48FE280836B
:10FB2000E881F98180819181019691838083EA81C6
:10FB3000FB8180818F5F8083DF91CF9108950F9348
:10FB40001F93CF93DF9300D000D01F92CDB7DEB7C5
:10FB50009C012F5F3F4F3F832E832FE2FC012083C8
:10FB600081E08D83CE0106969A83898301979C83D9
:10FB70008B8310E00BE180914413181758F4109F09
:10FB8000B00111246B557C4ECE0101960E946C7D14
:10FB90001F5FF1CF8D818B3558F463EB74E1CE019B
:10FBA00001960E946C7D8E819F8101979F838E8339
:10FBB000EE81FF81108227960FB6F894DEBF0FBE4C
:10FBC000CDBFDF91CF911F910F910895CF93DF9318
:10FBD000EC010E94F0791B82DF91CF910895109281
:10FBE000411080914F138F7B8B7F80934F130E9426
:10FBF000E0F3882321F083EB94E10C94E67D0895F3
:10FC000080914F1382FF0AC0806480934F138091CC
:10FC10004F13877F806280934F1308950E94EF7D7A
:10FC2000F6CFCF93DF9380914F13877F80934F134D
:10FC300080917213882321F08FE693E10E94E67D84
:10FC40008091501390915113DC01ED91FC91019042
:10FC5000F081E02D45E360E0199581110EC00F940D
:10FC6000A10B8AEC90E20E94B1F780914F1383FFC1
:10FC700030C0DF91CF910C94ED6EC0915013D091B4
:10FC8000511361E0CE010E94DFB081110BC060E032
:10FC9000CE010E94DFB0811105C00F949D0B86EB51
:10FCA00090E2E1CF6AE171E18FE693E10E947F7813
:10FCB000811105C00F949D0B85EA90E2D4CF80910D
:10FCC0004F13886080934F130F94A10B89E990E242
:10FCD000CACF80911706882339F06FEF8CE890E245
:10FCE000DF91CF910C94693CDF91CF91089540E072
:10FCF00050E0BA010C94257A0F931F93CF93DF93B2
:10FD0000CDB7DEB7EB970FB6F894DEBF0FBECDBF11
:10FD100080914F1300E010E083FF23C08AE893E155
:10FD20000E94777E8BE1EAE8F3E1DE019196019093
:10FD30000D928A95E1F710E000E0BE016F5F7F4F02
:10FD4000CE0181960E9479AC18163CF4CE01019642
:10FD50000E945476080F111DF0CFCE0181960E94AB
:10FD6000D1EFC801EB960FB6F894DEBF0FBECDBF42
:10FD7000DF91CF911F910F9108950F931F93CF9310
:10FD8000DF93CDB7DEB76B970FB6F894DEBF0FBE2B
:10FD9000CDBF8C018AE893E10E94777E8BE1EAE88F
:10FDA000F3E1DE01119601900D928A95E1F7B80119
:10FDB000CE0101960E948576CE0101960E94D1EF78
:10FDC0006B960FB6F894DEBF0FBECDBFDF91CF911B
:10FDD0001F910F9108954F925F926F927F92AF9211
:10FDE000BF92CF92DF92EF92FF920F931F93CF9328
:10FDF000DF931F92CDB7DEB78C017B015A01C22E73
:10FE0000DB0159968D919C91F801928F818FCB01E6
:10FE10000E94777E712CF70180859185A285B3853C
:10FE2000418952896389748984179507A607B707A2
:10FE300008F052C055E0B695A795979587955A95C5
:10FE4000D1F7F82FFF70DF2ED70113968C918230F7
:10FE500010F480E0DBC041E050E0BE016F5F7F4FF7
:10FE6000C7010E94397C0197A1F7F7018085918530
:10FE7000A285B3854F96A11DB11D80879187A2876A
:10FE8000B387F0E2DF9EB00111246A5C714F611507
:10FE90007105F9F2DB018C91882341F0853E09F070
:10FEA0004CC0772029F077247394B5CF71100EC021
:10FEB0008091361090913710A0913810B091391080
:10FEC000F80184879587A687B787D08ADB018C9154
:10FED0008111E9CF772473948C2D8274823409F0D8
:10FEE000B8CF772009F4A2C0F801D08861E0C8013A
:10FEF0000E94CA79009709F4ACCF20E2DC011D9280
:10FF00002A95E9F72BE0F501DC0101900D922A9585
:10FF1000E1F721E238E2FC01318B208B40E058E030
:10FF200057874687338B228B318F208F578B468B99
:10FF30000E94FC6E811109C08CCF4BE050E0C501DE
:10FF40000F94EF36892B09F066CFF0E2DF9ED001E7
:10FF500011249D012A5C314FF9018385817121F0C3
:10FF60008C2D827109F001C1F801818D928D409133
:10FF700036105091371060913810709139104487C5
:10FF8000558766877787D08AFD01EA5CF14F448800
:10FF90005588712C612C320155244424D801559682
:10FFA0004D925D926D927C925897428D538D70E088
:10FFB00060E0442955296629772955964D935D932C
:10FFC0006D937C935897D9011B962C91287109F059
:10FFD000BEC0848D958DA68DB78DF801818B928BD7
:10FFE000A38BB48B81E083838C2D8F70F801818388
:10FFF0001482158216821782108611861286138645
:020000021000EC
:1000000081E0C4FE03C0C8010E949EAD0F90DF9145
:10001000CF911F910F91FF90EF90DF90CF90BF9005
:10002000AF907F906F905F904F900895D701139697
:100030008C911397823009F40CCF51968D919D913C
:100040000D90BC91A02D803E9F4FAF41B10508F0AF
:1000500000CFC7010E94CF78882309F4FACE0E940E
:10006000FC6E882309F4F5CED7015996ED91FC91E9
:100070005A9714964D905D906D907C901797B2E0D2
:100080004B1A510861087108858504C0440C551C41
:10009000661C771C8A95D2F786859785A089B189D9
:1000A000480E591E6A1E7B1E81E080933E104092CE
:1000B0003610509237106092381070923910E6E383
:1000C000FEE080E092E0DF019C011D922150304073
:1000D000E1F7DD24D394D7015996ED91FC91848109
:1000E000D816C0F480913F1090914010DC01ED9142
:1000F000FC910288F389E02D26E33EE0B301A201E2
:100100004D0D511D611D711D1995882309F4A1CE56
:10011000D394E1CF258580E092E0A0E0B0E004C078
:10012000880F991FAA1FBB1F2A95D2F7F701418993
:10013000528963897489840F951FA61FB71F818B0D
:10014000928BA38BB48B86E39EE0D12CD6CE20314C
:1001500061F498012F5E3F4F0E941578882329F0A3
:1001600084E0D80113968C933FCFD80113961C924C
:1001700070CE2F923F924F925F926F927F928F92AA
:100180009F92AF92BF92CF92DF92EF92FF920F9326
:100190001F93CF93DF93CDB7DEB7C354D1090FB60A
:1001A000F894DEBF0FBECDBF4C015B016A01222E69
:1001B00019821C821C8E1F8E6115710521F510E0BD
:1001C000CE014C960E94D1EFCE0101960E94D1EF54
:1001D000812FCD5BDF4F0FB6F894DEBF0FBECDBFD2
:1001E000DF91CF911F910F91FF90EF90DF90CF9013
:1001F000BF90AF909F908F907F906F905F904F9047
:100200003F902F900895FC0183818111D8CFFA018E
:1002100080818F32A1F18B01CE0101967C013C01DE
:1002200080E2382E2E019CE1490E511C2396EFAE40
:1002300023972496FFAE249722963FAE22972196CD
:100240003FAE21973FAE3EAE3DAE3CAE3BAE3AAE8A
:1002500039AE38AE3FAA960190E047E0D9018D91C2
:10026000882309F447C08F3209F444C08E3209F55F
:100270004A3009F4A4CF98E04AE09D01EFCFFB019A
:10028000838182508B01823060F0618D728DCE014E
:100290004C960E947F788E01045E1F4F882309F4DC
:1002A0008ECFC6016C010196F60120812F32D1F369
:1002B000B3CFE8E6F0E22491222321F031968213B5
:1002C000FACF7DCF491708F47ACF813208F477CF7F
:1002D0008F3709F474CF3FE9380F3A3108F420EE34
:1002E000E7E3F0E0EC0FFD1FE90FF11D820F8083C3
:1002F0009F5FC3CF8FA9803209F461CF6901F901F3
:1003000080812F5F3F4F8F32C9F3882301F121E0B5
:10031000AE01495C5F4FB801C7010E94EB7E8823A4
:1003200009F44DCF0A151B0519F0C8010E94E67D9E
:10033000942D852D6E147F0431F023969FAD239765
:1003400024968FAD24978701E92EF82E75CF222DA4
:10035000AE01495C5F4FB801C4010E94EB7E182FCB
:100360002FCF1F93CF93DF93CDB7DEB76D970FB627
:10037000F894DEBF0FBECDBF1D8E1C8EAC01BE013A
:10038000645E7F4F80E00E94DCAF10E00097A9F030
:1003900019821C826C8D7D8D21E0AC01CE0101960D
:1003A0000E94B980182F882321F0CE0101960E9467
:1003B000E67DCE0101960E94D1EF812F6D960FB69A
:1003C000F894DEBF0FBECDBFDF91CF911F9108958E
:1003D000EF92FF921F93CF93DF9300D000D000D015
:1003E0001F92CDB7DEB780914F1383FF0E94117E1D
:1003F00080914F1383FF3CC00E94BFEF811138C032
:100400008091451390E08F969F938F938FEF91E2A9
:100410009F938F93CE0101967C019F938F930F94AE
:100420009C2C80914F130F900F900F900F900F9076
:100430000F9083FF1DC0C7010E94B181182F882330
:10044000B9F00E94ED6EC7010E94F67580914513C8
:100450008F5F80934513812F2A960FB6F894DEBFE5
:100460000FBECDBFDF91CF911F91FF90EF90089508
:100470001092451310E0EFCF81E0809345130C9468
:10048000E881CF9390914F1393FF23C0909157131E
:1004900091111FC02AE5811121E0C82F4EEF52E0D3
:1004A0006FE673E184E593E10E94B980811105C094
:1004B0008EEF92E0CF910C94E575C1110AC06EEFFA
:1004C00072E084ED91E20F94930B8AE0CF910C944B
:1004D00089F7CF910895CF9321E04EEF52E06FE678
:1004E00073E184E593E10E94B980C82F882321F04D
:1004F00084E593E10E94E67D8C2FCF910895FF92D1
:100500000F931F93CF93DF93CDB7DEB76D970FB6E1
:10051000F894DEBF0FBECDBF20914F1323FF2DC037
:10052000AC01BE01645E7F4F80E00E94DCAF8C01B5
:10053000009719F16C8D7D8D19821C8222E0AC012F
:10054000CE0101960E94B980811123C0F12CCE0109
:1005500001960E94D1EFB801FF2081F183EA91E278
:100560000F94930B8AE00E9489F710924B1310921C
:100570004C1310924D1310924E136D960FB6F894C3
:10058000DEBF0FBECDBFDF91CF911F910F91FF90C6
:100590000895CE0101960E949EAD8823B9F261E0D4
:1005A000CE0101960E94CA79009781F225EEFC01E6
:1005B00020831C820E94FC6EF82EC9CF8BE891E24A
:1005C0000F94930B88E891E20E94B1F7D6CF0E9476
:1005D0006B82882331F00E94A9EF8EEF92E00C9499
:1005E0007F8208950F931F93CF93DF931F921F92E3
:1005F000CDB7DEB720914F1323FF32C08C01BC0171
:1006000082E00E94A671109246130E94EF7DA8011D
:10061000BE016F5F7F4F80E00E94DCAF8C010097CE
:10062000F9F069817A8126E5AC0183EB94E10E94BF
:10063000B9808823E1F080914F13816080934F133C
:10064000C8010E94BD7E10924313B80184ED91E26F
:100650000F94930B8AE00E9489F7C8010E9475AF3E
:100660000F900F90DF91CF911F910F910895C801C6
:100670000E94E575F5CFCF92DF92EF92FF920F9334
:100680001F93CF93DF931F921F92CDB7DEB72091B8
:100690004F1323FF62C08C01613009F470C008F46D
:1006A00067C0623009F4CFC00E94EF7DA801BE018F
:1006B0006F5F7F4F81E00E94DCAF8C01009709F4EF
:1006C0004CC069817A8121E0AC0183EB94E10E9406
:1006D000B980882309F4BEC08091C4149091C514D8
:1006E000A091C614B091C7148093471390934813F8
:1006F000A0934913B0934A1310924B1310924C13CA
:1007000010924D1310924E13B80180E191E20F94B4
:10071000930BC0904713D0904813E0904913F0908A
:100720004A1388E091E20E94B1F74AE0C701B6019E
:100730000E941F758AE00E9489F789EF90E20E946B
:10074000B1F7C8010E94BD7E8091BD10882311F0D1
:100750000DEB10E1C8010E9475AF0F900F90DF9173
:10076000CF911F910F91FF90EF90DF90CF90089560
:10077000BC0182E00E94A6711092461395CF0E94A0
:10078000E0F3811105C0B80181E00E94A6718CCF11
:1007900080914613882391F00F949D0B61E070E0E7
:1007A00089E691E20E9404FA8AE00E9489F740E01B
:1007B00070E060E088E591E20F947B0E8FE495E0B5
:1007C0000E949F7DE091461384E0E89FF001112490
:1007D000E55BFA4F80914B1390914C13A0914D1310
:1007E000B0914E1380839183A283B3830F94A10BA6
:1007F000B8018FE391E20F94930B6091461389E661
:10080000689FB0011124615B7A4F84E391E20F94F9
:10081000930BC0904B13D0904C13E0904D13F0907D
:100820004E138EE291E20E94B1F74AE0C701B60191
:100830000E941F758AE00E9489F7809146138F5F9E
:100840008093461331CF0F94A10B8EE191E20E9469
:10085000B1F72ACFC8010E94E5757FCF6F927F92D2
:100860008F929F92AF92BF92CF92DF92EF92FF92C0
:100870000F931F93CF93DF93CDB7DEB7C356D10944
:100880000FB6F894DEBF0FBECDBF5C018B016DB615
:100890007EB67E0187E5E80EF11CBE016F5F7F4FDB
:1008A000C5010E9479AC18160CF0A4C08C85887123
:1008B000803109F076C08DB69EB6BE016F5F7F4F66
:1008C000C7010E946F760115110509F466C0F80191
:1008D0008081882309F461C001900020E9F73197F5
:1008E000CF01801B910B20E0F70101900020E9F778
:1008F0003197EE19FF09E80FF91F32968DB79EB7B1
:100900008E1B9F0B0FB6F8949EBF0FBE8DBFEDB729
:10091000FEB731966F01B801222311F065E074E053
:10092000C6010F942E37B701C6010F94183765E042
:1009300074E0C6010F94183719A21CA221E0A70188
:10094000B501CE0181960E94B98081110AC00F9431
:10095000A10BB70188E790E20F94930B8AE00E9405
:1009600089F78BE1FE01B196DE01DC9601900D92D4
:100970008A95E1F7B601CE01CC960E942E84CE0175
:10098000CC960E94D1EFCE0181960E94D1EF0FB696
:10099000F8949EBE0FBE8DBE80CF21E081E090E036
:1009A000A3CFCE0101960E945476882309F475CF17
:1009B000BE016F5F7F4F80EB90E10E946F76011563
:1009C000110519F0C8010E94E47980EB90E10E94C2
:1009D000E47980E20E9489F76D8D7E8D8F8D98A1DC
:1009E0004AE00E941F758DE00E9489F78AE00E940C
:1009F00089F753CF0FB6F8947EBE0FBE6DBECD59AA
:100A0000DF4F0FB6F894DEBF0FBECDBFDF91CF91A1
:100A10001F910F91FF90EF90DF90CF90BF90AF901C
:100A20009F908F907F906F900895CF93C82F0F94D1
:100A3000A10B84E50E9489F78C2F0E946BAC80E2A9
:100A40000E9489F786E590E2CF910C94B1F78F92DE
:100A50009F92AF92BF92CF92DF92EF92FF92CF938D
:100A60006B017C01B42E20E030E0A9010F94052D2C
:100A700087FF07C08DE20E9489F7F7FAF094F7F834
:100A8000F094C0E060E070E080E09FE3CB1541F0BF
:100A90002DEC3CEC4CEC5DE30F946B2DCF5FF6CF6F
:100AA000A70196010F94D5336B017C010F94483553
:100AB0004B015C014AE00E941F75CC2379F1C5010E
:100AC000B4010F940A2D9B01AC01C701B6010F942C
:100AD000D4336B017C018EE20E9489F7C150F0F0A3
:100AE00020E030E040E251E4C701B6010F946B2DE5
:100AF0006B017C010F9448354B015C014AE00E9478
:100B00001F75C501B4010F940A2D9B01AC01C701EB
:100B1000B6010F94D4336B017C01E0CFCF91FF90ED
:100B2000EF90DF90CF90BF90AF909F908F900895FF
:100B3000EF92FF920F931F93CF937C018B01C2E43E
:100B40004F3F09F0C4E580E20E9489F78C2F0E9494
:100B500089F78AE30E9489F7F701608171818281B8
:100B6000938142E00E94278582E490E20E94B1F7DF
:100B7000F801608171818281938142E00E94278522
:100B800062E070E080E090E0CF911F910F91FF90C4
:100B9000EF900C9458C81F93CF93DF9300D000D0F0
:100BA0001F921F92CDB7DEB7182F60910B11709175
:100BB0000C11072E000C880B990B0F940C2D6D83D4
:100BC0007E838F8398876091091170910A11072E97
:100BD000000C880B990B0F940C2D69837A838B83FF
:100BE0009C834AEFBE016B5F7F4FCE0101960E944E
:100BF00098856091A0107091A110072E000C880BB1
:100C0000990B0F940C2D6D837E838F839887609151
:100C10009E1070919F10072E000C880B990B0F945B
:100C20000C2D69837A838B839C834FEFBE016B5FAE
:100C30007F4FCE0101960E9498856091A2101F3FC0
:100C400039F085E11802F0011124EB5FFE4E60855A
:100C500070E08AE490E20E9404FA6091A21070E0D1
:100C600085E490E20E9404FA28960FB6F894DEBF5D
:100C70000FBECDBFDF91CF911F9108952F923F926C
:100C80004F925F926F927F928F929F92AF92BF929C
:100C9000CF92DF92EF92FF920F931F93CF93DF9348
:100CA000CDB7DEB763970FB6F894DEBF0FBECDBFEA
:100CB000898B81E0809325021A821B821C821D820F
:100CC00019861A861B861C861D862CE32E873CE11E
:100CD0003F8746E4488B312C212C50E85A8B8FEB10
:100CE0008B8B198291E09887812C912C5401009173
:100CF000A0101091A110B801012E000C880B990BC7
:100D00000F940C2D6B017C01232D322D4A895B89B8
:100D10000F94052D882389F080919E1090919F104B
:100D2000A989A111E4C0B1E0B983081719070CF033
:100D300019823C2C2D2CEA8AFB8A0E948BC86B01FD
:100D40007C01DC01CB0129853A854B855C85821BC2
:100D5000930BA40BB50BB7FD2FC0D701C60188516B
:100D60009C4FAF4FBF4F89879A87AB87BC8780E086
:100D70000E94CB8582E590E20E94B1F78114910434
:100D8000A104B10409F4DFC0C501B40168577C4E69
:100D90008F4F9F4F6C197D098E099F0928EE33E014
:100DA00040E050E00F944933CA01B9014AE00E9483
:100DB00090F78AE00E9489F780E00F944C0F0E9420
:100DC0008BC86093941070939510809396109093B5
:100DD000971060919E1070919F10072E000C880B49
:100DE000990B0F940C2D6E837F838C019B01AC01BA
:100DF000632D722D8A899B890F94D4332B013C017A
:100E000020E030E0A9010F94353687FF04C077FA5F
:100E1000709477F8709481149104A104B10409F0DE
:100E200096C020E030E040E85FE3C301B2010F94D8
:100E3000052D87FF10C09885812C912C5401992392
:100E400031F082E8882E86E0982EA12CB12C8C0CF3
:100E50009D1CAE1CBF1CA981AA2391F12A813B8154
:100E60004C815D81211531054105510541F0D701C6
:100E7000C601821B930BA40BB50BB7FD21C02E81BD
:100E80003F81A8016D857E858F8598890F94D43325
:100E900020E030E040E85FE30F94052D87FD2AC095
:100EA000D701C601805A9541AF4FBF4F8A839B83BC
:100EB000AC83BD839E819D87AF81AE870F87188BE2
:100EC000809125028823B1F081149104A104B1041A
:100ED00061F0B8E8CB1AB3E1DB0AE108F108C81801
:100EE000D908EA08FB08F7FE05C0188600CF0817E6
:100EF00019071CF5209125022983222321F0109245
:100F000025020E94ADAF898163960FB6F894DEBFCB
:100F10000FBECDBFDF91CF911F910F91FF90EF904A
:100F2000DF90CF90BF90AF909F908F907F906F9009
:100F30005F904F903F902F9008953C2C2D2CEA8A83
:100F4000FB8A1982FACE8FE30E9489F732CF20E024
:100F500030E040E450E4C301B2010F943536181676
:100F60000CF079CF4601570176CF2F923F924F92E6
:100F70005F926F927F928F929F92AF92BF92CF9229
:100F8000DF92EF92FF920F931F93CF93DF93CDB732
:100F9000DEB765970FB6F894DEBF0FBECDBF8A8B64
:100FA0006B8B20914A05298B10924A0581E0809332
:100FB00025021A821B821C821D8219861A861B86B4
:100FC0001C861D863CE33E874CE14F8756E4588BD8
:100FD000312C212C80E88C8B9FEB9D8B1982A1E01A
:100FE000A887812C912C540100910B1110910C11A8
:100FF000B801012E000C880B990B0F940C2D6B017E
:101000007C01232D322D4C895D890F94052D882379
:1010100089F08091091190910A11BB89B111E4C046
:1010200021E02983081719070CF019823C2C2D2C7C
:10103000EC8AFD8A0E948BC86B017C01DC01CB012C
:1010400029853A854B855C85821B930BA40BB50BD8
:10105000B7FD2FC0D701C60188519C4FAF4FBF4F7E
:1010600089879A87AB87BC878A890E94CB858EE463
:1010700090E20E94B1F781149104A104B10409F433
:10108000E2C0C501B4016053784F8F4F9F4F6C1978
:101090007D098E099F0928EE33E040E050E00F946F
:1010A0004933CA01B9014AE00E9490F78AE00E94E0
:1010B00089F780E00F944C0F0E948BC860939410C6
:1010C00070939510809396109093971060910911EA
:1010D00070910A11072E000C880B990B0F940C2DA0
:1010E0006E837F838C019B01AC01632D722D8C89F3
:1010F0009D890F94D4332B013C0120E030E0A901FD
:101100000F94353687FF04C077FA709477F870949F
:1011100081149104A104B10409F099C020E030E0E9
:1011200040E85FE3C301B2010F94052D87FF10C0B3
:101130009885812C912C5401992331F08AE9882ECD
:1011400082E0982EA12CB12C8C0C9D1CAE1CBF1CD7
:10115000A981AA2391F12A813B814C815D812115CE
:1011600031054105510541F0D701C601821B930BA2
:10117000A40BB50BB7FD21C02E813F81A8016D8561
:101180007E858F8598890F94D43320E030E040EC41
:101190005FE30F94052D87FD2AC0D701C601805A51
:1011A0009541AF4FBF4F8A839B83AC83BD839E81A4
:1011B0009D87AF81AE870F87188B8091250288238A
:1011C000B1F081149104A104B10461F0B0EDCB1A27
:1011D000B7E0DB0AE108F108C818D908EA08FB08FB
:1011E000F7FE05C0188600CF0817190734F53091AF
:1011F00025023983332321F0109225020E94ADAFDE
:10120000298920934A05898165960FB6F894DEBF37
:101210000FBECDBFDF91CF911F910F91FF90EF9047
:10122000DF90CF90BF90AF909F908F907F906F9006
:101230005F904F903F902F9008953C2C2D2CEC8A7E
:10124000FD8A1982F7CE8FE30E9489F72FCF20E025
:1012500030E040E450E4C301B2010F943536181673
:101260000CF076CF4601570173CF0F930FB70F9352
:1012700000916E000B7F00936E0078940F930BB774
:101280000F930CB70F921F922F933F934F935F933F
:101290006F937F938F939F93AF93BF93EF93FF933E
:1012A00011240E94168AFF91EF91BF91AF919F91F7
:1012B0008F917F916F915F914F913F912F911F90EF
:1012C0000F900CBF0F910BBF0F910460F894009327
:1012D0006E000F910FBF0F9118952091A0103091C3
:1012E000A11021153105E9F080919E1090919F1079
:1012F000029624503109821793079CF490938B0631
:1013000080938A060E948BC8605E70448D4F9F4F09
:1013100060938C0670938D0680938E0690938F0653
:10132000089510928C0610928D0610928E061092DF
:101330008F060895CF93DF9310924A05C5E0D1E15F
:101340001F821E820E9497C818862C98CAE9D0E195
:101350001F821E820E946D89188680910201807210
:1013600080930001DF91CF910895EF92FF920F9348
:101370001F93CF93DF93C82F7B018A0180911706BB
:101380008130A1F40F949D0BC7010E94B1F78AE14F
:101390009FE10E94B1F7C7FD33C08C2F0C2E000CCB
:1013A000990B0E9472AC8AE00E9489F70E949A8988
:1013B000A89580916006811132C081E0809360061B
:1013C00080E8809317060E949A89D5E1D150409A0F
:1013D000E1F069E170E080E090E00E9458C8A895D3
:1013E000409868E270E080E090E00E9458C8A895BC
:1013F00068E270E080E090E00E9458C8A895E6CFCF
:1014000086E19FE10E94B1F7CECF6FE07FE1CF3F51
:1014100011F063E17FE140E0C8010F947B0EDF91A2
:10142000CF911F910F91FF90EF9008950F931F930D
:10143000CF93DF9380911A028F3708F442C08F5701
:1014400090910D11909394069923C9F12C9A2091B3
:10145000A210209393069091020121119095907211
:10146000909300018F5F80931A028091920691E021
:1014700089278093920680911902C1E0C80F8530B8
:101480000CF0C0E0823009F4D8C03CF58823D9F1D3
:10149000813009F4C6C0C09319020E946A3280915B
:1014A000320890913308009729F001979093330800
:1014B00080933208DF91CF911F910F9108952C985E
:1014C000C6CF90919406891708F02C9890919306B6
:1014D000891740F290910201C2CF843009F4C5C04F
:1014E0000CF4BEC08530B9F690919106911102C0FE
:1014F0008093910680919106815080939106882374
:1015000051F2C5E0C8CF809118028F5F80311CF482
:1015100080931802C0CF109218028091900681111A
:1015200013C080910511909106119093081180933A
:10153000071180919A1090919B1090939D10809329
:101540009C1081E080939006109206111092051174
:1015500010929B1010929A1000910711109108118F
:1015600080910B1190910C11D1E0181619062CF0F6
:1015700080910D11811101C0D0E080911F029091E6
:101580002002081719073CF444E050E261E170E2E0
:1015900080E00E94B589DD2371F080911D02909159
:1015A0001E02801791073CF443E250E260E370E2D0
:1015B00080E00E94B5898091A0109091A110D1E0A7
:1015C000181619062CF08091A210811101C0D0E0EC
:1015D00020919C1030919D108091960690919706D5
:1015E000281739073CF444E050E261E170E28FEFE4
:1015F0000E94B589DD2309F44ECF20919C103091D3
:101600009D1080911B0290911C02821793070CF091
:1016100042CF43E250E260E370E28FEF0E94B5896F
:101620003ACF88E080937B0085E480937C008091B2
:101630007A00806480937A002ECF80917A0086FDB4
:1016400027C0209178003091790080910511909108
:101650000611820F931F90930611809305111BCFE3
:1016600088E080937B0086E4E0CF80917A0086FD5D
:1016700011C0209178003091790080919A1090915A
:101680009B10820F931F90939B1080939A1003CF0F
:10169000C2E001CFC4E0FFCE2F923F924F925F9203
:1016A0006F927F928F929F92AF92BF92CF92DF9272
:1016B000EF92FF920F931F93CF93DF9300D0CDB79C
:1016C000DEB79B838A836B015A0129831801870146
:1016D00081E090E02F3F11F090E080E025E0289F2E
:1016E000F001299FF00D1124E05CFA4F84818823DA
:1016F00009F48FC0EA81FB81148215821682178259
:101700001086EA81FB8184818230B9F0833009F44C
:1017100000C1813009F067C025813681478150853D
:10172000F60160817181828193810F94052D87FD7F
:101730005AC082E0EA81FB818483EA81FB81858053
:101740009680A780B084F601C080D180E280F380CB
:10175000B801110F880B990B0F940C2D2B013C0134
:10176000809117028823F9F0F981F1111CC0809152
:101770002F088823A9F020E030E040E85EE3C301B1
:10178000B2010F946B2D9B01AC01C501B4010F9404
:10179000D433A70196010F94052D18160CF464C0DC
:1017A00080E880931502A3019201C501B4010F9452
:1017B000D433A70196010F94052D18160CF499C087
:1017C0000E948BC86B017C019101A8EEB3E00F94DD
:1017D0009D33C60ED71EE81EF91EEA81FB81C0822A
:1017E000D182E282F3820F900F900F90DF91CF9120
:1017F0001F910F91FF90EF90DF90CF90BF90AF902F
:101800009F908F907F906F905F904F903F902F9020
:101810000895F5014080518062807380A301920198
:10182000EA81FB8165817681878190850F94052D02
:10183000882309F466CFEA81FB814582568267825C
:101840007086FF24F39420E030E0A901F501608167
:101850007181828193810F94353618160CF0F12C2A
:10186000EA81FB81F4824DCF23E830EC4AEA5EE363
:10187000C301B2010F946B2D9B01AC01C501B401F2
:101880000F94D433A70196010F94052D181614F068
:1018900080E687CF20E030E040E05FE3C301B201A3
:1018A0000F946B2D9B01AC01C501B4010F94D4338F
:1018B000A70196010F94052D181614F080E471CF3E
:1018C0002DEC3CEC4CE45FE3C301B2010F946B2DB3
:1018D0009B01AC01C501B4010F94D433A70196015B
:1018E0000F94052D181614F080E25BCF10921502AC
:1018F0005ACF0E948BC8EA81FB810081118122812D
:101900003381601B710B820B930B97FD6CCF83E0CF
:10191000848344EE5FE164EF7FE189810F900F9053
:101920000F90DF91CF911F910F91FF90EF90DF907B
:10193000CF90BF90AF909F908F907F906F905F906F
:101940004F903F902F900C94B5898F929F92AF92B9
:10195000BF92CF92DF92EF92FF920F931F93CF939C
:10196000DF93EC018A01072E000C880B990B0F9472
:101970000C2D4B015C01C880D980EA80FB80A70157
:1019800096010F94353618162CF488829982AA8213
:10199000BB8210C0B801110F880B990B0F940C2D4E
:1019A0004B015C01AC019B01C701B6010F943536B8
:1019B00018165CF3DF91CF911F910F91FF90EF907C
:1019C000DF90CF90BF90AF909F908F9008952F920F
:1019D0003F924F925F926F927F928F929F92AF92BF
:1019E000BF92CF92DF92EF92FF920F931F93CF930C
:1019F000DF93CDB7DEB763970FB6F894DEBF0FBEA7
:101A0000CDBF80913F058111F3C080913E058111CA
:101A1000DEC080919006811119C063960FB6F894CC
:101A2000DEBF0FBECDBFDF91CF911F910F91FF9011
:101A3000EF90DF90CF90BF90AF909F908F907F906E
:101A40006F905F904F903F902F9008950E948E71FD
:101A50000E948BC84B015C010091091110910A1181
:101A60008091230290912402801791070CF404C204
:101A700080914405882309F4E4C160910B117091B1
:101A80000C11072E000C880B990B0F940C2D6D83F5
:101A90007E838F839887B801110F880B990B0F9461
:101AA0000C2D69837A838B839C834AE0E42EF12C8E
:101AB0000CE310E020E0AE014B5F5F4FBE016F5FB3
:101AC0007F4F88E391E10E944C8B009109111091A6
:101AD0000A118091210290912202801791070CF443
:101AE0008EC0F12CF0920D11809101119091021194
:101AF000A0910311B09104110097A105B10539F12E
:101B0000A5019401281B390B4A0B5B0BDA01C901B3
:101B1000B7FD1DC08091FF109091001108171907A3
:101B20000CF437C380910B1190910C11009739F090
:101B30000E5F1F4F0497081719070CF440C310924B
:101B400001111092021110920311109204110091D0
:101B50009E1010919F10073911050CF0F0C1809173
:101B60008C0690918D06A0918E06B0918F060097FD
:101B7000A105B10509F48CC1A5019401281B390BFD
:101B80004A0B5B0BDA01C901B7FD82C180918A065D
:101B900090918B06081719070CF4EBC26091A01006
:101BA0007091A1106115710549F0C80102969B0161
:101BB00024503109821793070CF414C310928C0639
:101BC00010928D0610928E0610928F0665C11092AB
:101BD0003E050E94E1290E94A0238EEF0E94D03092
:101BE0000E945C3180919006882309F416CF2ECF95
:101BF00041E070E060E086E59FE10F947B0E80910C
:101C0000230290912402081719070CF06ACF609103
